:020000040000fa
:080000001202040000000000e0
:020000040000fa
:100400002f4d220000be27000001880000000000e0
:10041000000e200010028800f0af2a00b002070092
:10042000090037002f4d220000be27000001880080
:1004300000000000000e200010028800e402070007
:10044000c2010700ee023200f000200040118800d7
:100450002222ef0000802800001188002342a9001a
:100460009580a9008580a9004022ef004222ef007c
:100470004422ef0000002600001c88000000240039
:10048000601c8800a0002000101c8800701c8800e0
:1004900000402000201c880000602000801c880094
:1004a00080242000401c8800a01c8800f01f200031
:1004b000501c8800b01c88008220a9002aa3ef00ed
:1004c0002ca3ef006ca3ef0040002500101688005d
:1004d00010c02d0000168800d001210040168800b1
:1004e00060fc210030168800400020007016880053
:1004f000000025006016880000102000a01688006b
:1005000040b023009016880000002000d01688001c
:1005100000042000c0168800c003200000178800d7
:1005200040152000f01688000020240030178800b5
:100530000008200020178800000320002008880001
:10054000800888001428ef00c382af002100370024
:1005500004fa2f00a202070089020700d6a2a90010
:100560008680af000300370084e0af001900370039
:10057000fbff3700900207008680a90001e02700fa
:1005800031407800220720000284e7001100370084
:1005900031407800520720000284e7000d00370048
:1005a00031407800e20620000284e70009003700ad
:1005b000314078001d020700120220000284e7008b
:1005c00004003700f0af2a00450207008002070050
:1005d0007a0037006a0207007d0207005b0107000e
:1005e000870232002342a8001002070020042000e6
:1005f000f8010700f0042000f6010700f0042000d5
:10060000f401070040052000f2010700e00320008c
:10061000f0010700e0032000ee010700fc010700e5
:10062000f00320001428b60055020700c842ae00af
:10063000050037008460af001428a90005e1ae0072
:1006400005e1a800080037001428a80000032000d6
:10065000200888008460a9000000200000088800ad
:10066000f0ff2f0010088800a0408000f003b200c7
:10067000daff32002222af002222a90010118000ee
:100680002202af000b0037008680ae00e7ff370084
:10069000490207008680a90001e027003140780068
:1006a000f00fb200e0ff3200f14088001aa8ef001e
:1006b0000300370040020700301180001a28ef00c5
:1006c000f10120000100e100d7ff3900a105200061
:1006d0000100e70055003700710520000100e70028
:1006e000fe003700510520000100e7002601370019
:1006f000f045b200210520000100e700b0003700fe
:10070000b6ff3200310520000100e700710037001c
:10071000310420000100e700570037006105200088
:100720000100e70024003700110520000184e700e4
:10073000aaff37005e010700db010700f00fb200df
:10074000f10f20000100e7000200370014e8a800c4
:10075000a2ff3700d4010700f1ff2f000100e700de
:1007600002003700f0ff2f00dd01070050042000d9
:1007700098010700800720009601070090062000de
:100780009401070040072000920107002004200088
:1007900090010700c00420008e01070097010700a8
:1007a0000000eb00d14080000180e700f401070069
:1007b0009b010700120237003d01070000052000e1
:1007c000840107009004200082010700300420000b
:1007d00080010700300320007e0107003003200065
:1007e0007c010700100420007a01070000022000ad
:1007f0007801070060052000760107000002200054
:10080000740107002003200072010700e0022000ad
:1008100070010700000320006e0107002003200084
:100820006c0107007a0107006cff37002001070008
:10083000028020001240900081c7b3000184e700cd
:1008400066ff3700441180001240780021c3b300d6
:100850000104e700f400200031c3b3000104e70005
:100860007400200041c3b3000104e70034002000fd
:100870004411880059ff37000d0107000480200053
:10088000b4417800f345b20021c5b300011ce70074
:100890000c00370071c5b300019ce7004fff370023
:1008a0000000eb0034417800280107000100a60099
:1008b000fcff37000000e00001003a00f0ff2f00cd
:1008c00087010700780107006f010700500107004a
:1008d00042ff3700f60007008001eb000480200093
:1008e000b44178000000eb003441780017010700a4
:1008f0000100a600fcff3700800278000000eb003a
:1009000034417800110107000100a600fcff370008
:10091000000378000000eb00344178000b01070071
:100920000100a600fcff370000017800f345b2008b
:1009300021c5b300011ce7001600370061c4b300f5
:10094000019ce70025ff3700950188000000eb00bf
:100950009603ba00f70fb200070040009603ba00f2
:10096000c83bde00070040003680ba00f70fb20037
:10097000070040001680ba00c83bde0007004000b8
:100980000201e900f2ff3a003f01070020010700e1
:1009900012ff370000822000060340000000eb0039
:1009a000b6437800f70fb200070040000201e900eb
:1009b000fbff3a00340107001501070007ff37006d
:1009c000bb00070004802000b44178000000eb0069
:1009d00034417800dd0007000100a600fcff37006d
:1009e000800278000000eb0034417800d700070057
:1009f0000100a600fcff3700000378000000eb00b8
:100a000034417800d10007000100a600fcff370048
:100a10000001780003007800f045b20021c5b30062
:100a20000104e7001d00370061c4b3000184e70042
:100a3000eafe3700950188001600ba000302b200f2
:100a400007003a00800378004800de00e10007005c
:100a500007007800f00fb200de0007000300370047
:100a600009010700c0022000da0007003680ba0042
:100a70000302b20002003a00d6000700030037006c
:100a800001010700c0022000d20007000201e900b6
:100a9000e9ff3a00de000700d0fe370000822000a8
:100aa000060340000000eb0036407800f70fb2006c
:100ab0000302b20002003a00c6000700030037003c
:100ac000da000700c0022000c20007000201e900ae
:100ad000f5ff3a00ce000700c0fe37000000eb0033
:100ae0008000eb000001eb008001eb000002eb0056
:100af000ac0007004801dd00aa000700f00fb200bb
:100b0000000141000000eb00a6000700f00fb2005a
:100b1000800178000082200002014000a10007004f
:100b2000005978008301e900fcff3a000404e0006a
:100b300002003a00100420000200370030042000b8
:100b400014c8a800a3000700b7fe3700d682a8008b
:100b5000d50007001408a9001448a900a15a2500cf
:100b60000100e7001408a800f1af2a000100e70027
:100b70001448a800c842ae001428a800a040800075
:100b8000f003b200000006000000eb008000eb0064
:100b90000001eb008001eb000002eb008100070088
:100ba000f00fb200b04088007e000700c800dd00f2
:100bb0007c000700f00fb20000804000c0408800b9
:100bc00078000700f00fb200000178007500070000
:100bd000c800dd0073000700f00fb2008081400004
:100be000700007000404e000d4ff3a00b040800029
:100bf0000200e100d1ff3a00c04080000300e100a4
:100c0000ceff3a00b040800090018800c0408000d4
:100c10000008bb0020042400003b88004200f800cc
:100c2000000e20004220b70050052000303b880015
:100c3000a00a2000303b880061e7a8000000000007
:100c4000000000004200f900b040800090018800e0
:100c5000c2408000018220008300200004042000a4
:100c600010002400003b88003109bb003199bb0013
:100c70000402e900fcff3a004200f800000e2000e8
:100c80004220b70050052000303b8800a00a200019
:100c9000303b880061e7a800000000000000000071
:100ca0004200f9008301e900ecff3a00a1ff3700a0
:100cb00043012000028020000059eb008301e9007d
:100cc000fdff3a00a3002000028020000400200065
:100cd000c30007000c00070084e0af00000006001e
:100ce000010020003108880084e0a9000059780044
:100cf000d1c0b3000104e700020037008301e9001e
:100d0000f4ff3a00000006001a08e20009003a0069
:100d100084e0af00000006002222af002222a900da
:100d2000101180002202ae00f9ff370026c2bf007a
:100d300000000600811f7800f140800031407800fb
:100d4000f1408800cf00780000000600fac2b3002e
:100d50000a14e600110037009ac3b3000a14e60033
:100d600008003700f245b2007ac4b3000a94e600e6
:100d70000a0037000ac4b3000a14e600070037006f
:100d80009240b000f200b2000a0120000a80b800d0
:100d9000000041008000eb00000006001100200070
:100da0000000060011e1a900f0ff2f006008880094
:100db000000020003008880084e0a90011e1a800ac
:100dc000d1ff070084e0af000000060000424200af
:100dd000000006002322af00feff3700201188002c
:100de000811f7800e140800080587800e140880051
:100df0008058eb00cf00780000000600801f7800cc
:100e000000022000f3ff07004f00780000000600fa
:100e1000a0002000efff0700d0002000edff07003a
:100e20002302ae00feff370000000600811f78009d
:100e3000801f7800800078000040d3000040d3007d
:100e40000040d3000040d300f000b200f100b20037
:100e50006a04e100010033007000b0000003b0003c
:100e6000dcff0700010078006a04e10001003300a4
:100e70007000b0000003b000d6ff07004f007800fc
:100e8000cf00780000000600801f78000080fd0081
:100e9000e6ff07004f007800801f7800e3ff07009f
:100ea0004f007800000006000000eb008000eb001f
:100eb000820f200092018800020120001200ba0077
:100ec000820f200092018800220120009200ba00c7
:100ed000c808dd00f00fb20001004000000006006d
:100ee000dc62a800801f7800820f20009201880039
:100ef000020120000049bb0000002400003b8800e4
:100f00004200f800000e20004220b70050052000eb
:100f1000303b8800a00a2000303b880061e7a80031
:100f200000000000000000004200f9004f007800bf
:100f30004800de00820f200092018800220120007c
:100f40000049bb0000002400003b88004200f8007c
:100f5000000e20004220b70050052000303b8800e2
:100f6000a00a2000303b880061e7a80000000000d4
:100f7000000000004200f900dc62a9000000060049
:100f80008480a90085c0a90041e2a8004012800029
:100f90008540a90040c2a9008de3a80081e3a80014
:100fa00083e3a8008680a90000e027000058eb003a
:100fb000d6a2a80000000600d6a2a9008de3a900d1
:100fc00081e3a90041e2a90001000700000006003a
:100fd00001c02700e14088008048eb0000000600c7
:100fe00011e1a900f0ff2f006008880004007800dc
:100ff0003008880084e0a90011e1a8000000060084
:10100000840b0400000000001a55040002000000d8
:101010001a550400020000001a55040002000000e6
:101020001a550400020000001a55040002000000d6
:101030001a550400020000001a55040002000000c6
:101040001a550400020000001a55040002000000b6
:101050001a550400020000001a55040002000000a6
:101060006c390400010000006c3d04000100000028
:101070001a550400020000001a5504000200000086
:10108000303a0400010000001c3a04000100000096
:101090001a550400020000001a5504000200000066
:1010a000ea370400010000001a55040002000000a5
:1010b0001a55040002000000803d040001000000f9
:1010c0001a550400020000001a5504000200000036
:1010d0001a550400020000001a5504000200000026
:1010e000943d04000100000084370400010000006a
:1010f0001a550400020000001a5504000200000006
:101100001a550400020000001a55040002000000f5
:1011100018390400010000001a5504000200000004
:101120001a55040002000000ce390400010000003e
:101130006a380400010000002a38040001000000a1
:101140001a550400020000001a55040002000000b5
:101150001a550400020000001a55040002000000a5
:101160001a550400020000001a5504000200000095
:101170001a550400020000001a5504000200000085
:101180001a550400020000001a5504000200000075
:10119000a0380400010000001a55040002000000fd
:1011a0001a550400020000001a5504000200000055
:1011b0001a550400020000001a5504000200000045
:1011c0001a55040002000000f43904000100000078
:1011d0001a550400020000001a5504000200000025
:1011e0001a550400020000001a5504000200000015
:1011f000383d040001000000523d040001000000e1
:101200001a550400020000001a55040002000000f4
:101210001a550400020000001a55040002000000e4
:101220001a550400020000001a55040002000000d4
:101230001a550400020000001a55040002000000c4
:101240001a550400020000001a55040002000000b4
:101250001a550400020000001a55040002000000a4
:101260001a550400020000001a5504000200000094
:101270001a550400020000001a5504000200000084
:101280001a550400020000001a5504000200000074
:10129000c064040000000000cc64040000000000f2
:1012a00014650400000000006e65040000000000ea
:1012b0007e650400000000008e6504000000000050
:1012c000b865040000000000e666040000000000ad
:1012d0006c67040000000000c2670400000000000a
:1012e000347004000000000086700400000000005c
:1012f000d8700400000000000e740400000000001c
:101300006074040000000000b274040000000000db
:1013100018750400000000006a7504000000000059
:101320007c75040000000000ce7504000000000081
:10133000de750400000000004c7604000000000090
:101340009e76040000000000f0760400000000001b
:101350009877040000000000ea7704000000000015
:10136000d0b5040000000000eab504000000000051
:10137000d6b60400000000006eb5040000000000b6
:10138000f8b70400000000003eb8040000000000b0
:10139000a6b80400000000002cb904000000000002
:1013a00082b904000000000028ba04000000000018
:1013b000c0bc0400000000003abd040000000000b2
:1013c0001abe04000000000044be0400000000003b
:1013d00078bf0400000000001cc0040000000000f2
:1013e000b6c0040000000000c2c0040000000000fd
:1013f0004cc104000000000058c1040000000000bf
:10140000d8c104000000000006c204000000000073
:1014100024c204000000000062c2040000000000ba
:1014200080c2040000000000aec304000000000001
:101430002cc404000000000050c4040000000000a0
:10144000ecc8040000000000b6c904000000000061
:10145000a0ca04000000000084cb040000000000cb
:1014600022cc040000000000f6cc040000000000c4
:1014700046cf0400000000007acf04000000000006
:10148000a6cf040000000000dacf04000000000036
:1014900038d3040000000000b8d3040000000000ae
:1014a00096d40400000000006ad50400000000008b
:1014b00092d504000000000070d604000000000077
:1014c0009ed6040000000000dcd6040000000000ee
:1014d00060d704000000000050d8040000000000a5
:1014e000d8d904000000000038db04000000000030
:1014f00092db0400000000000edc0400000000008d
:1015000094dd040000000000d4dd040000000000b1
:1015100062de0400000000001cdf04000000000088
:1015200006e00400000000007ae004000000000073
:10153000c4e0040000000000ece104000000000032
:1015400064e204000000000022e304000000000048
:10155000d8e304000000000052e504000000000091
:1015600064e604000000000048e9040000000000f8
:10157000b4ea0400000000005aec0400000000007f
:10158000bced04000000000052ef04000000000069
:10159000d4ef0400000000004af004000000000046
:1015a00086f004000000000022f1040000000000aa
:1015b0008ef10400000000004af204000000000068
:1015c00070f204000000000050f30400000000006e
:1015d0009af304000000000006f40400000000007c
:1015e000e0f40400000000004af5040000000000e0
:1015f000b6f6040000000000dcf704000000000064
:1016000064f9040000000000c804040001000000a8
:10161000f0040400010000000606040001000000c0
:101620003a060400010000007206040001000000f8
:10163000c206040001000000da08040001000000f6
:101640001409040001000000ee0a0400010000007b
:10165000480b040001000000ce0b04000100000054
:101660003e0e040001000000a80e0400010000006e
:10167000be3f0400010000006040040001000000c3
:101680009c4004000100000026430400010000000b
:101690004243040001000000604604000100000015
:1016a00086470400010000008e470400010000008e
:1016b000844a040001000000004b04000100000007
:1016c0009c4b0400010000008e4d0400010000004e
:1016d0003a4e040001000000cc4e0400010000005e
:1016e00010480400010000005850040001000000f0
:1016f000203c040002000000843c040002000000c2
:10170000a6400400010000002f4d220000be27006b
:1017100000018800000000000c00070020342500b4
:101720002100200011000700000020000000e00060
:101730000200320000000200000000001a870200d0
:10174000010000000040da000000fe004440a90053
:10175000801921000000e00003003200400020005a
:10176000a00188004440a800000006009101880004
:10177000800078000000eb0015003700e280400098
:1017800032a0b4009101ba00e280400032a0b4005f
:101790009102ba00e280400032a0b4000002eb00e7
:1017a000472bde00f507b200602ce10004003a0090
:1017b0000059eb008301e900fdff3e000400370003
:1017c0006128e100010032000082eb000400070004
:1017d0001101ba000200e000e8ff3a000000060034
:1017e0003159ba008301e9000c0032002159ba00d6
:1017f0008301e900080032000400e00003003a0021
:10180000e280400032a0b400f5ff370011d9ba00e1
:101810008301e900faff3a008100e800e18040001e
:1018200032a0b400000006000003b1000b00350038
:101830009000b100080034008000b10007003500be
:101840005000b10004003400b001b10003003500c5
:101850005000b10001003c00100005000000050030
:10186000800078001106b100030035009101b1003d
:1018700001003c000050a100000006001004b1006f
:10188000070035009001b100040034007000b10081
:10189000030035009001b10001003c00100005007c
:1018a000000005006900e100040035006d00e10062
:1018b000030034000002b100010032000000050006
:1018c00010000500020ab900001bb9000200b800b0
:1018d000810042008100430000000600889fbe0096
:1018e0008a9fbe00010578000100e0000400350079
:1018f00008003c000000e000200032000500370036
:1019000060001000e080180002003b0001f02c0095
:101910001a0037000004be006011b8006b092000f7
:101920000982cf00020039000882cf000441b000d4
:10193000694252000e00320008003b0082817100b3
:10194000610164008904d1000884d3008b05e8009c
:101950000442e800f9ff3a0005003700080444009b
:1019600089844c008b05e9000442e900fbff3a0042
:10197000750307000af0a70001f0a0004f05be00a4
:101980004f04be000000060003f0a200889fbe00c6
:101990008a9fbe008c1f78009103070098033300d4
:1019a0006450e1004f0032006420e1005200320038
:1019b00003826c0007003b000905d0000306d0003d
:1019c000820f54000c065d00020039000200320054
:1019d00089017800030678008582550004003d00e7
:1019e0000003fd008103fd008502ea008b854200b3
:1019f000840f720002003b0060001000e0801800bd
:101a00006011b8000005eb007a28e1000a003900f7
:101a100006007800c75ddd00f707b200878075001b
:101a20002d003700828171000a0178006105600095
:101a30008180d1000080d3008502e900f9ff3b00de
:101a4000060440008784480002003b006004140044
:101a5000e0841c000988a300070032008a8171001d
:101a600082817100610164008904d1000884d3007f
:101a70008b05e800170037000978a30013003a002f
:101a80000b00e000130034008b05e900080444005b
:101a900089844c000a4474000978a3000d003a00c0
:101aa0000b00e000070034008b05e9000804440047
:101ab00089844c0001003a000b0020000978a30043
:101ac000f7ff32000001eb00020037008281710055
:101ad0000a0178001c0307000cf0a70001f0a00029
:101ae000500337006420e10002003a00838f6c004d
:101af000500333000801be000200be004903370056
:101b0000889fbe008a9fbe008c1f780034030700a8
:101b10003b03330003866c006450e1002400320074
:101b20006420e100270032006150e1002200320011
:101b30006120e100210032008b854200eb07b100fb
:101b40000134b800003ab8000804420089844a0011
:101b5000013ab8000030b8008880400009014a000e
:101b60000400330000004000818048000201490069
:101b70008b05e900c909dd00830170000100320016
:101b800013002000c814de004814dd004709de0001
:101b90001200b200c808de0008847000ea020700e4
:101ba00001f0a1000cf0a70001f0a0001d03370018
:101bb0006120e1001f0332000801be000200be00e8
:101bc000f7ff37006150e100fcff3a0019033700ce
:101bd000889fbe008a9fbe008c1f7800000307000c
:101be0000703330003866c006450e1002e003200ce
:101bf0006420e100330032006150e1002f00320028
:101c00006120e1003100320085855500eb07b0000e
:101c100009002000080420000500370008044400e3
:101c200089844c000a0031000603430087834b007f
:101c30000001530081815b00f8ff33000203be0006
:101c40000800a0000804440089844c00f6ff390015
:101c5000c639dd008301730001003200130020004b
:101c60008904d1000884d3000998a300050032003c
:101c70000800a7000300a0008904d1000884d30055
:101c80008b05e8008904d1000884d3000001eb0033
:101c90000281d200ac02070001f0a1000cf0a70005
:101ca00001f0a000df0237006420e100e102320011
:101cb0000801be000200be00f7ff37006120e1000e
:101cc000dc0232006000b800f3ff370000002000a3
:101cd00001f82700f0ff37000001be00d80207001e
:101ce0000470a70003f0a10003f8a30013003a005a
:101cf0006509b10010003200090035006928e100d3
:101d0000020035000100280000000500000040002e
:101d1000818048008502e900fcff3a0000000600cf
:101d2000f88f4200050035008100d1000080d3000b
:101d30008502e800fcff3a00000006008000eb008e
:101d4000000005001400fa00889fbe008a9fbe00b4
:101d50008c9fbe000005be000206be006800470062
:101d60000c90be000a90be00ca0207006400e100a9
:101d70001a00320016003e006100e1001a00320035
:101d80006e049000fe0490000e0b90009e0b9000dd
:101d90006011b8009e0590000b38b100d5012000fd
:101da00082817100610164008703d1000683d30042
:101db0008984d3000884d3008502e900f8ff3a0043
:101dc000610207000df0a70001f0a000ec0237004f
:101dd000f1ff2700f0ff2f00e902370001f827008c
:101de00000002000f7ff37006000b800f5ff370063
:101df000f4ff2f00e70237000001be009002070049
:101e00000470a70003f0a1006509b10016003200bc
:101e10000d0035006828e10006003500f0ff2f00b6
:101e2000f1ff27000300e00013003b000100280041
:101e30000000050000004000818048008502e900a4
:101e4000fcff3a0008003700f88f420002003c0017
:101e50008000eb00000005008100d1000080d3006d
:101e60008502e800fcff3a000300e00002003b00ae
:101e700060001000e0801800000006008103780078
:101e80006f0207000001be006000b8000478a300e4
:101e900013003a006220e10015003e000d003900f9
:101ea0008301d1000281d3008180d3008301d1005e
:101eb0000281d3008180d3008301d1000281d3004d
:101ec0008180d3000538b000c42add00f300b200e1
:101ed0008381720007f0a70003f0a0000000060055
:101ee000f3ff2700f2ff2f006110b900fbff37005e
:101ef00003ff2700f7ff37002800fa00889fbe0085
:101f00008a9fbe008c9fbe0003866b00880207007c
:101f10006400e100440032006408e1004a0032003d
:101f20006100e100460032006108e1004900320032
:101f3000ec0647006000b8003d02be003d03be0055
:101f4000f48657006011b8003d04be003d05be0098
:101f50007d0320000b0037000000a0008d06e90083
:101f6000130032000402420085824a0006034b003f
:101f700087834b0000004000818048000201490037
:101f8000838149000802520089825a000a035b00db
:101f90008b835b00f0ff3b000802420089824a000d
:101fa0000a034b008b834b008d06e900edff3a00de
:101fb0008482720086827200f707b2008782720004
:101fc00001003200150020001e0490003e0b90001e
:101fd00006035400e63fb0000368a3000700320088
:101fe0000000a7000500a0008301d1000281d300fa
:101ff0008180d3000080d3000603e8008301d10074
:102000000281d3008180d3000080d3000002eb0066
:102010000482d2007a02070003f0a1000cf0a700ae
:1020200003f0a00056023700640247006408e10094
:10203000500232003400be003401be00f6ff37000b
:102040006108e1004b0232006011b8006000b80086
:10205000f1ff370003ff270002002000fbff3700dd
:10206000140020004b0237002800fa00889fbe00b1
:102070008a9fbe008c9fbe0003866b002c02070067
:102080000028a30064003a000128a30067003a007a
:102090000008a30062003a000108a30065003a00ae
:1020a0001e009000be08900081064000ed3fb10088
:1020b000f4805700ee019000111ab8008e099000cc
:1020c000311bb8009e099000311cb800511db800aa
:1020d000f485570046000700fe0190003a00070013
:1020e0008b85e8003e0007008e0990004000070045
:1020f000ee019000340007008b85e80038000700ef
:102100008e099000400007009e0990001b18b8003f
:10211000890440000a854800fe0190003400070051
:102120008b85e80038000700ee01900030000700c2
:102130008e0990001b18b800890440000a854800e9
:102140000a98a30008003a000402420085824a006f
:1021500006034b0087834b0008044c0089844c0025
:102160000a054d008d06e900848272008502730025
:102170004c3add008502720001003200150020009b
:10218000443ade001400b2004538de00cb45dd00e5
:102190000b007000c540de00cb4ddd008b80700071
:1021a0004549de00cb55dd000b017100c551de0055
:1021b0000d0378001202070003f0a1000cf0a70045
:1021c00003f0a000ee0137001b18b80085024000a4
:1021d00006834800e0834b0060044c000700370092
:1021e0001b18b8000603400087834800faff370039
:1021f0001b18b8008703400008844800e0844c00a6
:1022000060054d00000006001b18b80008044000df
:1022100089844800faff37000108a300d5013a007d
:102220005800be005801be00e3ff37000008a300bd
:10223000d0013a0009047800f9ff37002800fa00bd
:10224000889fbe008a9fbe008c9fbe000706780054
:10225000878669000c003b0003047800870478003f
:1022600008f0a10009f0a100840f5000858f5800ec
:10227000860f5900890f5c00030033000cf0a200a8
:1022800001003a000cf0a100a90107006400e10080
:102290005f003200780147006408e100610032000d
:1022a0006c014700748557003200be001201be0069
:1022b0003a04be001a05be001e039000be0a90003c
:1022c0008503530006003d000004fd008104fd006d
:1022d0000205fd008305fd008703ea000503780081
:1022e0000df8a3000400320060041400e0841c0018
:1022f00060051d00e0851d006022b8007d03200000
:102300000d38e1008006eb000b0039004433dd009e
:10231000f300b20083017300390037008482720039
:102320000d027800e10664008b85d1000a85d30098
:102330008984d3000884d3008703e900f7ff3b00ba
:1023400008004000898048000a0149008b8149004b
:1023500004003b0060001000e080180060011900dc
:10236000e08119000358a300090032008d82720039
:1023700084827200610260008301d1000281d30077
:102380008180d3000080d3000603e8001b003700e3
:102390000348a30017003a000600e00017003400cd
:1023a0000603e9000d00a3000000480081804800fa
:1023b00002014900838149000348a3000f003a004d
:1023c0000600e000090034000603e90000004000b8
:1023d00081804800020149008381490001003a00e0
:1023e0000003eb000348a300f5ff32006022b800b1
:1023f000020037008482720061826600800107005b
:1024000003f0a1000cf0a70003f0a0005c0137006e
:10241000640147006408e10002003a000df8a300df
:1024200054013a003200be001201be0054013700d0
:102430001400fa00889fbe008a9fbe008c9fbe00d9
:102440000004be000205be00680047000a90be00fe
:102450000890be000f0107000070a7000bf0a1005c
:102460000bf8a30016003a009e02900030432000b3
:1024700080825200b0fe2f000028e1000d003c00d9
:10248000b0fc2f000028e1000d0034001e09900070
:102490008e0890007e0090000501b0000201d1007e
:1024a0008180d3000080d3008502e800fbff3a0062
:1024b0003301370001002800000020003001370000
:1024c0006000b8002e0137001400fa00889fbe009b
:1024d0008a9fbe008c9fbe000004be000205be00a5
:1024e000680047000a90be000890be00e90007009f
:1024f0000070a7000bf0a100304320009e02900066
:1025000080825200b0fe2f000028e10011003d0043
:10251000b0fc2f000028e100150034001e099000d7
:102520008e0890007e0090000501b0000201d100ed
:102530008180d3000080d3008502e800fbff3a00d1
:102540000b00e0000e013b0060001000e08018006e
:102550000b013700f0ff2f00f1ff27000b00e00018
:1025600007013b00010028000000200004013700a3
:102570006000b8000201370007f0a2002fff37000b
:102580004f89de008201780049013700809feb000f
:102590007e0107008f87e9000000e00000000600d0
:1025a0008f1fd100790107008f87e9000000e0004c
:1025b00000000600839f68000100e00002003d006b
:1025c00060001000e08018000300e00002003d0001
:1025d00060011100e0811900050007004f00e000d4
:1025e00002003b0060001000e080180000000600c0
:1025f0006022b800060220000000d0008180d200d6
:102600000482d2008582d2000000a00002025200a3
:1026100083825a00030031000202420083824a0092
:102620000000a1000603e900f3ff3a0000000600e5
:10263000040020007e013700811f78000100e000c7
:1026400002003d0060001000e08018000300e00080
:1026500002003d0060011100e08119003302070013
:102660004f00e00002003b0060001000e080180016
:1026700000000600889fbe008a9fbe008c1f780065
:102680000004be006e0007000478a30026003a0094
:102690006120e1002500320009f8a30025003a007e
:1026a0006420e10021003200f507b1000508a30015
:1026b0000200320000004000818048006044b80001
:1026c000031020000200200000004000818048002c
:1026d0000805440089854c000a0541008b854900a6
:1026e0000a0550008b855800030033000a00be0025
:1026f00002047400838474008301d1000281d3003a
:10270000830f7100f0ff3a008904d1000884d300e0
:102710006001490082017800c1adde00fb07b00016
:10272000090007003f0037000960a0000800be0054
:102730003c0037001202200002408800f0ff2f000a
:10274000f1ff27003700370081002000618055002d
:102750000b003d000b00200061fe2f000100e10096
:102760001d00340082817100610164008904d10080
:102770000884d3000000e800faff3a00710020004e
:102780006100640003007000020060000900320074
:1027900061044400e0844c000988a5000500320073
:1027a0008b05e8006808e10002003a008904d100c6
:1027b0000884d300f20f20000258e10005003d001c
:1027c000c75ddd00f907b200898075000800780058
:1027d000000006000bf827008b00780000000500c1
:1027e0000004be00160007000003be000405be0082
:1027f0000200be0012000700844f750000000600b2
:102800000200be006450e100050036006420e100d3
:10281000020036000968a30001003a000800be006b
:102820000160a0004f0678004f05be004f04be00b7
:1028300000000600f0ff2f00f1ff2700f9ff37002e
:10284000c70ade00f107b200f50fb200080032003f
:10285000e1cf4200020032000170a0002400050018
:10286000810f7000010032000408050044000500db
:10287000810f700002003a00140005008502e90093
:102880000000400081c04800fcff3b000170a00038
:1028900024000500800078005002be005003be00f6
:1028a0004439de00f700b200f37f2000030161002d
:1028b000090032000218e10016003a00850172009a
:1028c00083017300838173000008200015003a0023
:1028d000400020001300370085017200830173005f
:1028e0008381730005003a0004a8be0006a8be005c
:1028f000100020000b0037000201e9000402420032
:1029000085824a0006034b0087834b000748a300db
:10291000f9ff32000740a00004a8be0006a8be00d0
:10292000200020008000980092009800000006001f
:10293000680447000294be000094be00fc044700f7
:102940008694be008494be0009007800d1ff070081
:1029500008007800cfff070099007800814f7000d1
:102960000b003b000800be00730107004f00b100e0
:1029700003003700f3ff2700f2ff2f006110b900ba
:102980004f06be004f05be004f04be000080fa0097
:1029900000000600889fbe008a9fbe00841f78004a
:1029a0008fff07004f00780011003300f0ff2f0069
:1029b000838f6c0006003b00040565000a00a70039
:1029c0000800370009f0a6001000200008003700ba
:1029d000820f5400838f5c00030039001000200038
:1029e00001003e000000200009f0a7000000ea00fe
:1029f0004f05be004f04be000000e00000000600ce
:102a00001800200057002000080453000d003d006e
:102a10000600200097fc2f000740e1001e00340054
:102a200084827200610260008301d1000281d300c0
:102a30008180d3000080d3000804e800f8ff3a004a
:102a40004700200061046000050474000404640071
:102a50000d00320061004000e08048006001490044
:102a6000e081490003b8a500070032000603e80032
:102a70006538e10004003a008301d1000281d300ef
:102a80008180d3000080d300f87f20000830e1006f
:102a900003003500080378006000b8006011b8003a
:102aa0004433dd00f300b200830173000000060030
:102ab000889fbe00830478000300e0002c003500ee
:102ac00003003c0000827000040271002600320006
:102ad00036432000c50020008383cf000a00390060
:102ae0000541b1008283cf00070039000541b100e4
:102af0008183cf00040039000541b1008083cf00fd
:102b0000010039000541b10085c353006022b800bf
:102b1000120032000a003b008482720061026000f1
:102b20008301d1000281d3008180d3000080d300d3
:102b30000603e8008743e800f7ff3a000700370084
:102b40000000400081804800020149008381490063
:102b50000603e9008743e900f9ff3a00a8ff0700f0
:102b600009f0a70003f0a0004f04be00000006001b
:102b700060001000e080180060011900e081190079
:102b8000d3ff3b00033e2c00f7ff3700889fbe00b9
:102b90008a9fbe008c9fbe000404be000605be00d6
:102ba000809fbe00829fbe00f100070004067800ef
:102bb0000800be000a01be00ed0007008406780090
:102bc0004f03be004f02be008d4f76007fb09700ce
:102bd00013003300f0ff2f008b8f6b0006003b00cb
:102be0000d0666000c00a7000a00370007f0a600db
:102bf000100020000a003700880f5200898f5a0009
:102c00008a0f5b008b8f5b000300390010002000ef
:102c100001003e000000200007f0a7000000ea00cd
:102c20004f06be004f05be004f04be000000060068
:102c30000800fa00889fbe008a9fbe008c9fbe00dd
:102c40000406780003f0a7000cf0a0000004be000a
:102c50000205be00c60007006420e100af003e0090
:102c6000ab0032000bf0a1000800be000a01be005c
:102c700007ff2300060020006022b80043fe070083
:102c8000a3003c000800be000a01be0067e4230068
:102c9000e6092a00f5672600d4bc230040fe0700a1
:102ca0000800be000a01be007d00350007fe2300bb
:102cb00006002000050020000400200033fe07006d
:102cc00008003c000800be000a01be000802be0069
:102cd0000a03be00e4fc0700009fbe000297be008e
:102ce000160037000c10a20003ff23000200200092
:102cf0006000b8000802be000a03be001efe070006
:102d000007fe23000600200005002000040020002c
:102d1000d5fc0700009fbe000297be00a60007007a
:102d200007002c0006002000050020000400200001
:102d3000cdfc07000004be000205be003e00be0040
:102d40002e01be0077032c00862e2d0095ef260065
:102d5000f461280039fd07003e02be002e03be00cc
:102d6000c1fc070027062400c6e72d009565290051
:102d700004c7210031fd07003e02be002e03be0045
:102d8000b9fc070077072c00e6dc2d0065c52f0095
:102d900084842a0029fd07003e02be002e03be00e7
:102da000b1fc0700a7072400f6242100e50121005b
:102db00034842b0021fd07003e02be002e03be001e
:102dc000a9fc070047062c00066c2800b5e223008a
:102dd000c47c280019fd0700809fbe00829fbe00b2
:102de00063fe2b00d2bb2400615e2b0050e6210065
:102df0003e02be002e03be009bfc070047022400db
:102e000076e12400c54e2600749223000bfd0700d6
:102e10003e02be002e03be0093fc070037042c00c8
:102e2000c6822d00659a2a00f4a92d0003fd070033
:102e30003e02be002e03be008bfc0700c704240028
:102e400076aa2900a5602300a4482d00fbfc0700fa
:102e50003e02be002e03be0083fc0700b7032c0019
:102e600056e52500a5832a0024a62000f3fc0700d0
:102e70003e02be002e03be007bfc07004f03be00d7
:102e80004f02be001cfc07000802be000a03be0081
:102e900075fc07000802be000a03be00e7fc07003d
:102ea0000c00a7000900370097ff2300b61f22007f
:102eb0004544250084d122000c10a700dffc070048
:102ec0000cf0a70003f0a200100037000cf0a700e0
:102ed0000200370003f0a20006003700970024002c
:102ee000b61f22004544250084d122000c10a60004
:102ef0000500370097ff2300b61f22004544250038
:102f000084d122000c10a700ccfc07009cfe3700e7
:102f1000f3ff2700f2ff2f006110b9000330a0007b
:102f20001402200004408800f8ff3700b0fd0700bd
:102f30000400be0000000600e48240001078a300f8
:102f400007003200640240001178a3003400be0084
:102f50001401be00040032000330a7000000060088
:102f60003500be001501be000330a00000000600c1
:102f700005ff270005826100070032000428e100f8
:102f800001003200240005000600070001003a009d
:102f9000440005000408050002000700f9ff3a009c
:102fa000140005006f8261008102700085027100cb
:102fb00085027200000006001400fa00889fbe001f
:102fc0008a9fbe008c9fbe000004be000205be00aa
:102fd000680047000a90be000890be002dfe070062
:102fe0000078a3003d003a006100e1003c0032009f
:102ff0000bf8a3003d003a006400e1003800320005
:103000006c0347001e009000f03fb1003602be0086
:103010001603be000008a3000400320004024200b0
:1030200085824a0006034b0087834b0010079800f7
:103030008e1f78006000b8006011b8005c002000ae
:103040006d0120006e002000020037008d86e9002f
:10305000fc0020000402420085824a0006034b0067
:1030600087834b000004400081844800020549002a
:10307000838549006060e1001d60ad0008045200d6
:1030800089845a000a055b008b855b0003003900c8
:103090001e60ad000802be000a03be000c06e90077
:1030a000ecff3b000e87e900e8ff3b004f0778008c
:1030b00061026000840278008301d1000281d300a4
:1030c0008180d3000080d3001e03900041b3de0056
:1030d000f63fb0004afe070029fe37000b30a00083
:1030e0000800be000a01be0025fe370012022000c3
:1030f000024088001ffe3700881f78000004780017
:103100005001be004000be00040040008580480021
:103110000601490087814900009cbe000294be0060
:103120000400e1000588e1000690e1000798e10055
:1031300002003100680044001008e8004f047800e5
:1031400000000600f4874700889fbe008a9fbe00eb
:103150008c9fbe008e1f78000205be000004be00da
:10316000d4b79f00e5b79f00f6b79f0087bf9f00c9
:103170000000eb00c0b79f00b0b79f00a0b79f0052
:1031800090b79f0080b79f000d042000bfb097004c
:103190004fb09700000140000000e0000f003d002c
:1031a0004f08de0000007100c0b79f009e000700be
:1031b00001003d0012002000a100070001003d00b9
:1031c00012002000a6000700b1000700b6000700ab
:1031d0000f004000c8ff0700220037004f08de0044
:1031e00000067100ccb79f008f00070001003d0072
:1031f000120020009200070001003d001200200094
:1032000097000700a20007000fb297009fb2970037
:103210002fb39700bfb39700a9000700000052002a
:1032200081805a0002015b0083815b0080b79f00b0
:1032300091b79f00a2b79f00b3b79f000007eb00b4
:103240009f0007000020e10001a8e10002b0e100ba
:1032500003b8e100010031001e0020000e005600fe
:10326000c0b79f004fb297000400e0000700350090
:1032700010002000010020006011b8000804700058
:10328000898470000a0571008b8571008d06e90044
:10329000beff3a000400e00003003d00820007008a
:1032a0000f00400094ff07004fa897000000e000c7
:1032b00004003a000fb497009fb497002fb5970011
:1032c000bfb59700940007004f0778004f06be0077
:1032d0004f05be004f04be004f01b10000000600c4
:1032e000881f780018002000881f780095ff0700cd
:1032f0008f87e9004f04780000000600801feb0074
:1033000090ff07008f87e90000000600889fbe003d
:103310008a9fbe008c1f78006e00070007003d00ea
:1033200073000700e00f5b00e08f5b0007003d00cb
:10333000320007000006eb000400370034000700ed
:1033400002003d002a0007001c0020007200070058
:10335000e3ff07000203be000002be000c00e00015
:1033600001003200220007000400be000601be007a
:103370004f0678004f05be004f04be000000060057
:10338000889fbe008a9fbe008c1f780051000700f6
:1033900005003d0056000700e00f5b00e08f5b007a
:1033a00006003d00040037001900070003003d003f
:1033b0006000b8006011b800100007005600070058
:1033c000ceff07000203be000002be000c00e000ba
:1033d00001003200060007000400be000601be0026
:1033e0004f0678004f05be004f04be0000000600e7
:1033f0006000b8006011b8000000370004025000ff
:103400008582580006035900878359000000060092
:103410000006eb00e00f5200e08f5a00e00f5b0067
:10342000e08f5b00000006000180400090b79f0025
:103430000001eb008fb097000100e00000000600e3
:103440000200700090b79f000180400080b79f008d
:103450000001eb00ffa897000100e000000006005b
:103460000200700080b79f00018040006faa9700a3
:10347000cf20de0001007000f0af9f000402420088
:10348000250007004f18de00000272000000060051
:10349000e4af9f000804440089844c000a054d00f5
:1034a0008b854d00000006003fb29700cfb2970019
:1034b0005fb39700efb3970000fe2f0000000600f7
:1034c0003fb09700cfb097005fb19700efb1970082
:1034d000000006000205be000004be00e00f500020
:1034e000e08f5800e00f5900e08f590000000600ff
:1034f0006000b8006011b8000804500089845800ca
:103500000a0559008b8559001c002000e00f52006d
:10351000e08f5a00000006000800be000a01be004d
:1035200000000600801feb0098fd07008f87e90070
:103530000000e000000006001400fa00889fbe00b2
:103540008a9fbe008c9fbe00040678000004be0067
:103550000205be00680047000a90be000890be0049
:10356000ccfc07006200e1000800be000a01be00ba
:10357000040020000b003a001e029000e43fb1005e
:103580006e009000fe0090000e0990009e099000d1
:10359000f300b20005fe2300858171000bf0a70047
:1035a00003f0a000040e7800f5fc37001400fa00c8
:1035b000889fbe008a9fbe008c9fbe000004be0094
:1035c0000205be00680047000a90be000890be00d9
:1035d000b0fc07000070a7000bf0a1000bf8a300df
:1035e00020003a009e0990000e099000fe00900015
:1035f0006e0090009e0290003443200084825200ae
:10360000dffc32000a003c00b4fc2f000428e1007b
:10361000140034008301d1000281d3008180d300e3
:103620000080d3008502e800faff3a00d4fc37009e
:10363000b40020000428e10007003c000000400026
:103640008180480002014900838149008502e90028
:10365000faff3a00cafc37000300280002002000ed
:10366000010037006011b8006000b800c4fc3700ea
:10367000889fbe000004be00060037000804e80072
:103680000000fb0089007800b5010700e10f400051
:1036900004003200184078000004e000f7ff3a0010
:1036a0000000eb004f04be0000000600881f7800f9
:1036b000e14a2200eeff070000047800e14a220000
:1036c000a0002000a6010700080078004f04780041
:1036d00000000600889fbe008a9fbe008000780020
:1036e00000c2b3000100370089007800810478002f
:1036f00039447800804f5400fbff3200e94f5400fa
:10370000f9ff3200d0c2b300804f540004003a00e9
:10371000194478008184e8001ac0b300060037001d
:103720000045eb00b0c2b300804f540002003a00e5
:10373000194478008184e8006022b8000a0037004c
:10374000a2002000030020000400be005df8070076
:103750000b4144000281fb000300200000024100f5
:1037600081824900394478000880fb000bfd2f005e
:103770000b004000e90f5000f1ff36000a04e000a2
:103780000200320060021200e0821a000400be0053
:103790004f05be004f04be00000006008000780008
:1037a0003004e000feff3a00010050000000e90094
:1037b00000000600f0874700889fbe008a9fbe0079
:1037c0008c9fbe008e1f78000006780081bf9f008e
:1037d0000100e0000300320080087800010037009b
:1037e0000c06e8001c4478000800fb002df80700d8
:1037f000800078000000e000f9ff3a00d0c2b3007a
:10380000804f540003003a000c06e8001ec0b300cd
:1038100005003700b0c2b300804f540001003a00e9
:103820000c06e800014778000000eb00a0b79f00fd
:10383000b0b79f006000b8006011b800c0b79f002b
:10384000d1b79f00e2b79f00f3b79f000e48a300d7
:1038500005003a00e0c2b3009c4f100002003a009d
:103860000e44a000300037009c4678000d00fb009d
:103870000003b100e90f50002d003e000e14a0001f
:103880000e00fb002fb19700f20f51002100320013
:103890000048a30003003200bfb197008301e90094
:1038a000b3b79f002fb097000000e800a0b79f00bb
:1038b0006022b80006002000470224004fb09700a5
:1038c000dfb097006fb19700ffb19700e6f90700ee
:1038d0000004be000205be0001cdb30001c04600d9
:1038e0000080fb00cf80de0025fb07000002be0049
:1038f0000203be000800be000a01be004ffa070026
:10390000c0b79f00d1b79f00e2b79f00f3b79f00f9
:10391000050037000048a30003003a003fb19700bc
:103920000201e800b2b79f000c06e800c7ff3700ad
:1039300050c6b30080cf5600040032000002eb00f6
:1039400050c4b30080cf560032003a008c01e8002a
:1039500093407800d0c2b30080cf500002003a00fc
:103960000e34a00003003700b0c2b30080cf500077
:1039700003003a008c81e800010037008301e80071
:103980009340780006c3b30086cf5000fbff32009f
:103990000100fb0005fd2f0005004000e90f50006d
:1039a00003003600030678000002eb001600370023
:1039b00006c050000082fb000306e8001c417800ae
:1039c0000200fb0005004000e90f50000e003e0021
:1039d0006a20b900064151000281fb00000241004b
:1039e0000386e8009c4078000100fb0005004000d1
:1039f000e90f500004003e006a21b90006c05000e3
:103a00000080fb00020240000e38a30001003200db
:103a10000402ea00bfb19700848641000fb8970006
:103a20000000e000030032000e18a3000100320085
:103a30000c0878004fb09700dfb097006fb1970087
:103a4000ffb197000004be000205be006022b8006e
:103a50006033b800d2fa07006022b8006033b800c3
:103a60000000e000ad00320030c02f00808f560013
:103a700003003d002002200000408800a70037001e
:103a800000402000808f56000e00340020022000ed
:103a9000004088000e08a30005003200f4ff2f004c
:103aa000f5ff2f00f6ff2f00f7fe2f009b003700d9
:103ab000f4ff2f00f5ff2f00f6ff2f00f7fe270081
:103ac000960037000d00e00042003d000d04ea00c2
:103ad0000e003700d4372c0045592200d69a240016
:103ae000274b25004fb09700dfb097006fb19700cc
:103af000ffb1970000f90700c0b79f00d1b79f0042
:103b0000e2b79f00f3b79f004806b10030062000df
:103b1000800f5400efff3c000e003700040020002f
:103b200005002200f6052a00272024004fb0970048
:103b3000dfb097006fb19700ffb19700eef8070074
:103b4000c0b79f00d1b79f00e2b79f00f3b79f00b7
:103b50006a045400e90f5400f0ff3c008004eb00bd
:103b60000d0037006022b800060020004702240044
:103b70004fb09700dfb097006fb19700ffb197008b
:103b8000ddf80700c0b79f00d1b79f00e2b79f00e4
:103b9000f3b79f008904e800888f5400f1ff3a00d2
:103ba0004fb09700dfb097006fb19700ffb197005b
:103bb0000004be000205be006022b800060020001e
:103bc0000701200076fa07000000e0004e003d00eb
:103bd000430037000d00e0000f003c004a003700b2
:103be000d4372c0045592200d69a2400274b2500b3
:103bf0004fb09700dfb097006fb19700ffb197000b
:103c000019f90700c0b79f00d1b79f00e2b79f0026
:103c1000f3b79f004d06b10030062000808f56009c
:103c2000efff3c000e0037000400200005002200da
:103c3000f6052a00272024004fb09700dfb0970038
:103c40006fb19700ffb1970007f90700c0b79f0059
:103c5000d1b79f00e2b79f00f3b79f00ea865600f6
:103c6000e9cf5600f0ff3e000004eb000d003700e6
:103c70006022b80006002000470224004fb09700e1
:103c8000dfb097006fb19700ffb19700f6f807001b
:103c9000c0b79f00d1b79f00e2b79f00f3b79f0066
:103ca0000804e8008d0f5400f1ff3a004fb0970070
:103cb000dfb097006fb19700ffb197000004be001e
:103cc0000205be00f4ff2f00f5ff2f00f6ff2f00c6
:103cd000f7fe27002dfa07000000e0000a0034007c
:103ce0000e08a300040032006022b8000600200085
:103cf00007012800090037006022b80006002000f4
:103d000007012000050037000e08a3000100320063
:103d10000bf0a2000802be000a03be000400be00b1
:103d20000601be004f0778004f06be004f05be00db
:103d30004f04be000f01b100000006008000eb0040
:103d40009cfe37000000fa00cfb89700688157004a
:103d5000e04a2200a90107000080fa0000000600e6
:103d6000889fbe000001780001047800b100900037
:103d70000118a3003d0032000198a30003003a009f
:103d8000180090000000e00038003a000190a00008
:103d90003104980082047800f90fb20018009000f6
:103da0000000e00002003a0028009000000c7800bb
:103db000ea8f540006003a00380090000078a30013
:103dc00003003a0088007800d0002000e4ff0700dc
:103dd0009800900058009000808f50000b00320037
:103de0000100e800100498001800780009587800d5
:103df000000c780011c0b300a04c220001487800ec
:103e0000ea8f54000600320019003700880078005d
:103e100009407800d20007008004780014003700c1
:103e2000380090000088a3001100320018019000b3
:103e3000a800900048009000327f07009800900092
:103e4000810f500004003200380090000003b300de
:103e5000300498008084eb000000eb001004980010
:103e600028009000000c7800010037008084eb00ef
:103e7000090078004f04be00000006000000fa00b0
:103e8000cfb8970068815700e04a22005b01070025
:103e90000080fa00000006000001780000c2b300b4
:103ea000010037000201e8009240780080cf500006
:103eb000fcff3200e9cf5000faff3200d0c2b3005d
:103ec00080cf500003003a000201e80014c0b300a4
:103ed000050037000042eb00b0c2b30080cf5000b5
:103ee00001003a000201e8008000eb0005fd2f0010
:103ef000040037006a08b9000080410085004000d6
:103f00000201e8009201fb0005804100e90f50002a
:103f1000f8ff36000404e000010032008100ea00ee
:103f20000100780000000600889fbe000004be006b
:103f30000d0037000900780018fe07000001780026
:103f40000800be00c90007000000e00002003a00bf
:103f500008007800090037009900fb000800e8001d
:103f60001b000700000478000800e0000200320097
:103f70001804e000efff3a000000eb004f04be0021
:103f80000000060080017800000178000100370081
:103f90000201e8001204e000fdff3a003140780021
:103fa000005978000004e000fcff3a0003007800ac
:103fb000000006000000fa00cfb8970068815700a3
:103fc000e04a22000d0107000080fa000000060010
:103fd00010417800814f5100040032000000e800d9
:103fe0000204e000faff3a000000eb0000000600c7
:103ff0000c00fa00889fbe0000047800cfb0970044
:10400000f0ff2700d0bf9f008004eb0099bf9f0006
:1040100088bf9f00a8bf9f00200c2000b0bf9f005a
:104020007881570070805700f40007000fb89700a0
:10403000094878000fb8970008045000080078007d
:104040004f04be000080fa000000060080017800e6
:104050000001780031407800005978000004e00049
:10406000fcff3a0003007800000006000000fa00a0
:10407000cfb8970068815700e04a2200df000700b0
:104080000080fa00000006000000fa00cfb8970098
:1040900068815700e04a2200d80007000080fa003b
:1040a000000006000100200070268900812689009a
:1040b00011c0b300c04c2200014878000000060087
:1040c000c24c22001204e00006003a00100020005a
:1040d00001002000702689008126890010c0b300ed
:1040e00000497800d2e62400631c24007026810079
:1040f00081268100f3f507000001be009003230034
:1041000001002000020040008380480070268900e2
:10411000812689004088de00cf80de0000f0a1000b
:10412000000006008001eb0002003700817178007a
:104130008301e800828f5100fcff3a000000060076
:1041400010417800b141510003003a000000e8003e
:104150000204e000faff3a000300fb000000060042
:104160000200fa00889fbe00a0ff9f0001047800b3
:10417000b1009000810478000904b200020032000e
:104180000000fb00360037000118a30005003a00cc
:104190000103b30031049800190498000080eb007b
:1041a0002f003700580090000000e00006003a00a1
:1041b0004800900012002000e6805700517e070062
:1041c0001904980024003700280090000000e00047
:1041d00008003a00604c220020049800000c78008f
:1041e0002000200050049800100498000130a00026
:1041f0003104980018019000a80090004800900039
:10420000407e070028009000000c78000080eb0042
:104210001004980018007800aff897000158780053
:10422000000c78002ff89700ea4f50000a003a007f
:10423000380090000088a3000700320018019000a9
:10424000a8009000480090002e7e070019049800f6
:10425000a8009000010c7800aff897000100fb0067
:104260004f04be000080fa000000060081017800c3
:104270000002eb000b003700e44078000104e0008e
:10428000030032000402e80093cf50000400320023
:104290008180fb001380fb000080500000000600be
:1042a0008301e800820f5200f3ff3a00000005008e
:1042b000889fbe008a1f7800000578000000e0009b
:1042c00020003d000005ea00d0062000611f22000a
:1042d000800f550040003400420620001100090004
:1042e0000205d80000017800010078004311dd00cc
:1042f000691f22001e003700a2002000811f7800e5
:10430000110009000205d8000001780001007800c2
:10431000cf0078004311dd00010141004300dd00c2
:10432000010040003002be002003be004220900089
:10433000d2209000f2219000622190004af70700fd
:104340002b003700d0062000612a2200800f550084
:104350002100340042062000110009000205d800a7
:1043600000017800010078004311dd00692a220075
:1043700009014100a8002000110009000800d80030
:104380004300dd000900400040229000d022900050
:1043900060239000f02390000288900092889000a3
:1043a000b2899000228990002ff70700801f7800c3
:1043b00001027800110009000805d8000102fd0083
:1043c0004f0078004322dd00090242005403be0082
:1043d0004402be00d9ff3700ea0f5500c6ff3c007b
:1043e0004350dd00010040005001be004000be000f
:1043f0004f0578004f04be00000006008f03b00098
:10440000889fbe008a9fbe008c9fbe008e1f7800d2
:10441000e0b79f00f1b79f0082bf9f000000eb0054
:10442000a0b79f00e00437008001eb0050c2b3004a
:1044300080cf5000090032000100fb00efb0970070
:1044400047fe0700e10f4000d7043200afb09700ed
:104450008100e800a1b79f00d30437007fb1970027
:1044600092407800d0c2b30080cf50000c003200e0
:1044700007003c006d40500080cf50000d0032001e
:104480006b40400080cf500019003a000e0037000a
:1044900000c3b30080cf500015003a000f00370072
:1044a0000330a0007fb297000402e800f4b79f0039
:1044b000eaff37000300a000ffb297008502e80082
:1044c000f5b79f00e5ff37000310a0007fb6970007
:1044d0000c06e800fcb79f00e0ff37000320a000b7
:1044e0007fb097000000e800f0b79f00dbff3700c7
:1044f0000318a300010032000300a1000338a30049
:10450000010032000320a1000100fb0002fd2f008a
:1045100002004000e90f500010003e008000eb0058
:10452000c1b79f00020278004fb197006a10b9002e
:10453000ffb297001501fb0000014100040141009a
:10454000c2b79f005500fb00f5b79f000400400074
:10455000e90f50000d003e00f3ff37000006eb00ae
:10456000ccb79f00a0c2b30080cf500007003a0034
:104570000fb89700c000780080bf9f00c1b79f00b0
:104580007fb197000201e800f2b79f00e0c2b300dc
:104590007fb29700944f100021003a008306780004
:1045a0000de0a0008400e80064405000914f10002e
:1045b00004003200f1b79f008002eb00b5b79f0006
:1045c000100037000fbe97004c0078008cbf9f0092
:1045d000b0b79f00ffb097008180e800f1b79f005f
:1045e000130037003fb297006a20b9000000410075
:1045f00003004000b0b79f00ffb297008502e800bb
:10460000f5b79f007fb697001c01fb0003fd2f004c
:1046100003004100e90f5000f2ff360004003700ac
:10462000830678000dc0a0000000eb00b0b79f002b
:104630007fb19700b2407800f2b79f00c17f9f0022
:10464000c0c6b30080cf50002700320014003c00e9
:104650006840500080cf50009d00320009003c00af
:104660006c40500080cf5000290032006b40400069
:1046700080cf5000720032000104e000500432008c
:104680008e00370060c6b30080cf50001c0032009f
:104690006340400080cf500088003a008c00370013
:1046a00030c7b30080cf50001c00320007003c0030
:1046b0006440500080cf5000130032000040e800fa
:1046c00080cf50007d003a001100370050c7b30082
:1046d00080cf50007d0032006340400080cf50000a
:1046e00076003a000b003700000028000d48a300b8
:1046f00001003a000001200080867600ccff3700e0
:104700000da0a000720037000d60a00070003700ff
:104710000d50a0000d70a0006d0037008fb99700fc
:104720004300780083bf9f00000478000000e00091
:1047300001003a00684722008004eb0001003700c6
:104740008104e80089007800088044001004e0003b
:10475000fbff3a003fb297000400e0000300320084
:10476000890f520001003100840478000007eb003b
:10477000cfb29700898f520001003600098752009e
:104780004368de00e106600019003a000d0678007b
:1047900009003700efb097000002200070fd07000d
:1047a000e10f4000030032002fb097000000e80046
:1047b000a0b79f000c06e8008e0f5600f5ff3a00e8
:1047c0000087eb000a003700880078003100fb000a
:1047d00001047800efb0970061fd0700e10f400091
:1047e00003003200afb097008100e800a1b79f003e
:1047f0000900e90080047800e10f4000f2ff3a0070
:104800000006eb000d00e0000a003a00e603370066
:10481000efb097000002200051fd0700e10f4000bb
:10482000030032002fb197000201e800a2b79f00f9
:104830000c06e8008e0f5600f5ff3a00da03370049
:104840008fb997004300780083bf9f00cf80de00c0
:1048500001017800820178000205be000004be005c
:104860000203be000002be004822de00482edd002a
:1048700004027600c47f9f000d48a3000a003200a6
:104880000404e00008003200e14f4200060032005c
:10489000d1fb2f00018047000448780018409800a1
:1048a0002900200002003700d07f9f00190020005f
:1048b000d2fb2f0002844700a6ff3700c3fb2f0066
:1048c0000384470019002000a2ff37000d0cb3003d
:1048d0000070200000826600210232000dc8a30093
:1048e0000200320064002000b4b79f008fba970026
:1048f0006881520082bf9f003200be001201be00dc
:10490000e0af9f00f1af9f0082b79f0093b79f0079
:104910006022b8006033b8006fa89700ffa8970026
:104920000fb197009fb197001df707000000e0004e
:104930000a003d006fa89700ffa897000fb19700ed
:104940009fb1970003f0a200e0af9f00f1af9f007e
:1049500082b79f0093b79f003d00b3000000eb00bb
:1049600080a79f006022b8006033b8006fa897004e
:10497000ffa897000fb197009fb19700e9fa0700d1
:104980000000e0003300320001fc2f0001824700ec
:104990006fa89700ffa897000fb197009fb19700ed
:1049a000e5fa07000fa097000000e9006300b900d6
:1049b000a2002000110009000200d8008000fd00c4
:1049c00081a79f000100e00002003d000100e90016
:1049d00080a79f000fa497000800ea0034fe07009c
:1049e0006faa9700ffaa97000fb397009fb3970095
:1049f0009df50700a0af9f00b1af9f00c2af9f0021
:104a0000d3af9f006022b8000600200007ff2300fc
:104a1000e3f607000000e00002003d000800e900a6
:104a20000b0037006022b800060020004702240077
:104a30002fa89700bfa897004fa99700dfa997005c
:104a4000d2f607000000e000020035000800e80090
:104a500080a79f003fb19700f80f510057003c001e
:104a6000d0c6b300804f5100290036000285fb00fc
:104a700042062000110009000285d80000017800dc
:104a8000010478004311dd006b1f22000b0141007f
:104a90006022b8000600200007fe23000288900074
:104aa00092889000b2899000228990006ef50700ec
:104ab000a9002000809fbe00110009000984d800d1
:104ac000000478004f00be004344dd000b044400a6
:104ad00048229000d822900068239000f82390008c
:104ae00061f50700801f78000102780011000900bd
:104af0000985d8000102fd004f0078004322dd0047
:104b00000b0242005403be004402be001f003700e7
:104b10000280fb00691f2200ea4f5100140036009a
:104b2000a2002000110009000280d80000017800d6
:104b3000010478004311dd00090141006022b80042
:104b40000600200007fe230042209000d2209000a3
:104b5000f22190006221900043f507004344dd00fc
:104b6000090444003802be002803be0007003700d5
:104b70004300dd00090040006022b800060020006c
:104b800007fe23005001be004000be0036f50700be
:104b90000002be000203be006fa89700ffa89700a6
:104ba0000fb197009fb19700a4f50700e0af9f00f9
:104bb000f1af9f0082b79f0093b79f000fa49700ab
:104bc000e90f540015003c006022b8006033b800c3
:104bd0006fa89700ffa897000fb197009fb19700ab
:104be00050fa07000000e000320032006fa8970082
:104bf000ffa897000fb197009fb197006bfa0700cd
:104c0000e00f5000e08f5800e00f5900e08f59008e
:104c100028003a00e10f54002600340054692d00aa
:104c200065822e00b6e02200170124002fa897000d
:104c3000bfa897004fa99700dfa9970058f6070073
:104c40000000e00002003d00730054000100370046
:104c50007200540080a79f000fa0970094fd0700ea
:104c6000a0af9f00b1af9f00c2af9f00d3af9f0026
:104c70000002be000203be006fa89700ffa89700c5
:104c80000fb197009fb197009bf4070047fa070008
:104c90000205be000004be006000b8006011b8004c
:104ca000a0a79f00b1a79f00c2a79f00d3a79f0006
:104cb0002e0037006fa89700ffa897000fb197004c
:104cc0009fb1970039fa07000205be000004be003c
:104cd000e00f5000e08f5800e00f5900e08f5900be
:104ce0000200350072f707001300370010002000a3
:104cf000010020006011b800080060008980600099
:104d00000a0161008b8161008b03d1000a83d3000b
:104d10008982d3000882d300000072008180720073
:104d2000020173008381730061f707000002be0077
:104d30000203be0041f507000002be000203be00f0
:104d40006fa89700ffa897000fb197009fb1970039
:104d500009f60700a0a79f00b1a79f00c2a79f0068
:104d6000d3a79f000000eb0080a79f0014c0b300f2
:104d7000653522000b0037000400fb004300dd0016
:104d8000050040005001be004000be000040e100b0
:104d900001c8e10002d0e10003d8e10003003900be
:104da0000442e800f44f5200f3ff3a00c47f9f0032
:104db0000400fb00bfb09700008040008fa0970068
:104dc000010040004fb1970000075100bfb19700ac
:104dd0000300e000010032000e07e9006380660076
:104de000010032000e07e9000d28a3002600320062
:104df000e18066000d18a3000c003200d0022000f4
:104e00000100e00001003a000080e900efb09700e7
:104e1000d3fb0700e10f4000180032002fb29700cb
:104e20000402e800a4b79f00140037000100e0006e
:104e300012003200efb0970000022000c8fb07000c
:104e4000e10f40000d003200afb297008502e8008c
:104e5000a5b79f0009003700efb0970000032000be
:104e6000bffb0700e10f4000030032002fb69700a0
:104e70000c06e800acb79f000e07e9000e00e0004a
:104e8000f5ff3c003d0037000d38a3000a0032005a
:104e90000b003700efb0970000022000b0fb0700c6
:104ea000e10f4000030032002fb097000000e8003f
:104eb000a0b79f000e07e9000e00e000f5ff3c00e0
:104ec000e18066000d18a3000c003200d002200023
:104ed0000100e00001003a000080e900efb0970017
:104ee0009ffb0700e10f400024003200afb09700a5
:104ef0008100e800a1b79f00200037000100e0001a
:104f00001e003200efb097000002200094fb070063
:104f1000e10f4000190032002fb197000201e800b4
:104f2000a2b79f00150037000000fb004300dd0022
:104f300061352200010040003002be002003be00a7
:104f40000800be000a01be00e5f80700a40020002a
:104f5000050020006033b800e8f807000003b00047
:104f6000efb097007efb0700e10f40000300320026
:104f7000afb197008301e800a3b79f004f7a970075
:104f80000440e900c07f9f00e14f4000e6ff3a0087
:104f90000b003700efb097000003200070fb070004
:104fa000e10f400003003200afb297008502e80035
:104fb000a5b79f000fa097000000e90080a79f0001
:104fc0000fa097000000e000f2ff3c003fb6970002
:104fd00020c1b300f20f560001003c006fe09700c3
:104fe000c07f9f00cf7897000100fb003fb1970082
:104ff00000005100e0a79f000104e000080032001b
:10500000efb09700e002200055fb0700e10f4000e1
:1050100003003200afb197008301e800a3b79f00ff
:105020004f7a97000400fb00a1fc07000002be00bd
:105030000203be002fa09700bfa097004fa19700ca
:10504000dfa1970008f4070058f907001e00370099
:105050000000fb004300dd006c3522000c00400026
:105060003002be002003be000800be000a01be00e0
:105070009bf80700a4002000050020006033b80062
:105080009ef807000003b000efb0970034fb070064
:10509000e10f400003003200afb297008502e80044
:1050a000a5b79f00cf7897000100fb004300dd000b
:1050b0000c0040003002be002003be000800be000d
:1050c0000a01be008df807000205be000004be0004
:1050d0004f7997000240e900c07f9f00e14f4000f8
:1050e000dbff3a000006eb0009003700efb0970045
:1050f000000320001afb0700e10f4000030032000c
:10510000afb197008301e800a3b79f000c06e80049
:105110006fa29700840f5600f4ff3a000d38a300e9
:10512000a10132000e00e0009f0134000006eb00f8
:10513000efb097000002200009fb0700e10f4000dc
:1051400003003200afb297008502e800a5b79f00c8
:105150000c06e8008e0f560093013200f4ff370072
:105160000d007800000cb20028003a000d00e000ad
:1051700005003d000fbe97004c05be004c04be006c
:105180008cbf9f00140037000d48a3000b003200b5
:105190000fb997004200be0082bf9f004f89de001a
:1051a000cf91de000002be00020378008203780087
:1051b0000605be000404be00070037008fb9970043
:1051c0004300780083bf9f0000047800cfc4de0056
:1051d000090578008a057800e00f5400e08f5c0034
:1051e000e00f5d00e08f5d0020003d003d00b3005a
:1051f0006000b8006011b8000804500089845800ad
:105200000a0559008b855900180037000d00e00091
:1052100005003d000fba97004405be004404be00df
:1052200084bf9f00110037000d48a3000800320022
:105230008fba97004500be0085bf9f00040178002b
:10524000840178000205be000004be00070037009c
:105250000fbe97004c0078008cbf9f0000047800c0
:10526000090020000a0020000b0020003fb097003a
:105270000000e00007003a00e00f5400e08f5c00ff
:10528000e00f5d00e08f5d0002003a001100200099
:10529000b1b79f000d0778000e0cb200000420008b
:1052a000800f57002f00320003003c000e00e0008a
:1052b000070032003f00370000082000800f570031
:1052c00014003200000c2000800f570039003a0013
:1052d00014c0b300653522000b0037000400fb004a
:1052e0004300dd00050040005001be004000be004c
:1052f0000040e10001c8e10002d0e10003d8e10074
:105300002b0039000442e800f44f5200f3ff3a004a
:105310002700370000012000010020006011b800c4
:1053200014c0b3000040e10001c8e10002d0e10078
:1053300003d8e1001e003900450020000000d00025
:105340008180d2000281d2008381d2008502e900ef
:10535000faff3a000442e800f04f5200f1ff3a0031
:105360001300370080002000010020006011b80009
:1053700014c0b3000040e10001c8e10002d0e10028
:1053800003d8e1000a0039003c0020000000d000f2
:105390008180d2000281d2008381d2000c06e90014
:1053a000faff3a000442e800f54f5200f1ff3a00dc
:1053b000c47f9f00cf7897000100fb003fb19700aa
:1053c000820f500002003d00c27f9f0004003700a2
:1053d000bfb19700808f510001003d00b0b79f0022
:1053e0004fb297000400e0000400320063806600c2
:1053f000020032000402e900c4b79f000de8a300d8
:105400000b003200cfb297003fb697008c8f52004e
:1054100003003c000000eb00c0b79f000400370011
:10542000cfb097003fb1970082805000c1b79f0076
:10543000cf7997000300fb000002eb0094a79f00c8
:10544000cfb29700808f52000200340000805200db
:1054500090a79f000d28a30037003200e18066006e
:105460000d18a3000c003200d00220000100e00063
:1054700001003a000080e900efb0970038fa070019
:10548000e10f40000e0032002fb697000c06e80036
:10549000acb79f000a0037000100e00008003200ae
:1054a000efb09700000220002dfa0700e10f400046
:1054b000030032002fb097000000e800a0b79f0063
:1054c0009fa097000100e0000f0032000006eb00f3
:1054d000efb097000003200021fa0700e10f400021
:1054e000030032002fb197000201e800a2b79f002d
:1054f0000c06e8009fa19700830f5600f4ff3a00c6
:105500000002eb0094a79f00bfb29700c328dd0004
:10551000e03422008080400091af9f004228dd00ef
:105520006400500080af9f006328b900f0a79f007f
:1055300063065000820037001fa697000c00e000b1
:1055400011003200688066000f003a000006780003
:10555000efb097000002200001fa0700e10f4000c1
:10556000030032002fb097000000e800a0b79f00b2
:105570000c06e8009fa09700810f5600f4ff3a0048
:105580000001eb0092a79f00e18066000d18a300c8
:105590000c003200d00220000100e00001003a00bf
:1055a0000080e900efb09700edf90700e10f40003f
:1055b000d5ff3200afb197008301e800a3b79f0089
:1055c000d1ff37000100e000cfff3200efb09700bd
:1055d00000022000e2f90700e10f4000caff32009c
:1055e0002fb297000402e800a4b79f00c6ff37005f
:1055f00000042000800f57003000320003003c0000
:105600000e00e000070032003d00370000082000d7
:10561000800f570011003200000c2000800f57004f
:1056200037003a001fa897003002be002003be00da
:105630000800be000a01be0029f70700a4002000f0
:10564000050020006033b8002cf7070004c3b30046
:1056500004424000c47f9f0029003700d547220044
:10566000d5b79f000d58a30002003a00e048220081
:10567000d0b79f0014002000050020006033b80060
:105680008fa897008100e900050033000402d000d4
:105690008582d2000683d2008783d200f9ff3700cb
:1056a0000800be000a01be000df707006f00600091
:1056b0005fb19700624078001000370014002000ae
:1056c000050020006033b8008c0178008301e900f8
:1056d000050033000402d0008582d2000683d20088
:1056e0008783d200f9ff37000800be000a01be0020
:1056f000fbf60700674060000043b000c07f9f00da
:105700004f7a97000400fb00efb0970094f9070070
:10571000e10f400003003200afb297008502e800bd
:10572000a5b79f001fa897006800500090af9f008a
:105730008fa89700e480500081af9f006306560059
:10574000d0ff2f003fb197000090b900ffa1970054
:105750000080410063005000800f5600a4ff3a0013
:105760000d38a300100032001fa297000400e000d3
:105770000d0034000006eb00efb09700000220009f
:1057800077f90700e10f400003003200afb2970045
:105790008502e800a5b79f000c06e8001fa097004f
:1057a000800f5600f4ff3a007fb19700b2407800b6
:1057b000f2b79f00c17f9f000104e0001afb3a008e
:1057c0002fb097004f0778004f06be004f05be0070
:1057d0004f04be008f03b100000006000600fa006f
:1057e0001f0107000040eb00004f78000000200080
:1057f000010220001007980021079800809f800078
:10580000919f80004508de000100200061006000db
:105810000004e0000300320010c0b300004f780025
:1058200006003700a8200200020000000004e0008b
:105830000200320010c0b300004f78001e04e000e8
:105840001a003200800020006c0907001007980041
:10585000210798002000200052090700709f88004f
:105860001e019000ae019000000020000102200007
:1058700000007100818071001007980021079800d6
:10588000719f80000000220000807000709f8800df
:105890001e019000ae01900080002000a8080700c3
:1058a000719f80002000200094080700fe0f020076
:1058b000010000000080fa00000006007800fa00f5
:1058c000103f980041f79800323f98000000eb002d
:1058d000300798001f0037003e0090006c00b900b0
:1058e000800078001e389000808040000000eb00af
:1058f000800878003e0090006c00b90080007800bd
:105900001e389000808040000040eb00a0409800ce
:105910003e0090006c00b900800078001e389000b6
:10592000808040000040eb00b04098003e009000b6
:105930006c00b900800078001e3890008080400024
:105940000040eb00c04098003e0090000000e800de
:10595000300798003e009000e10f5000deff340059
:105960006a004700a1c0b300e6d4020001000000b5
:105970000080fb00400798000000eb00000f78005b
:105980006a014700a00520000e0040000002eb0065
:10599000ce01900091002000c80302000100000029
:1059a000300798003e0090000000e000a0003500a5
:1059b000a00520000e004000104090000080fb0079
:1059c000200798002e009000c800dd00a0052000f0
:1059d0000e004000204090000080fb00008040004e
:1059e000200798001e0078006c00b9008000780045
:1059f0001e38900000804000ae0090000108780042
:105a00001e0078006c00b900800078001e389000fd
:105a100080804000a00520000e0040003040900033
:105a2000a04098001e0078006c00b900800078004b
:105a30001e38900080804000a00520000e0040002d
:105a400040409000b04098001e0078006c00b90003
:105a5000800078001e389000008140003e009000d9
:105a6000ea0047004300dd000100400010407800dc
:105a7000404198001e0078006c00b900800078005a
:105a80001e389000008140003e009000ea00470070
:105a90004300dd000100400010409000504198009c
:105aa0001e0078006c00b900800078001e3890005d
:105ab000008140003e009000ea0047004300dd0006
:105ac0000080e8000100400010407800604198002c
:105ad0001e0078006c00b900800078001e3890002d
:105ae000008140003e009000ea0047004300dd00d6
:105af0000080e800010040001040900070419800d4
:105b00001e0078006c00b900800078001e389000fc
:105b1000008140003e009000ea0047004300dd00a5
:105b200064004000010040001040780000499800e7
:105b30001e0078006c00b900800078001e389000cc
:105b4000008140003e009000ea0047004300dd0075
:105b5000640040000100400010409000104998008f
:105b60001e0078006c00b900800078001e3890009c
:105b7000008140003e009000ea0047004300dd0045
:105b80006600400001004000104078002049980065
:105b90001e0078006c00b900800078001e3890006c
:105ba000008140003e009000ea0047004300dd0015
:105bb000660040000100400010409000304998000d
:105bc0004ef090000004e000180032003e389000d3
:105bd0000000e000150032000000eb001007980004
:105be0000f0037001e0078007800b90080007800b0
:105bf0003e389000808140001e0190009e00900081
:105c0000a00520000e0040000080400010407800f9
:105c100000f179001e0090000000e80010079800d5
:105c20001e009000f70f5000eeff34001e0fe8003a
:105c3000be0090004e009000808f500006003d0096
:105c40003e0090000000e00003003400100020003f
:105c50009e0f10004aff34000080fa00000006008a
:105c60002e00fa00881f78006604470060022000ba
:105c70000e004000010220008b0807006002200097
:105c80000e00400007000900305c78008800b10079
:105c90008000b100ee004700660047005c0207008c
:105ca0000080fb00100798009e009000e00f20008d
:105cb000808f500004003a00e0e42c00561b0200e4
:105cc00000000000290237009e009000d00f200045
:105cd000808f500022023c006e0047001040780088
:105ce000e24f500004003200d0e82c00561b0200a6
:105cf000000000001d02370002002c0023012000dc
:105d0000001b20008e0707006e0047001040900027
:105d10000080fb00200798002e009000c800dd00e6
:105d20006e004700204090000080fb000080400093
:105d300020079800ae009000c0062200808f50001f
:105d40002c013a006e004700b040900020c3b30021
:105d500080cf50000e0032006e004700b04090002f
:105d600070c3b30080cf5000090032006e004700be
:105d7000b0409000f0c4b30080cf50000400320067
:105d8000c0ea2c00561b020000000000f70137009b
:105d90006e00470050409000f1c5b300014f600015
:105da0006e004700b040900020c3b30080cf500089
:105db0008f003a0020c4b3009e4f100070003600e0
:105dc0006e00470040409000e14f500018003a003c
:105dd000c1062200000120006b07070021032000fc
:105de0002001200068070700e10120004001200099
:105df0006507070052722900235d20008000200003
:105e00004f070700f17c2000200020003b0707001f
:105e1000e217200003002000c018200048070700f8
:105e200020002000df070700709f8800cf013700a7
:105e30006e00470040409000e24f500018003a00ca
:105e4000c1062200000120004f07070021032000a7
:105e5000200120004c070700f10120004001200034
:105e60004907070052702900235d200080002000b0
:105e700033070700f1fc2000200020001f07070067
:105e8000e217200003002000c01820002c070700a4
:105e900020002000c3070700709f8800b30137006f
:105ea0006e00470040409000e34f500018003a0059
:105eb000c106220000012000330707002103200053
:105ec00020012000300707000102200040012000cf
:105ed0002d07070052722900235d2000800020005a
:105ee00017070700f17c20002000200003070700af
:105ef000e217200003002000c01820001007070050
:105f000020002000a7070700709f88009701370036
:105f10006e00470040409000e44f500034003a00cb
:105f2000c1062200000120001707070021032000fe
:105f3000200120001407070011022000400120006a
:105f40001107070012702900235d20008000200047
:105f5000fb060700d1ec200020002000e706070028
:105f6000e217200003002000c0182000f4060700fc
:105f7000200020008b070700709f88007b013700fe
:105f80006e00470040409000e14f500018003a007a
:105f9000c106220000012000fb06070021032000ab
:105fa00020012000f8060700e10120004001200048
:105fb000f506070052722900235d200080002000b2
:105fc000df060700f13c200020002000cb06070080
:105fd000e217200003002000c0182000d8060700a8
:105fe000200020006f070700709f88005f013700c6
:105ff0006e004700b040900070c3b30080cf5000e7
:1060000057003a006e00470040409000e14f5000ba
:1060100018003a00c106220000012000da0607003d
:106020007103200020012000d7060700e1012000b5
:1060300040012000d406070052722900235d200091
:1060400080002000be060700f17c20002000200018
:10605000aa060700e217200003002000c018200055
:10606000b7060700200020004e070700709f880039
:106070003e0137006e00470040409000e24f500064
:106080001b003a00c106220000012000be060700e6
:106090007103200020012000bb060700f101200051
:1060a00040012000b806070012702900235d20007f
:1060b00080002000a2060700d1bc200020002000a4
:1060c0008e060700f1fc2000200020008b06070050
:1060d000e217200003002000c018200098060700e7
:1060e000200020002f070700709f88001f01370045
:1060f0006e00470040409000e34f500018003a0007
:10610000c1062200000120009f0607007103200045
:10611000200120009c060700010220004001200011
:106120009906070052722900235d2000800020009c
:1061300083060700f17c2000200020006f06070086
:10614000e217200003002000c01820007c06070092
:106150002000200013070700709f8800030137000c
:106160006e004700b0409000f0c4b30080cf5000f4
:10617000fe003a006e00470040409000e14f5000a2
:10618000fa003a00025a220063022000001b20009d
:106190006b060700c1062200000120007a060700f6
:1061a000210320002001200077060700e1012000e4
:1061b000400120007406070052722900235d200070
:1061c000800020005e060700f17c200020002000f7
:1061d0004a060700e217200003002000c018200034
:1061e0005706070020002000ee060700709f880079
:1061f000de003700ae00900020072200808f5000a4
:10620000ab003a006e004700b040900030c2b300cf
:1062100080cf5000090032006e004700b04090006f
:1062200070c2b30080cf50000400320060ed2c003b
:10623000561b020000000000cc0037006e00470033
:10624000b040900030c2b30080cf500036003a001a
:106250006e00470040409000e14f500017003a00a8
:10626000210722000001200047060700310220001c
:106270002001200044060700e10120004001200029
:106280004106070042702100635d2000800020006d
:106290002b060700b1bc21002000200017060700d4
:1062a0006011b800c018200025060700200020005b
:1062b000bc060700709f8800ac0037006e004700e6
:1062c00040409000e34f500017003a0021072200a1
:1062d000000120002c0607003102200020012000d0
:1062e00029060700e10120004001200026060700e2
:1062f00042722100635d200080002000100607002c
:10630000b17c210020002000fc0507006011b800ce
:10631000c01820000a06070020002000a106070080
:10632000709f8800910037006e004700b0409000d9
:1063300070c2b30080cf50005d003a006e0047008d
:1063400040409000e14f50001b003a00025a2200ea
:1063500063022000001b2000f9050700210722002e
:106360000001200008060700710220002001200023
:1063700005060700e1012000400120000206070099
:1063800042702100635d200080002000ec050700c2
:10639000b1bc210020002000d80507006011b80022
:1063a000c0182000e6050700200020007d06070039
:1063b000709f88006d0037006e00470040409000dd
:1063c000e24f50001b003a00025a220063022000f4
:1063d000001b2000da050700210722000001200031
:1063e000e90507007102200020012000e6050700f2
:1063f000e101200040012000e30507005270210068
:10640000635d200080002000cd050700b1bc2100a5
:1064100020002000b90507006011b800c018200056
:10642000c7050700200020005e060700709f880057
:106430004e0037006e00470040409000e34f500090
:106440001b003a00025a220063022000001b2000b9
:10645000bb0507002107220000012000ca05070034
:106460007102200020012000c7050700e101200083
:1064700040012000c405070042722100635d200036
:1064800080002000ae050700b17c21002000200024
:106490009a0507006011b800c0182000a805070081
:1064a000200020003f060700709f88002f00370063
:1064b000ae00900000fd2100808f500028003a00bf
:1064c0006e004700b040900050c2b30080cf500033
:1064d00004003200e0ef2c00561b02000000000018
:1064e000220037006e00470040409000e14f50000e
:1064f0001b003a0001fd210000012000a205070059
:1065000051022000200120009f0507008102200089
:10651000400120009c05070052702900235d2000e7
:106520008000200086050700f1bf20002000200029
:1065300072050700200020001a060700709f8800df
:10654000e217200003002000c01820007c0507008f
:106550008000eb00e01620008b05070003003700e9
:1065600010f22c00561b0200000000004f047800bf
:106570000080fa00000006000800fa00889fbe00b4
:10658000400020001d0607000004be00800020001f
:106590001a060700880178000902780000017800d7
:1065a0000100780082806100000062006101b80093
:1065b00022079800330798002e019000be0190003a
:1065c000c011dd0002002000220798003307980068
:1065d0002e019000be019000028fbe006109b8003c
:1065e00022079800330798002e009000be0090000c
:1065f0001e1f70001e9770001e01be00400020008c
:106600004f0507004f04be000080fa00000006009e
:106610000a00fa003007980041079800d0cfb30075
:106620002047980050c0b300404798002f00370023
:106630004e009000000f78004e4090000080fb005c
:106640007800b900784050000041780083c1b30061
:106650009e0078003e009000d0d6020001000000ad
:106660000004e00003003a00e0cfb30020479800a8
:106670002100370010c0b300304798000040eb0005
:10668000504798000a0037001e007800104078003c
:10669000e14f4000020032000040eb00304798001c
:1066a0001e0fe8005e4090000040e8005047980050
:1066b0005e409000f74f5000f3ff36003e409000e0
:1066c0000004e00006003a004e4090000080fb000d
:1066d0007800b90078405000204798000600370045
:1066e0004e4090000040e900404798004e40900026
:1066f0000004e000ceff3a003e409000e14f500021
:1067000005003a004e4090000004e00002003a000c
:1067100000c0eb00204798002e4090000080fb0056
:106720000080fa00000006001000fa0050079800f0
:10673000610798006e0090000000e00003003a003e
:1067400010002000700798002b0037006e009000aa
:10675000e10f400003003a000000eb0070079800d2
:1067600025003700309e8000000f78001e00780062
:106770000100200030079800410798005e0090005b
:106780006101b8006e00900001002000020040008e
:106790008380480010079800210798005e00900051
:1067a0009e0f5000080036003e009000ce00900082
:1067b00002002000130020000000410081804900f9
:1067c00030079800410798003e019000ce019000ec
:1067d0001e009000ae009000800f5100818f590084
:1067e00003003900100020007007980002003700f5
:1067f0000000eb00700798007e0090000080fa0017
:10680000000006001000fa00500798006107980089
:106810006e0090000000e00003003a00100020002d
:10682000700798002b0037006e009000e10f4000c9
:1068300003003a000000eb007007980025003700c5
:10684000209e8000000f78001e00780001002000cc
:1068500030079800410798005e0090006101b80081
:106860006e0090000100200002004000838048007c
:1068700010079800210798005e0090009e0f5000be
:10688000080036003e009000ce009000020020007c
:10689000130020000000410081804900300798006b
:1068a000410798003e019000ce0190001e0090002c
:1068b000ae009000800f5100818f59000300390015
:1068c0001000200070079800020037000000eb0065
:1068d000700798007e0090000080fa00000006001b
:1068e0000600fa0010079800209e8000000f780034
:1068f0001e0090009e0f50000a0036001e009000ff
:106900001e0050000000e00003003d0010002000c9
:10691000200798000d0037000000eb0020079800ca
:106920000a0037001e0090009e001000e0ff2700c4
:10693000808f500003003e001000200020079800c8
:10694000020037000000eb00200798002e009000a6
:106950000080fa00000006000800fa00008fbe0068
:106960001e00be00e00f5000e08f5800060035000a
:106970001e00be006e0c0200000000002007980000
:1069800031079800170037001e0078006101600091
:106990006000b800030020000200700083807000d7
:1069a0001e01be008301d1000281d30002007000ed
:1069b000838070006e0c0200000000002007980029
:1069c000310798002e019000be0190002e0090002b
:1069d000be009000c60c02000000000020079800d6
:1069e00031079800a2992900935924002e009000a5
:1069f000be009000800d0200000000000200200098
:106a000003402400e80d0200000000006c0e0200ac
:106a100000000000020007000080fa0000000600ed
:106a20000400fa00008fbe001fe1a9000000eb0087
:106a3000a00888000000eb00c00888001e00780055
:106a4000d00888001e00be004008de0001002000c3
:106a5000e00888008780a9009780a800119f800027
:106a6000f0fe2f0000806000109f8800119f8000c2
:106a70000002200000807000109f88001fe1a80025
:106a80000080fa00000006000800fa00008fbe0037
:106a90001e00be00e00f5000e08f580006003500d9
:106aa0001e00be006e0c02000000000020079800cf
:106ab00031079800170037001e0078006101600060
:106ac0006000b800030020000200700083807000a6
:106ad0001e01be008301d1000281d30002007000bc
:106ae000838070006e0c02000000000020079800f8
:106af000310798002e019000be0190002e009000fa
:106b0000be009000c60c02000000000020079800a4
:106b100031079800a2992900935924002e00900073
:106b2000be009000800d0200000000000200200066
:106b300003402400e80d0200000000006c0e02007b
:106b40000000000001002000020007000080fa00a1
:106b5000000006000400fa00008fbe002de1a9002d
:106b60000000eb00100988000000eb0030098800ed
:106b70001e007800400988001e00be004008de00ac
:106b800001002000500988008a00a9009a00a8008e
:106b90002de1a800119f8000f0fb2f000080600015
:106ba000109f8800119f8000000820000080700066
:106bb000109f88000080fa00000006000200fa0022
:106bc000000f78009e007800b01e2000d64c020016
:106bd000000000000080fa00000006000800fa0033
:106be000204798002e4090000080fb00300798005e
:106bf0003e009000e20f5000220032003e00900064
:106c0000e20f500007003c003e0090000000e00052
:106c10000e0032003e009000e10f500012003200e2
:106c2000680037003e009000e40f50003d00320045
:106c30003e009000e40f5000260035003e0090001a
:106c4000e50f50004b0032005e00370023c2bf004a
:106c5000614060000004e0005a003a00100020008b
:106c6000200798005900370033c2bf006140600020
:106c70000004e00053003a001000200020079800b4
:106c800052003700709f80004300de00610060000a
:106c90000004e0004b003200ca82a90000c4b30027
:106ca0006c20020001000000004f7800ca82a8009a
:106cb0001e80fb004600de000000a20061006000b4
:106cc0000004e0003f003200100020002007980080
:106cd0003e003700709f80004400de0061006000cd
:106ce0000004e00037003200ca62a90000c4b3000b
:106cf0006c20020001000000004f7800ca62a8006a
:106d00001e80fb004600de000000a2006100600063
:106d10000004e0002b003200100020002007980043
:106d20002a003700709f80004500de00610060008f
:106d30000004e00023003200e922a90000c4b300ef
:106d40006c20020001000000004f7800e922a8003a
:106d50001e80fb004600de000000a2006100600013
:106d60000004e00017003200100020002007980007
:106d700016003700709f80004600de006100600052
:106d80000004e0000f003200d042a90000c4b300ac
:106d90006c20020001000000004f7800d042a800e3
:106da0001e80fb004600de000000a20061006000c3
:106db0000004e000030032001000200020079800cb
:106dc000020037000000eb00200798002e00900022
:106dd0000080fa00000006000600fa002047980034
:106de0002e4090000080fb00200798002e009000ad
:106df000e30f50005b003200ae009000e38f5000c4
:106e00000a003c002e019000e10f510035003200d5
:106e10002e009000e10f500044003c00ae009000b6
:106e20000100e0001d003200820037002e019000ba
:106e3000e50f5100710032002e009000e50f500068
:106e40005b00350030062000ae009000808f5000bf
:106e50000100320077003700514580006045800016
:106e6000808f5000fcff320051458000a088200038
:106e70006141780012479800504580000000e8000a
:106e80005045880050458000ff0f50006b003400d3
:106e90000000eb0050458800680037001142800078
:106ea00020428000808f5000fcff320011428000a1
:106eb0002080200061417800124798001042800035
:106ec0000000e8001042880011428000f00320001a
:106ed000808f5000590034000000eb001042880001
:106ee000560037003144800040448000808f5000bd
:106ef000fcff320031448000608420006141780052
:106f000012479800304480000000e80030448800b8
:106f100031448000f0032000808f5000470034008f
:106f20000000eb003044880044003700ca82a9000a
:106f30000040eb006c20020001000000004f7800d0
:106f40000040eb006c200200010000001047980098
:106f5000ca82a8001e4078000004e000f3ff3d0054
:106f600036003700709f80004400de006100600042
:106f70000004e00031003200ca62a9000040eb00ca
:106f80006c20020001000000004f78000040eb0080
:106f90006c2002000100000010479800ca62a8009f
:106fa0001e4078000004e000f3ff3d00230037009e
:106fb000709f80004500de00610060000004e0007a
:106fc0001e003200e922a9000040eb006c20020004
:106fd00001000000004f78000040eb006c20020030
:106fe0000100000010479800e922a8001e40780028
:106ff0000004e000f3ff3d0010003700d042a9007c
:107000000040eb006c20020001000000004f7800ff
:107010000040eb006c2002000100000010479800c7
:10702000d042a8001e4078000004e000f3ff3d00bd
:10703000020037000040eb00104798001e4090000f
:107040000000fb000080fa00000006000600fa00c5
:10705000204798002e4090000080fb0020079800f9
:107060002e009000e10f5000180032003006200082
:10707000ae009000808f5000040032002e0090007f
:107080000000e00009003200180037005145800080
:1070900060458000808f5000fcff32005145800029
:1070a000a0882000614f7800120037001142800054
:1070b00020428000808f5000fcff3200114280008f
:1070c00020802000614f78000a00370031448000a2
:1070d00040448000808f5000fcff3200314480002b
:1070e00060842000614f7800020037000040eb0010
:1070f000004f78001e00fb000080fa000000060030
:107100000600fa00204798002e4090000080fb0007
:10711000200798002e009000e30f5000500032002e
:10712000ae009000e38f50000a003c002e0090005b
:10713000e10f50002e003200ae009000e18f5000b1
:1071400039003c002e0090000000e0001a003200e0
:1071500077003700ae009000e58f500066003200e7
:107160002e009000e50f5000500035003006200042
:10717000ae009000808f5000010032006c0037009c
:1071800060458000804078005045800000c050007d
:10719000104798009e40900000c2b30080cf50007e
:1071a000650036001e40900001ceb3000140400053
:1071b000104798006000370020428000804078002f
:1071c0001042800000c05000104798009e40900080
:1071d00000c4b30080cf5000570036001e4090001e
:1071e00001ccb30001404000104798005200370026
:1071f00040448000804078003044800000c050004f
:10720000104798009e40900000c4b30080cf50000b
:10721000490036001e40900001ccb3000140400000
:1072200010479800440037000040eb0010479800da
:10723000ca82a90000c4b3006c2002000100000053
:10724000004f7800ca82a8001e4078000004e000c9
:1072500039003d0010c0b3001047980036003700d9
:10726000709f80004400de00610060000004e000c8
:10727000310032000040eb0010479800ca62a900bc
:1072800000c4b3006c20020001000000004f780031
:10729000ca62a8001e4078000004e00026003d00fd
:1072a00010c0b30010479800230037000040eb00e7
:1072b00010479800709f80004500de00610060006c
:1072c0000004e0001c003200e922a90000c4b30061
:1072d0006c20020001000000004f7800e922a800a5
:1072e0001e4078000004e00013003d0010c0b30011
:1072f00010479800100037000040eb00104798003e
:10730000d042a90000c4b3006c20020001000000bc
:10731000004f7800d042a8001e4078000004e00032
:1073200005003d0010c0b300104798000200370070
:107330000040eb00104798001e4090000080fb00ca
:107340000080fa00000006000800fa00404798009c
:107350004e4090000080fb00300798003e009000f7
:10736000e30f500050003200be009000e38f500049
:107370000a003c003e009000e10f50002600320061
:10738000be009000e18f500032003c003e009000b3
:107390000000e000110032008b003700be009000ba
:1073a000e58f5000740032003e009000e50f500061
:1073b0005700350030062000be009000808f50003e
:1073c00001003200800037000000eb0060458800bb
:1073d0000000eb00504588007b0037009560a90055
:1073e0000000eb00204288000000eb001042880003
:1073f00002003700301180002047980022c2bf00f1
:10740000614060000004e000faff3a008560a900d6
:107410009560a8006c00370097c0a9000000eb0041
:10742000404488000000eb00304488000200370030
:10743000b01180002047980032c2bf006140600058
:107440000004e000faff3a0087c0a90097c0a80036
:107450005d00370080002000000f78000f0037002b
:10746000ca82a9000040eb006c200200010000006d
:10747000204798000040eb006c2002000100000053
:10748000ca82a8001e0fe9002e4090000004e00010
:10749000020035000000eb00000f78001e00e00045
:1074a000efff3c0048003700709f80004400de0082
:1074b000610060000004e000430032008000200012
:1074c000000f78000f003700ca62a9000040eb00ef
:1074d0006c20020001000000204798000040eb00f3
:1074e0006c20020001000000ca62a8001e0fe90023
:1074f0002e4090000004e000020035000000eb0088
:10750000000f78001e00e000efff3c002e00370067
:10751000709f80004500de00610060000004e00014
:107520002900320080002000000f78000f00370093
:10753000e922a9000040eb006c20020001000000dd
:10754000204798000040eb006c2002000100000082
:10755000e922a8001e0fe9002e4090000004e00080
:10756000020035000000eb00000f78001e00e00074
:10757000efff3c001400370080002000000f78006f
:107580000f003700d042a9000040eb006c20020041
:1075900001000000204798000040eb006c20020032
:1075a00001000000d042a8001e0fe9002e4090000c
:1075b0000004e000020035000000eb00000f78003e
:1075c0001e00e000efff3c000080fa000000060013
:1075d0001c00fa00881f7800404798003107980087
:1075e000024f9800134f98004e40900097fe0700fe
:1075f00080407800c0c2b30080cf500005003a0040
:107600004e409000f4fd0700020037004e4090000d
:10761000f1fd07004e4090008cfe0700804078008e
:1076200000c2b30080cf5000f8ff32000040eb00f2
:10763000104798000a0037001e4090000080fb00b1
:10764000800078003e009000808040000040eb0009
:10765000804878001e4090000040e80010479800e5
:107660009e4090000e48900080cf5000f2ff3900fd
:107670000040eb00004f78000040eb0010479800fe
:10768000700037004e40900070fe070020479800c1
:107690001e4890000004e0002c003a000040eb007f
:1076a000305f9800ae409000c0c2b30080cf500061
:1076b00002003a0011c0b300315f98000041eb00b6
:1076c000225f98002e409000ea4f500002003a00de
:1076d00010c0b300205f9800be5890002e59900053
:1076e00002c070000080fb00400f98000000eb001b
:1076f000300f98002e409000ed4f500002003a00ed
:1077000011002000310f98004e099000be08900033
:10771000010071000000e000030032000e499000fb
:1077200012479800440037001e80fb00800078005c
:107730003e009000008440004e409000a6fd0700ef
:10774000004c78001e4fe8003b0037002e409000b0
:107750008000fb0000fd2f00008040008040eb0017
:1077600051579800e90f500002003e0012c0b300cc
:10777000525798000040eb0040579800ae409000f0
:10778000d0c2b30080cf500002003a0011c0b30055
:10779000415798005e519000ce509000014071001a
:1077a0000080fb00100f98000001eb00020f980012
:1077b000ae409000b0c2b30080cf500002003a004b
:1077c00010002000000f98009e0890000e09900005
:1077d00082807000710798000000eb00600798003d
:1077e000ae409000e0c2b30080cf500002003a00eb
:1077f00011002000610798007e019000ee009000cb
:10780000010071000000e000090032001e80fb0052
:10781000800078003e009000008440004e409000c0
:107820006dfd0700004c78001e4fe8000200370095
:107830000e499000124798001e4090000040e8005a
:10784000104798009e4090000e48900080cf500056
:107850008cff39001e80fb00800078003e00900005
:10786000808040000040eb00804878000040eb0042
:10787000304f9800ae409000c0c2b30080cf50009f
:1078800002003a0011c0b300314f9800009f800001
:107890004500de00610060000080fb000041eb005d
:1078a000224f98000000e0000200320010c0b30038
:1078b000204f9800be4890002e49900002c0600002
:1078c0000004e0000500320020002000bbfc07009f
:1078d00020f42c00561b0200000000004f0478002a
:1078e0000080fa00000006001800fa0020579800f7
:1078f000220f9800330f9800e400470013c0b30034
:10790000b2c0b3002e50900031ff07006400470062
:10791000104078000004e0000500320064004700d9
:107920006a1b020000000000008fbe000300370049
:107930002e089000be089000008fbe001e00be0002
:107940000080fa00000006001a00fa00881f780084
:1079500040579800320f9800430f9800e600470008
:107960008041eb00b2c0b3004e50900018ff0700fa
:1079700066004700104078000004e0003400320048
:107980006000b80010079800210798000040eb0045
:1079900010479800260037001e4090008080fb00b2
:1079a000660047000080400010407800004f7800db
:1079b0001e80fb00140c0200000000000000e0002c
:1079c0001600320090c3b3009e4f10000300360033
:1079d0001e40780069404000004f78001e4078004b
:1079e0006f4f60001e009000ae0090004409dd0063
:1079f000cc01de00830171004401dd001e407800ef
:107a00000080fb000100200002004000838048004d
:107a100010079800210798000200370030c6b30015
:107a2000104798001e4090000040e8001047980062
:107a30001e4090000084fb0066004700ce1b020041
:107a400000000000800f5400d3ff3900040037000d
:107a50003e089000ce08900010079800210798007b
:107a60001e009000ae0090004f0478000080fa00e5
:107a7000000006002c00fa0060679800421798008a
:107a800053179800ec00470013c0b30072c1b30055
:107a90006e609000cefe07006c004700104078003a
:107aa0000004e0000d0032006c0047009e1e020042
:107ab00000000000009fbe000297be006c0047005f
:107ac0009e1e020000000000a20e02000000000046
:107ad0004007980051079800040037004e109000ae
:107ae000de10900040079800510798004e0090006b
:107af000de0090000080fa00000006000600fa0098
:107b00001007980021079800640f4700220020000a
:107b10009e0090001e007800681b0200010000001b
:107b2000220020009e0090001e0078002e1c020003
:107b3000010000000080fb000080fa000000060049
:107b40000800fa00100798002207980033079800f1
:107b5000640f4700420020009e0090001e00780045
:107b6000681b020001000000420020009e009000ff
:107b70001e0078002e1c0200010000000080fb00a7
:107b80000080fa00000006000600fa0010079800c6
:107b900021079800640f4700220020009e009000fb
:107ba0001e007800681b0200010000002200200077
:107bb0009e0090001e0078002e1c020001000000b4
:107bc0000080fb000080fa00000006000800fa00b8
:107bd000100798002207980033079800640f4700a9
:107be000420020009e0090001e007800681b0200ea
:107bf00001000000420020009e0090001e0078005e
:107c00002e1c0200010000000080fb000080fa0032
:107c1000000006000c00fa001007980064004700fe
:107c200001087800120098002300980034009800a2
:107c3000640f4700720020009e0090001e00780034
:107c4000681b020001000000720020009e009000ee
:107c50001e0078002e1c0200010000000080fb00c6
:107c60000080fa00000006000c00fa0010079800df
:107c70006400470001087800120098002300980073
:107c800034009800640f4700820020009e0090009e
:107c90001e007800681b0200010000008200200026
:107ca0009e0090001e0078002e1c020001000000c3
:107cb0000080fb000080fa00000006000c00fa00c3
:107cc0001007980024079800350798004607980089
:107cd00057079800640f4700820020009e00900024
:107ce0001e007800681b02000100000082002000d6
:107cf0009e0090001e0078002e1c02000100000073
:107d00000080fb000080fa00000006001800fa0066
:107d1000200f9800310f98002e0890004400dd00dd
:107d2000100798003e0890004400dd00000f780026
:107d300064004700020120009e009000e21b020048
:107d40000100000064004700020120009e0078004e
:107d5000681b0200010000006400470002012000cf
:107d60009e0078002e1c0200010000000080fb0035
:107d70000080fa00000006000400fa0010079800d6
:107d8000120020009e0090000e007800e21b02000e
:107d9000010000001e4078000080fb000080fa0017
:107da000000006000600fa00200798000e8fe80089
:107db00022002000ae0090001e007800e21b0200ae
:107dc000010000001e0090000080fa000000060084
:107dd0000600fa00200798000e8fe800220020001d
:107de000ae0090001e007800e21b020001000000bf
:107df0001e0090000080fa00000006000800fa0053
:107e0000300798000e8fe80042002000be0090006e
:107e10001e007800e21b0200010000001e0090001e
:107e2000ae0090000080fa00000006000800fa0092
:107e3000300798000e8fe80042002000be0090003e
:107e40001e007800e21b0200010000001e009000ee
:107e5000ae0090000080fa00000006000c00fa005e
:107e6000881f780000047800510798000e8fe80002
:107e700072002000de0090001e007800e21b02006d
:107e8000010000000e80e80006000900305c780068
:107e90007800b1007000b100080078004f0478004d
:107ea0000080fa00000006000c00fa00881f78002d
:107eb00000047800510798000e8fe800820020002f
:107ec000de0090001e007800e21b020001000000ae
:107ed0000e80e80007000900305c78008800b100df
:107ee0008000b100080078004f0478000080fa009c
:107ef000000006000c00fa00881f780000047800db
:107f0000510798000e8fe80082002000de009000ec
:107f10001e007800e21b0200010000001e0090001d
:107f2000ae0090003e019000ce019000009cbe008b
:107f30000294be00080078004f0478000080fa0028
:107f4000000006001000fa00400798005107980052
:107f500062079800730798004e0090002007980071
:107f60002e489000204798003e4890001047980007
:107f70004e489000004f78009e80fb001e4090000d
:107f80000081fb002e4090000080fb00811f7800e4
:107f9000821f7800801f78002e009000801f7800dc
:107fa00050f42c00801f7800a21e02000000000088
:107fb000ea8757005e4890007f4060000044b000b0
:107fc00060479800e14a22006e4090000000fb00ec
:107fd000b01e0200000000006e4890007f4060006c
:107fe0000044b00060479800e14a22006e409000d3
:107ff0000000fb00b01e0200000000007e48900060
:108000007f4060000044b00060479800e14a2200d1
:108010006e4090000000fb00b01e02000000000057
:108020005e4890008080fb00000e20000080600011
:108030004581de006e4890008080fb00000e20002d
:10804000008060000080d100000141007e48900067
:108050008080fb00000e2000008060004300dd00f7
:1080600000004100200798002e009000801f78003b
:1080700040f52c00801f7800a21e020000000000c6
:10808000e48757000080fa00000006001600fa009e
:10809000200f98008e0078002e089000080007003e
:1080a0008e1f7800a0f52c00801f78003e1f020074
:1080b00000000000e48757000080fa00000006007e
:1080c0000400fa00000f7800110798001e007800e5
:1080d000704090000081fb001e007800104090006e
:1080e0008081fb001e007800204090000082fb0091
:1080f0001e007800304090008082fb001e00780057
:10810000404090000083fb001e007800504090002b
:108110008083fb001e007800604090008080fb00a0
:108120001e007800104078000080fb00821f78005d
:10813000831f7800841f7800851f7800861f7800d1
:10814000871f7800811f7800801f7800d0f52c00f1
:10815000801f78001e009000f81f02000000000041
:10816000f28757000080fa00000006000200fa00c3
:108170000000eb00000f7800140037001e007800ac
:108180004200dd00c00bb00028ff07006011b800fe
:10819000f80e0200000000000000e00001003c00ba
:1081a00005003700e14a2200b0022000b01e0200a4
:1081b0000000000004003700e14a2200f002200025
:1081c000b01e0200000000001e0fe8008001200029
:1081d0009e0f1000e9ff3400109f80004e00de006b
:1081e000610060000004e00005003200e14a220066
:1081f00060022000b01e02000000000004003700f2
:10820000e14a2200d0022000b01e0200000000005f
:108210000080fa00000006000800fa00200798001d
:10822000614798006e4090008080fb002e00900017
:10823000008f68000000eb00100798001000370066
:108240001e007800610060000004e00006003200bb
:108250001e0078000000d100000f780010002a00f6
:108260001e0f6800030037001e0078000000d100d8
:10827000000f78001e0090000000e8001007980032
:108280001e009000e70f5000edff34001e00780044
:108290000080fa00000006000a00fa00200798009b
:1082a00061479800420798000080eb001007980093
:1082b0000040eb00004f7800090037001e80fb00f3
:1082c000800078002e0090000080400090407800f0
:1082d0001e009000d0ff0700100798001e4fe80016
:1082e0006e4090009e4f1000f4ff39001e00900079
:1082f0004800de00804078004e0090000148780081
:108300004e0090008000e8001e0090008048780039
:108310000080fa00000006000600fa0020479800de
:10832000210798002e4090000080fb00ae009000d6
:1083300012000700104798002e4090000080fb00bc
:10834000800078002e00900000804000904078006f
:108350001e40900080cf500003003a0010c0b300d0
:10836000004f7800020037000040eb00004f78001b
:108370001e80fb000080fa00000006000800fa00e2
:1083800020079800310798000040eb00004f78006c
:108390000000eb00100798000c0037001e00900052
:1083a000800078003e00900000804000104078007f
:1083b0009e40780096d3020001000000004f780034
:1083c0001e0090000000e800100798009e0090003a
:1083d0002e009000808f5000f0ff3500009f80003d
:1083e0004500de00610060000004e0000200320091
:1083f000a0cab300004f78001e80fb000080fa0086
:10840000000006000600fa006011b80040002000dd
:10841000cbfd07006011b800c0002000c8fd0700b8
:108420006011b80000192000c5fd07006011b800f8
:10843000001a2000c2fd07006011b800c01820001b
:10844000bffd0700e0f72c004c1f020000000000f9
:1084500020079800ae009000c0012000cafd070070
:1084600000f82c004c1f02000000000020079800bc
:10847000ae009000e0012000c3fd07008000eb008b
:10848000c0042000c0fd070001002800e004200017
:108490009afd07008000eb0040042000bafd0700b1
:1084a000010028006004200094fd070011592300fa
:1084b000c0042000b4fd070031202300e0042000a8
:1084c0008efd0700518f220080042000aefd0700c2
:1084d00061662600a004200088fd070001812100bc
:1084e00000052000a8fd070081c42600200520000b
:1084f00082fd07000000eb0020079800080037000d
:108500002e0090004200dd000008b0006011b800ad
:10851000aefd07002e0090000000e8002007980044
:108520002e009000ed0f5000f5ff34006011b800f0
:10853000800b200082fd07000000eb002007980060
:10854000090037002e0090004200dd00c00bb00093
:108550000200200003f82b009cfd07002e00900075
:108560000000e800200798002e009000f80f50004f
:10857000f4ff3400011920000012200082fd0700e2
:1085800000412500515b2400008fbe001e00be008c
:10859000fc0e020000000000800078002012200085
:1085a00079fd07006011b8008012200087fd0700e8
:1085b0000200200003f82300c012200083fd070002
:1085c0000200200003f82300001320007ffd0700b5
:1085d0000200200003f82300002c20007bfd070090
:1085e0000200200003f82300402c200077fd070044
:1085f00002002000832c24004013200073fd07009c
:1086000021032000002820003cfd0700d1002000ad
:108610002028200039fd07008080eb004028200042
:1086200036fd07008000eb000015200033fd070039
:108630008000eb002015200030fd0700011920000c
:108640000016200050fd07001e00be00fc0e0200b8
:108650000000000080007800201620004afd07007e
:108660006011b8004016200058fd07006011b800e6
:108670008016200032fd07008000eb00c0162000ad
:1086800041fd07006011b800c02c20002cfd070040
:1086900011002000e01620003bfd07001100200023
:1086a0000017200038fd07008000eb002017200095
:1086b00035fd07008000eb00401720000ffd07008c
:1086c0000200200003182400801320003ffd070053
:1086d0006011b800c01320003cfd0700020020001c
:1086e000037024000014200038fd07006011b8005a
:1086f0004014200035fd0700020020000370240014
:108700008014200031fd07000081eb008081eb0028
:10871000c01320000afd07000081eb008081eb0000
:108720000014200006fd07000081eb008081eb00b3
:108730004014200002fd07000081eb008081eb0067
:1087400080142000fefc0700913e200080172000ce
:108750000dfd07008000eb00a01720000afd0700b8
:1087600031002000c017200007fd07008000eb004b
:108770000018200004fd0700e1ff2f002018200052
:1087800001fd0700e1ff2f0040182000fefc07005c
:10879000260007000c6c0200010000000800070022
:1087a00002002c0023012000001b2000e4fc070035
:1087b0000000eb00009e88000080fa000000060028
:1087c0000000fa0041012000002b2000cbfc070034
:1087d00081252000202b2000c8fc0700410120003b
:1087e000402b2000c5fc0700211c2000602b20002e
:1087f000c2fc0700a1002000802b2000bffc070066
:10880000a1002000c02b2000bcfc0700a10020001c
:10881000a02b2000b9fc070001322000e02b200033
:10882000b6fc07000080fa00000006000000fa0015
:10883000a100200000202000b0fc07008000eb0019
:1088400020202000d0fc0700e10120004020200073
:10885000aafc07008000eb0060202000cafc070093
:10886000a100200080202000a4fc07008107200038
:10887000a0202000c4fc070061042000c0202000cc
:108880009efc070041012000e0202000befc070004
:10889000a10020000021200098fc07008000eb00d0
:1088a00020212000b8fc07005100200040212000ba
:1088b00092fc07008000eb0060212000b2fc070062
:1088c00041062000802120008cfc07004138200058
:1088d000a021200089fc0700e1062000c021200023
:1088e000a9fc0700c103200060172000a6fc0700b8
:1088f0000080fa00000006000400fa000000eb000f
:10890000100798000d0037001e0090000000400086
:108910000020b00023fd0700000f78001e0090002b
:10892000000040000024b0009e00780073fc0700a7
:108930001e0090000000e800100798001e00900044
:10894000ee0f5000f0ff34000080fa000000060037
:108950000200fa00881f7800004f7800e0ab80002a
:108960008040780000c0eb0080c06000c0eb2000b9
:10897000014878001e84fb001e80fb00c1eb200034
:108980007efe070080407800c0eb20000174780074
:108990001e80fb00207c88004f0478000080fa00d5
:1089a000000006000200fa00881f7800004f7800df
:1089b000e0ab80008040780000c0eb0080c0600029
:1089c00060f82000014878001e84fb001e80fb0038
:1089d00061f8200069fe07008040780060f8200000
:1089e000017478004f0478000080fa00000006004f
:1089f0000400fa00000f7800d00220009e0f100043
:108a000003003a0010002000100798001a003700f9
:108a1000b00220009e0f100003003a00100020005a
:108a20001007980014003700e00220009e0f10008d
:108a300003003a0010002000100798000e003700d5
:108a4000900320009e0f1000030034000000eb0094
:108a50001007980008003700f00220009e0f100059
:108a600003003c000000eb001007980002003700f4
:108a700010002000100798001e0090000080fa00ef
:108a8000000006001400fa00881f780060079800b4
:108a900071079800020f98000040eb00004f78002b
:108aa0008e08900000c2b300804878000040eb00c0
:108ab00090409800fe0090006e009000941f02000d
:108ac0000000000050079800de0090006e0090004b
:108ad00000805000000478007e009000ce1b020051
:108ae0000000000000004400400798006e00900065
:108af000ce1b020000000000300798005e009000ce
:108b00000000e0004c003200030037004e009000ef
:108b10000000e800400798004e00900080007800b8
:108b20006e00900000804000904078000040eb0014
:108b30003057980000c2b30080cf500002003c00c4
:108b400011c0b300315798000041eb002257980044
:108b5000ce0090003e009000808f500002003d004b
:108b600010c0b30020579800be5090002e519000c6
:108b700002c060000004e000e4ff3a00be00900084
:108b80004e00900000805000100798000000eb009d
:108b900020079800220037004e00900080007800e7
:108ba0006e0090000080400010407800ff4f5000a1
:108bb000140034002e009000800078000e08900011
:108bc000008140004e009000800078006e00900010
:108bd000008040001040780000497800ae0090000e
:108be0000e089000008040008000e8000040eb008c
:108bf000804878004e0090000000e8004007980090
:108c00000400370010c0b300004f78003e00900011
:108c1000200798002e0090000000e8002007980030
:108c2000ae0090001e009000808f5000daff3500eb
:108c300010c0b300004f78001e80fb004f04780086
:108c40000080fa00000006007600fa00881f780015
:108c5000719b8000809b8000808f500003003a0051
:108c60000000eb00203f9800f8023700719b800065
:108c7000800c20000088b90080007800e00421000a
:108c8000e140780030c4b30080cf500042003a0089
:108c9000719b8000800c20000088b9008000e800f3
:108ca000e0042100e1407800d0c4b30080cf500040
:108cb00039003a00719b8000800c20000088b900c8
:108cc0008080e800e0042100e140780040c4b30067
:108cd00080cf500030003a00009f80004700de0047
:108ce0000000a200610060000004e00027003200e4
:108cf000519c8000709b8000808f500015003a00ce
:108d0000609c80000000e800609c8800609c8000ff
:108d1000e30f500011003400709b80000000e80059
:108d2000709b8800709b8000e30f500002003400ad
:108d30000000eb00709b88000000eb00309c880076
:108d40000000eb00609c88008000eb00213f980051
:108d5000be0237000000eb00609c8800709b800022
:108d6000509c8800709b800021372100000040004b
:108d70000100400010007800981602000100000079
:108d8000209f80000040a000209f8800100020004d
:108d9000203f9800ad023700709b80008000780073
:108da000800c20000088b90080007800e0042100d9
:108db00000804000ce1b0200000000005007980019
:108dc0000000eb00600798000080eb00400798006f
:108dd0000080eb00300798005f003700719b800037
:108de0006e019000800c20000088b90082004000d5
:108df000e0042100614078000000fb00103f980073
:108e0000a00320009e389000808f500005003200a3
:108e1000000520009e389000808f50003400320002
:108e20004a0037006e0090000000e80060079800dc
:108e3000719b80006e019000800c20000088b900ba
:108e400082004000e0042100614078008000fb00c7
:108e500000fd2f0000804000e90f500021003e007f
:108e6000709b800080007800800c20000088b90092
:108e700080007800e0042100008040006e0147007f
:108e8000a3002000ee009000246d0200010000000d
:108e90006e0090000000e800600798006e00470038
:108ea0004c1f020000000000400798006e004700c1
:108eb000104078000004e000070032006e00470018
:108ec000104078008000fb0000fd2f000080400073
:108ed000e90f5000200036000080eb0040079800aa
:108ee0001d0037000080eb00400798001a00370093
:108ef0006e0090000000e80060079800709b800002
:108f000080007800800c20000088b9008000780084
:108f1000e0042100008040006e014700a300200013
:108f2000ee009000246d0200010000006e00900031
:108f30000000e800600798006e0047004c1f020028
:108f40000000000030079800030037006e0090001a
:108f50000000e80060079800ee0090005e009000be
:108f6000808f50000a003d00719b80006e019000d0
:108f7000800c20000088b90082004000e00421003d
:108f8000e1407800c0c7b30080cf500093ff3a00a3
:108f90004e009000109c88004e0090000000e00001
:108fa00002003400ce009000219c8800709b80005d
:108fb000a1372100000040000100400010007800af
:108fc000109e88000040eb00004f7800109e80004b
:108fd000e10f500008003400109e8000e50f5000a3
:108fe00005003c004e0090000000e000020035004b
:108ff00010c0b300004f7800109e8000e10f5000b9
:109000000b003400109e8000e50f500008003c006b
:109010003e009000e10f5000030034003e0090003d
:10902000e50f50000200340010c0b300004f78007c
:109030001e04e0003d003200009f80000000e000c0
:1090400008003d00709c800025f60700e14f5000ad
:1090500004003a00009f8000f1ff2700010060003b
:10906000009f8800109f80004c00de000000a200de
:10907000610060000004e00029003200009f8000d1
:109080004700de000000a200610060000004e00074
:1090900023003200009f80000000e0002000350027
:1090a000519c8000709b8000808f500015003a001a
:1090b000609c80000000e800609c8800609c80004c
:1090c000e20f500011003400709b80000000e800a7
:1090d000709b8800709b8000e30f500002003400fa
:1090e0000000eb00709b88000000eb00309c8800c3
:1090f0000000eb00609c88000000eb00203f98001f
:10910000d20137000000eb00609c8800709b80005b
:10911000509c8800400020009816020001000000ca
:1091200011002000213f9800c80137003e00900048
:10913000e20f500002013a00719b80006e01900026
:10914000800c20000088b90082004000e00421006b
:10915000e1407800c0c7b30080cf5000ed003a0076
:109160006e0090000000e80060079800709b80008f
:1091700080007800800c20000088b9008000780012
:10918000e0042100008040006e014700a3002000a1
:10919000ee009000246d02000100000060079800be
:1091a0006e0047004c1f020000000000e0ab88008a
:1091b000e1ab8000f0072000808f500009003c00e8
:1091c000e0ab80008040780020df2000014878007c
:1091d000119f80000000220000807000109f880016
:1091e000cc003700e1ab800070082000808f500079
:1091f00095003a00119f800000002200008070005e
:10920000109f8800e0ab80008040780020df2000c5
:1092100001487800709b800080007800800c20005e
:109220000088b90080007800e00421000080400040
:109230006e014700a3002000ee009000246d0200a4
:1092400001000000600798006e0047004c1f0200fc
:10925000000000008040780030df200001487800e6
:10926000709b800080007800800c20000088b9008e
:1092700080007800e0042100008040006e0147007b
:10928000a3002000ee009000246d02000100000009
:10929000600798006e0047004c1f020000000000ad
:1092a0008040780040df200001487800709b8000fb
:1092b00080007800800c20000088b90080007800d1
:1092c000e0042100008040006e014700a300200060
:1092d000ee009000246d020001000000600798007d
:1092e0006e0047004c1f0200000000008040780024
:1092f00050df200001487800709b800080007800db
:10930000800c20000088b90080007800e004210073
:10931000008040006e014700a3002000ee00900096
:10932000246d020001000000600798006e004700f5
:109330004c1f0200000000008040780060df200029
:1093400001487800709b800080007800800c20002d
:109350000088b90080007800e0042100008040000f
:109360006e014700a3002000ee009000246d020073
:1093700001000000600798006e0047004c1f0200cb
:10938000000000008040780070df20000148780075
:10939000709b800080007800800c20000088b9005d
:1093a00080007800e0042100008040006e0147004a
:1093b000a3002000ee009000246d020001000000d8
:1093c000600798006e0047004c1f0200000000007c
:1093d0008040780080df200001487800709b80008a
:1093e00080007800800c20000088b90080007800a0
:1093f000e0042100008040006e014700a30020002f
:10940000ee009000246d020001000000600798004b
:10941000ee009000007d2000808f5000040034009a
:109420006e00900001832f0001004000600798004b
:109430006e0047004c1f02000000000080407800d2
:1094400090df200001487800e1ab8000b0082000e8
:10945000808f50002f003a00119f800000002200f2
:1094600000807000109f8800e0ab80008040780092
:1094700020df2000014878002000200050079800dd
:109480006e0090000000e8006007980011003700af
:10949000de019000719b80006e019000800c200026
:1094a0000088b90082004000e0042100614078009b
:1094b0008040780020df2000817178005e009000fd
:1094c0000000e800500798006e0090000000e800df
:1094d00060079800719b80006e019000800c200056
:1094e0000088b90082004000e0042100614078005b
:1094f000ff4f5000e6ff3c005e0090000080e90056
:10950000500798005e0090008040780030df200017
:1095100001487800709b80000000e800709b880084
:10952000709b8000e30f5000020034000000eb004d
:10953000709b880010002000203f9800c300370077
:109540003e009000e30f500018003a00709b80002e
:1095500080007800800c20000088b900800078002e
:10956000e004210000804000801f780020f82c00db
:10957000801f78003e1f020000000000e4875700b3
:10958000709b80000000e800709b8800709b80004a
:10959000e30f5000020034000000eb00709b8800d5
:1095a00011002000213f9800a80037003e009000e5
:1095b000e40f50009b003a00719b80006e01900008
:1095c000800c20000088b90082004000e0042100e7
:1095d000e1407800c0c7b30080cf500028003a00b7
:1095e0000000eb00100798006e0090000000e800fb
:1095f00060079800110037009e019000719b800069
:109600006e019000800c20000088b90082004000ac
:10961000e0042100e14078006e0047000080410036
:10962000014878006e0090000000e8006007980094
:109630001e0090000000e80010079800ee00900067
:109640005e009000808f5000ebff35009e00900080
:109650006e00470080804000d0c0b3008048780092
:109660001e0090000000e800100798009e00900087
:109670006e004700808040000040eb00804878008a
:10968000709b8000a13721000000400001004000d5
:109690009000780021079800709b80000000e8008f
:1096a000709b8800709b8000e30f50000200340024
:1096b0000000eb00709b88004e0090000000e0006e
:1096c0001b003500c0172000c1f907000004780016
:1096d00000182000bef9070000017800809b800080
:1096e00080007800800c20000088b900800078009d
:1096f000e004210000804000800078002e009000ef
:10970000801f7800881f7800821f78004e0090002c
:10971000801f780070f82c00801f7800010078000e
:10972000f81f020000000000ea8757001000370011
:10973000809b800080007800800c20000088b900a9
:1097400080007800e0042100008040008000780064
:109750002e009000801f780010fa2c00801f7800e7
:1097600001007800f81f020000000000e4875700a5
:109770006e00470042062000c12b2000a01202000c
:10978000010000000000e0000b003a00809b800018
:1097900080007800800c20000088b90080007800ec
:1097a000e004210000804000d1fa2c00c21f02001a
:1097b000000000000a003700809b800080007800d5
:1097c000800c20000088b90080007800e0042100af
:1097d00000804000ee004700c21f020000000000b1
:1097e000809b8000a13721000000400081004000e4
:1097f0004000200080087800809b80000000e80086
:10980000809b8800809b8000e30f500002003400a2
:109810000000eb00809b880011002000213f980091
:109820000a003700709b80000000e800709b8800f1
:10983000709b8000e30f5000020034000000eb003a
:10984000709b88000000eb00203f98002e389000ad
:109850004f0478000080fa00000006000400fa00bf
:10986000819b8000709b8000008f50001e00e000f4
:1098700002003d001e007800640f40002000200020
:109880009e0f100003003c001000200010079800fd
:10989000020037000000eb00100798001e00900047
:1098a0000080fa00000006000200fa00000f7800b5
:1098b000eaff07000004e0001f003200809b8000e8
:1098c000a13721000000400081004000200020005e
:1098d00080087800809b800080007800800c200049
:1098e0000088b90080007800e0042100008040007a
:1098f00061fb2c0003000900315878004000b100e2
:10990000809b8000213721000000400001004000c2
:109910001e087800809b80000000e800809b880083
:10992000809b8000e30f500003003400809b800088
:1099300064005000809b88000080fa000000060050
:109940000400fa00004f7800d0c2b3009e4f100010
:1099500003003a00100020001007980010003700a4
:10996000b0c2b3009e4f100003003a001000200068
:10997000100798000a0037001e00fb0001fd2f00b1
:1099800001004000e90f500003003e0010002000dd
:1099900010079800020037000000eb001007980045
:1099a0001e0090000080fa00000006000001780010
:1099b00000000000000000000201e900fcff3a0086
:1099c0008100e900f9ff3a00000006000000eb000a
:1099d0008000eb00820f200092018800020120002d
:1099e0001200ba00820f200092018800220120009c
:1099f0009200ba00c808dd00f00fb200010040007c
:109a000000000600801f7800820f2000920188006d
:109a1000020120000049bb0000002400003b880038
:109a20004200f800000e20004220b7005005200040
:109a3000303b8800a00a2000303b880061e7a80086
:109a400000000000000000004200f9004f00780014
:109a50004800de00820f20009201880022012000d1
:109a60000049bb0000002400003b88004200f800d1
:109a7000000e20004220b70050052000303b880037
:109a8000a00a2000303b880061e7a8000000000029
:109a9000000000004200f900000006000000d000b5
:109aa000031920000302d000611978002000b000e3
:109ab0000400e100010039000000eb008301e9002f
:109ac000f9ff3a000000060001004000810140005b
:109ad0000000eb008000eb003302780004f0a600e9
:109ae000060037000482ea000402e8000400500087
:109af000050031008100e900030037000400400048
:109b0000010039008100e8000201e900f2ff3a009b
:109b10000000060071015000030120007082510016
:109b200063807800e48278000028e1003e00310084
:109b30002400b000e48278000028e1003a003100ff
:109b40002400b000e48278000028e10036003100f3
:109b50002400b000e48278000028e10032003100e7
:109b60002400b000e48278000028e1002e003100db
:109b70002400b000e48278000028e1002a003100cf
:109b80002400b000e48278000028e10026003100c3
:109b90002400b000e48278000028e10022003100b7
:109ba0004400b000e48278000028e1001e0031008b
:109bb0002400b000e48278000028e1001a0031009f
:109bc0002400b000e48278000028e1001600310093
:109bd0002400b000e48278000028e1001200310087
:109be0002400b000e48278000028e1000e0031007b
:109bf0002400b000e48278000028e1000a0031006f
:109c00002400b000e48278000028e1000600310062
:109c10002400b000e48278000028e1000200310056
:109c20000300d100000006002300b0000201e9009b
:109c3000baff3a00f0ff2f0000000600710150004b
:109c4000030120007082510063807800e482780074
:109c50000500e1003e0031002400b000e4827800fd
:109c60000500e1003a0031002400b000e4827800f1
:109c70000500e100360031002400b000e4827800e5
:109c80000500e100320031002400b000e4827800d9
:109c90000500e1002e0031002400b000e4827800cd
:109ca0000500e1002a0031002400b000e4827800c1
:109cb0000500e100260031002400b000e4827800b5
:109cc0000500e100220031004400b000e482780089
:109cd0000500e1001e0031002400b000e48278009d
:109ce0000500e1001a0031002400b000e482780091
:109cf0000500e100160031002400b000e482780085
:109d00000500e100120031002400b000e482780078
:109d10000500e1000e0031002400b000e48278006c
:109d20000500e1000a0031002400b000e482780060
:109d30000500e100060031002400b000e482780054
:109d40000500e100020031000300d1000000060020
:109d50002300b0000201e900baff3a00f0ff2f0033
:109d60000000060000000600000278000000eb0082
:109d7000b44178004801de008381fb0003016900e3
:109d80000201d00003a52c00030141004800dd00c2
:109d9000120068008100e900f5ff3a0000000600ab
:109da0000002eb008002eb0003012000ca62a90060
:109db00000cab300165002000000000000000000be
:109dc000000000000000000006500200000000003b
:109dd0004801dd0006500200000000000080fb008a
:109de00000004100ca62a8004280de0000f0a60028
:109df000060037000080ea000000e8000002520080
:109e0000050031008502e90003003700000242002e
:109e1000010039008502e8008301e900e3ff3a0010
:109e20008500780004007800000006000002eb00c6
:109e30008002eb0003012000e922a90000cab30060
:109e400016500200000000000000000000000000aa
:109e50000000000006500200000000004801dd0084
:109e600006500200000000000080fb0000004100de
:109e7000e922a8004280de0000f0a60006003700bc
:109e80000080ea000000e8000002520005003100f6
:109e90008502e9000300370000024200010039009a
:109ea0008502e8008301e900e3ff3a0085007800bd
:109eb00004007800000006000002eb008002eb00c6
:109ec0000003eb008003eb000301200000cab30095
:109ed000ca62a9001650020000000000ca62a80071
:109ee000e922a9001650020000000000e922a800a3
:109ef000ca62a90006500200000000004801dd000f
:109f000006500200000000000080fb00000041003d
:109f1000ca62a8004280de0000f0a60006003700fa
:109f20000080ea000000e800000252000500310055
:109f30008502e900030037000002420001003900f9
:109f40008502e800e922a900065002000000000096
:109f50004801dd0006500200000000000080fb0008
:109f600000004100e922a8004280de0000f0a600c7
:109f7000060037000080ea000000e80000035300fc
:109f8000050031008703e9000300370000034300a8
:109f9000010039008703e8008301e900cbff3a00a4
:109fa0008502d1008480d3008502d1008180d30056
:109fb0008703d1000681d3008703d1000281d3003b
:109fc00040582100a418b400a418b4000108780077
:109fd000608a2100c61bb400c61bb40002087800ca
:109fe00000192000a438ec00a418e3000100390097
:109ff000a438ef00c63bec00c61be30001003900ab
:10a00000c63bef000200780000000600411380000c
:10a010006022af00feff37006862ef006002ae0012
:10a02000feff370068c2bf00000006004113800039
:10a030006022af00feff370068e2b7006002ae00aa
:10a04000feff370041138000000006004019880021
:10a05000010120000000ef0085a0a90021e3a80075
:10a0600085a0ae00feff370085a0a9000003b40064
:10a070008100e900faff3a0021e3a9000000060090
:10a08000401b8800010120000000ef0086a0a9000d
:10a0900061e3a80086a0ae00feff370086a0a900fd
:10a0a0004003b4008100e900faff3a0061e3a9002f
:10a0b000000006008001780068c2bf006022af0087
:10a0c000feff37000240780068e2b7006002ae0091
:10a0d000feff370068c2bf00805878008301e900a6
:10a0e000f6ff3a00000006000001780068c2bf00d9
:10a0f0006022af00feff37003140780068e2b70011
:10a100006002ae00feff370068c2bf000201e90036
:10a11000f7ff3a00000006003000b00000017800b0
:10a12000a2407800c808dd00a241780081c041004b
:10a13000224078004800dd009241780000c04100d4
:10a1400000000600005978004880de0000597800c1
:10a1500001597800c888de00014978000000060037
:10a160001000b00000017800224078004800dd00b7
:10a170009241780000c0410000000600805878003d
:10a180004880de008058780000000600000178005a
:10a19000b2407800c808dd00b241780081c04100bb
:10a1a000324078004800dd009241780000c0410054
:10a1b000000006003200b000005178004880de0048
:10a1c0000051780001517800c888de00014978000c
:10a1d0000000060000017800324078004800dd00f1
:10a1e0009241780000c04100000006001100b0005c
:10a1f000805078004880de00805078000000060023
:10a200000a00fa00881f7800e0162000e83e0200ed
:10a210000000000040079800809f8000919f800010
:10a220004608de0001002000610060000004e0003c
:10a2300088013200009f80004500de000000a2007f
:10a24000610060000004e00003003a004e0090004e
:10a25000e10f50007f013a004e009000803802006c
:10a26000000000000004e000780032004e00900082
:10a27000ec360200000000006047980000df20007c
:10a28000104078000004e00039003a00e0de2000d1
:10a2900010407800f04f500003003a006e409000ec
:10a2a000f04f500032003200e0de20001040780015
:10a2b000f04f500010003a006e409000e34f500005
:10a2c0000d003a00c0de2000104078000004e000dd
:10a2d00009003200d1de200010c0b30080487800b1
:10a2e000506f80000000e900506f8800506f8000c0
:10a2f0000000e900506f8800c0de200010407800a8
:10a300000004e0000b003200d0de20001040780096
:10a310000004e00007003a00516f800060d8200080
:10a320006e41900082707800506f80000000e8005d
:10a33000506f8800e0de200010407800f04f5000a1
:10a3400008003a006e409000e24f500005003a00cd
:10a35000c0de200011c0b300014878000000eb000f
:10a36000506f8800e0de2000ee4090000148780049
:10a37000c0de2000104078000004e00031003a0008
:10a380006e409000ff4f50000b003e0000df2000a9
:10a39000104078000004e0000700320011df2000c8
:10a3a00010c0b30080487800526f800061d8200050
:10a3b0000040eb0000f1780000df20001040780042
:10a3c0000004e0001200320010df2000104078008e
:10a3d0000004e0000e003a00516f800060d82000b9
:10a3e0006e41900082707800506f80000000e8009d
:10a3f000506f8800516f800030062000808f500021
:10a4000003003400506f80000000e900506f8800a6
:10a41000ee409000c0c3b30080cf500009003a0066
:10a4200000df2000104078000004e00005003a0042
:10a4300000df200011c0b300014878000000eb00ed
:10a44000506f8800548a020001000000c0de200026
:10a45000104078000004e000dc003200d0de200074
:10a46000104078000004e000d800320070d82000ce
:10a47000104078000084fb0020172000e83e020016
:10a4800000000000800f54000400320070d820004b
:10a49000104078000004e000c0003a000040eb00eb
:10a4a000104798000000eb00200798000a003700d2
:10a4b000ae00900060d82000614078009e4090007f
:10a4c00096d3020001000000104798002e00900073
:10a4d0000000e80020079800516f80002e009000d7
:10a4e000810f5000f2ff3500516f800060d82000ce
:10a4f000e14078001e40900080cf5000a7003a0055
:10a5000090d82000104078000080fb0020079800c1
:10a510002e0090004800dd0020079800a0d8200001
:10a52000104078008080fb002e0090000100400069
:10a530002007980080d8200010407800e14f50009c
:10a5400096003a0060d8200090407800f0de2000ad
:10a55000014878000000eb00100798000a0037005f
:10a560001e0190001e009000e500400060d8200011
:10a57000e140780020df2000017178001e0090008b
:10a580000000e800100798009e0090002e00900048
:10a59000808f5000f2ff350010c0b300b1060700f5
:10a5a000e0162000e83e020000000000400798008e
:10a5b00020172000e83e020000000000004f780055
:10a5c0008040eb004e009000ac1d02000100000036
:10a5d000a0002000de3502000000000001c1b30031
:10a5e0004e009000ac1d02000100000021c0b3002d
:10a5f0004e009000ac1d0200010000009e4078005b
:10a600004e009000ac1d0200010000008040eb00f5
:10a610001e40780096d30200010000001047980009
:10a62000f0de2000904078004e009000ac1d02004b
:10a6300001000000f0de2000104078009e409000f5
:10a6400096d30200010000001047980011c0b3002b
:10a650004e009000ac1d0200010000009e409000e2
:10a6600010c0b30096d3020001000000104798000c
:10a670002e00900002102000110009000200d800f6
:10a6800060479800ee4090004e009000ac1d020024
:10a69000010000009e4090006e40900096d30200a2
:10a6a00001000000104798002e00900080407800c4
:10a6b00000c0eb0000c0600060479800ee409000d2
:10a6c0004e009000ac1d0200010000009e40900072
:10a6d0006e40900096d302000100000010479800e1
:10a6e0000000eb00100798001c0037001e009000cf
:10a6f000c1eb200060c17800624798006e40900076
:10a70000f04f500009003a0001c1b3004e00900024
:10a71000ac1d0200010000009e4090006e409000c1
:10a7200096d302000100000010479800ee40900010
:10a730004e009000ac1d0200010000009e40900001
:10a740006e40900096d30200010000001047980070
:10a750001e0090000000e800100798009e00900086
:10a76000207c8000808f5000e0ff39009e409000e8
:10a770004e009000ac1d02000100000001c1b300ba
:10a780004e009000ac1d02000100000031c0b3007b
:10a790004e009000ac1d020001000000d1de200040
:10a7a0000040eb0080487800c1de20000040eb0054
:10a7b0008048780011df20000040eb0080487800de
:10a7c00001df20000040eb008048780000df20001f
:10a7d000104078000004e0001e00320010df20006e
:10a7e000104078000004e0001a0032001c0007004e
:10a7f0000004e0000b0032004e009000f09d880045
:10a8000060d82000801f7800a01a2c00801f7800dc
:10a81000da1f020000000000e48757000000eb0090
:10a82000f09d880011df20000040eb008048780098
:10a8300001df20000040eb0080487800d1de2000de
:10a840000040eb0080487800c1de20000040eb00b3
:10a85000804878004f0478000080fa00000006006d
:10a860000400fa00881f78000000eb00000f780059
:10a870000b0037001e0478009e00780060d820008e
:10a88000614078000080fb00300c020000000000f6
:10a890008040780060d82000017478001e0fe80026
:10a8a0001e04780060d82000ce1b020000000000cb
:10a8b000800f5400efff390060d82000f11a2c00ff
:10a8c000941f0200000000000000e00004003200bd
:10a8d0002a0007000080fb001007980023003700c3
:10a8e00060d82000411b2c00941f020000000000d3
:10a8f0000000e00004003200760207000080fb0048
:10a90000100798001900370060d82000911b2c0018
:10a91000941f0200000000000000e000040032006c
:10a92000e30307000080fb00100798000f003700ca
:10a9300060d82000c11b2c00941f02000000000002
:10a940000000e000040032002a0407000080fb0041
:10a95000100798000500370061d820000040eb0088
:10a96000804878000000eb00100798001e0090005f
:10a970004f0478000080fa00000006006200fa0030
:10a98000889fbe008a9fbe006000b800400f9800fc
:10a99000510f98000000eb00200f9800500020009d
:10a9a000300f980060d82000ce1b0200000000008d
:10a9b000e50f5000610036007c0147008042eb004b
:10a9c0000042eb0063022000be08900060d8200027
:10a9d00013210700300f98007c004700ce1b0200b7
:10a9e00000000000100f98007c0047001040780025
:10a9f0008000fb0000fd2f0000804000e90f5000a8
:10aa000008003e001e0890000000e0000500340031
:10aa10007c0047004c1f020000000000200f98003f
:10aa2000430037001e089000002f98008e289000e9
:10aa3000e28f5000130032000e299000e30f510006
:10aa40002d0032008e299000e18f5100010032006c
:10aa50003700370060d8200041052000e81f0200c1
:10aa6000000000000000e000310032004e089000bd
:10aa7000de0890000000a000400f9800510f9800e1
:10aa80002b00370060d82000f11b2c00941f02001f
:10aa9000000000000000e000080032004e089000b6
:10aaa000de08900042202000030120000200700018
:10aab00083807000400f9800510f980060d82000ec
:10aac000211c2c00941f0200000000000000e00088
:10aad000170032004e089000de089000024020006f
:10aae000830020000200700083807000400f9800f7
:10aaf000510f98000e00370060d82000511c2c0028
:10ab0000941f0200000000000000e0000800320076
:10ab10004e089000de08900002022800430020004a
:10ab20000200700083807000400f9800510f980061
:10ab30001e0890000000e0009fff3c004e089000bf
:10ab4000de089000e00f5000e08f580005003a004a
:10ab5000849f8000959f8000440f9800550f9800b7
:10ab60001e003700829f8000939f80004e08900057
:10ab7000de08900000027800810278000200780070
:10ab80008300780000016200018062006102b80069
:10ab9000142f9800252f98001e289000ae289000b2
:10aba000c000dd0000002000102f9800212f980029
:10abb0001e289000ae2890006112b800142f980053
:10abc000252f98001e299000ae29900002007000e9
:10abd00083807000400f9800510f98002e0890005d
:10abe0000000e0000700320020172000e83e0200cd
:10abf00000000000800078002e089000808f500038
:10ac000062013a0020172000e83e02000000000028
:10ac100061d82000801f7800901c2c00801f7800d5
:10ac200001007800f81f020000000000e4875700d0
:10ac300010c0b300404798004e08900061006000cb
:10ac40000004e00017003200070d070010a080008c
:10ac500021a080003e0f0200000000007c0247009f
:10ac6000809fbe00829fbe00201d2c00801f7800a8
:10ac700004007800f81f020000000000ea87570077
:10ac800060d82000fc004700c21f02000000000046
:10ac900010a0800021a08000430107000040eb00cd
:10aca000404798004e089000de08900042202000a7
:10acb0000301200000027800810278000200780081
:10acc0008300780000016200018062006102b80028
:10acd000342f9800452f98003e289000ce289000f1
:10ace000c000dd0000002000302f9800412f9800a8
:10acf0003e289000ce2890006112b800342f9800b2
:10ad0000452f98003e299000ce2990000200700047
:10ad100083807000e00f5000e08f5800290032005f
:10ad2000fa0c07004e089000de089000ce09dd0006
:10ad30004200de0000807100c208de006100600099
:10ad40000004e00005003200f49f800005a08000b0
:10ad500074079800050f980004003700b09f80002a
:10ad6000c19f800070079800010f98007e0090003e
:10ad70008e0890003e0f0200000000007c02470099
:10ad8000809fbe00829fbe00901d2c00801f780017
:10ad900004007800f81f020000000000ea87570056
:10ada00060d82000fc004700c21f02000000000025
:10adb0007e0090008e089000fb0007000040eb0032
:10adc000404798004e089000de08900002402000a6
:10add00083002000000278008102780002007800e1
:10ade0008300780000016200018062006102b80007
:10adf000542f9800652f98005e289000ee28900050
:10ae0000c000dd0000002000502f9800612f980046
:10ae10005e289000ee2890006112b800542f980030
:10ae2000652f98005e299000ee29900002007000c6
:10ae300083807000e00f5000e08f58002600320041
:10ae4000760e07004e089000de0890004308de00f2
:10ae500001002000610060000004e00005003200f5
:10ae6000b4a18000c5a18000340798004507980070
:10ae70000400370050a1800061a1800030079800d5
:10ae800041079800fc0047003e019000ce01900071
:10ae9000829fbe00101e2c00801f780001007800e9
:10aea000f81f020000000000e687570060d820006d
:10aeb000fc004700c21f0200000000003e0090009e
:10aec000ce0090006e0c020000000000b6000700eb
:10aed0000040eb00404798004e089000de089000cc
:10aee000020228004300200000027800810278005e
:10aef0000200780083007800000162000180620097
:10af00006102b800742f9800053798007e289000e1
:10af10008e309000c000dd0000002000702f9800ef
:10af2000013798007e2890008e3090006112b800a2
:10af3000742f9800053798007e2990008e3190007c
:10af40000200700083807000e00f5000e08f580016
:10af500084003200310e07004e089000de08900099
:10af6000c109dd004f00de0000807100cf08de0067
:10af7000610060000004e00009003200e0402100b0
:10af800020029000b002900074079800050f98000e
:10af9000e04021001001be005207980063079800ae
:10afa0004e089000de0890004208de0001002000fc
:10afb000610060000004e0000900320060412100ef
:10afc00020029000b002900074079800050f9800ce
:10afd000604121001001be005207980063079800ed
:10afe0004e089000de089000cb09dd004500de0031
:10aff00000807100c508de00610060000004e00010
:10b00000090032006040210020029000b002900050
:10b0100074079800050f9800604021001001be00e1
:10b020005207980063079800020020004333240071
:10b030007e0090008e089000800d0200000000004d
:10b040003e0f02000000000044742100154425005a
:10b05000b61f2200970024007c0f020000000000b1
:10b06000a20e02000000000070079800010f980077
:10b0700002002000433324005e009000ee009000a8
:10b08000800d0200000000003e0f020000000000e2
:10b090004474210015442500b61f220097002400a7
:10b0a0007c0f020000000000a20e02000000000061
:10b0b00050079800610798007e0090008e0890006d
:10b0c0003e0f0200000000000004be000205be00aa
:10b0d0005e009000ee0090003e0f020000000000b5
:10b0e0007c024700889fbe008a9fbe00809fbe00f2
:10b0f000829fbe00801e2c00801f78000400780014
:10b10000f81f020000000000f287570060d82000fe
:10b11000fc004700c21f02000000000002002000e7
:10b12000134624007e0090008e089000301002002c
:10b13000000000000000e0000100350004003700be
:10b140007e0090008e089000170007000300370073
:10b150005e009000ee009000130007000040eb003e
:10b16000404798004e4090000004e0000400320088
:10b1700060d82000611f2c00c21f020000000000e8
:10b180001300200073279800020037000002eb0034
:10b19000742798007e2090004f05be004f04be002b
:10b1a0000080fa00000006001e00fa00500f980010
:10b1b000610f980090a48000cf80de006e0c02002a
:10b1c000000000000200200003122400e80d02002d
:10b1d0000000000010079800210798000000eb0015
:10b1e000000f780002002000032724001e009000ba
:10b1f000ae009000f80e0200000000000000e00029
:10b2000008003c006011b8001e009000ae009000e5
:10b2100030100200000000000000e00001003500d6
:10b22000020037001e00a000110037001e00900031
:10b23000ae0090003e0f02000000000066024700d2
:10b24000809fbe00829fbe00c01f2c00801f780020
:10b2500004007800f81f020000000000ea87570091
:10b2600060d82000e6004700c21f02000000000076
:10b2700002002c0093472c005e089000ee0890001e
:10b2800030100200000000000000e0000100340067
:10b29000010037001e10a000e60047001e007800e5
:10b2a000801f780040202c00801f7800010078006b
:10b2b000f81f020000000000e487570060d820005b
:10b2c000e6004700c21f0200000000000080fa00f4
:10b2d000000006004800fa00889fbe008a9fbe005a
:10b2e0008c9fbe000000eb0030079800500020004b
:10b2f0004007980060d82000ce1b0200000000002c
:10b30000e50f500029013600710147008042eb0033
:10b310000042eb0063022000ce00900060d82000c5
:10b32000bf1e07004007980071004700ce1b0200b7
:10b3300000000000200798007100470010407800ce
:10b340008000fb0000fd2f0000804000e90f50004e
:10b3500013003e002e0090000000e00010003400ba
:10b36000710047004c1f02000000000030079800e9
:10b37000710147008042eb000042eb0063022000b5
:10b38000ce00900060d82000a51e0700400798005e
:10b3900071004700ce1b020000000000200798004b
:10b3a00060d82000a1202c00941f020000000000a3
:10b3b000000f78001e00e000fc0032002e0090001c
:10b3c000e20f5000f90034009e00780060d82000a1
:10b3d00062001000008040004007980010c0b300d9
:10b3e0002047980071014700e5c2b3000042eb001e
:10b3f00063022000ce00900060d82000881e070065
:10b400004007980071004700ce1b020000000000ba
:10b41000e10f500002003e000040eb002047980082
:10b42000710047004c1f02000000000080407800bf
:10b430006a004700214098006a00470020409000c1
:10b440000004e000040035006a004700204090003e
:10b45000f74f5000020034000040eb0020479800f6
:10b4600071014700e5c2b300e4c2b30063022000eb
:10b47000ce00900060d82000691e070040079800a9
:10b4800071004700ce1b020000000000e10f5000d9
:10b4900002003e000040eb0020479800710047008a
:10b4a0004c1f020000000000804078006a00470046
:10b4b000114098006a004700104090000004e0002e
:10b4c000050035006a00470090409000b0c3b3000b
:10b4d00080cf5000020034000040eb00204798006d
:10b4e00071014700b5c3b300e4c2b300630220009a
:10b4f000ce00900060d82000491e07004007980049
:10b5000071004700ce1b020000000000e10f500058
:10b5100002003e000040eb00204798007100470009
:10b520004c1f020000000000804078006a004700c5
:10b53000014878006a004700104078000004e000ed
:10b54000050035006a00470090407800b0c3b300a2
:10b5500080cf5000020034000040eb0020479800ec
:10b5600071014700f5c2b300b4c3b3006302200009
:10b57000ce00900060d82000291e070040079800e8
:10b5800071004700ce1b020000000000e10f5000d8
:10b5900002003e000040eb00204798007100470089
:10b5a0004c1f020000000000804078006a00470045
:10b5b000414098006a004700404090000004e000cd
:10b5c000040034006a00470040409000ff4f5000e4
:10b5d000020034000040eb00204798007101470052
:10b5e000f5c2b300f4c2b30063022000ce009000a5
:10b5f00060d820000a1e070040079800710047002d
:10b60000ce1b020000000000e10f500002003e00cf
:10b610000040eb0020479800710047004c1f0200db
:10b6200000000000804078006a0047005140980008
:10b630006a004700504090000004e000040034001d
:10b640006a00470050409000ec4f50000200340068
:10b650000040eb002047980071014700b5c3b300dc
:10b66000f4c2b30063022000ce00900060d8200036
:10b67000eb1d07004007980071004700ce1b020039
:10b6800000000000e10f500002003e000040eb000f
:10b6900020479800710047004c1f02000000000086
:10b6a000804078006a004700614098006a004700c7
:10b6b000604090000004e000050035006a0047008b
:10b6c000e040900030c6b30080cf5000020034004c
:10b6d0000040eb0020479800710147008042eb00da
:10b6e000b4c3b30063022000ce00900060d82000f5
:10b6f000cb1d0700400798007100470010407800fc
:10b700000004e00011003200710047004c1f0200ed
:10b7100000000000804078006a0047003140980037
:10b720006a004700304090000004e000040034004c
:10b730006a00470030409000e74f50000600340098
:10b740000040eb002047980003003700ea00470064
:10b7500010c0b300b04098003e0090000000e00030
:10b760000900320020172000e83e0200000000001f
:10b77000800078003e009000808f50000200320070
:10b780000040eb00204798002e4090000004e000ad
:10b79000060032006a004700c803020002000000f1
:10b7a00080d62100c8ff0200010000003e0090008a
:10b7b0000000e0000700320020172000e83e0200f1
:10b7c00000000000800078003e009000808f500054
:10b7d0002f003a006a004700c8ff02000100000085
:10b7e0006a004700304090000004fb006a004700f8
:10b7f000604090008004fb006a00470050409000c9
:10b800000005fb006a004700404090008005fb00f7
:10b810006a004700104078000006fb006a004700fd
:10b82000104090008006fb006a0047002040900016
:10b830000000fb003027980020172000e83e02009f
:10b840000000000061d82000881f7800891f780060
:10b850008a1f78008b1f78008c1f78008d1f78005e
:10b860003e219000821f7800801f7800d0202c009d
:10b87000801f780001007800f81f0200000000001f
:10b88000f2875700100020002027980002003700a0
:10b890000001eb00222798002e2090004f06be00ea
:10b8a0004f05be004f04be000080fa0000000600f5
:10b8b0003a00fa000000eb0010079800300020006a
:10b8c0002007980060d82000ce1b02000000000076
:10b8d000e30f500025003600660147008042eb0070
:10b8e0000042eb0063022000ae00900060d8200010
:10b8f0004b1d07002007980066004700ce1b020082
:10b9000000000000000f780066004700104078003b
:10b910008000fb0000fd2f0000804000e90f500078
:10b9200012003e001e00e0001000340066004700d8
:10b930004c1f02000000000010079800660147003d
:10b940008042eb000042eb0063022000ae0090005a
:10b9500060d82000321d07002007980066004700cd
:10b96000ce1b020000000000000f78001e009000b7
:10b970000000e0000700320020172000e83e02002f
:10b9800000000000800078001e009000808f5000b2
:10b9900013003a00b0232c004c1f020000000000ee
:10b9a0008000780062d82000d0232c00801f78000f
:10b9b000811f7800f0232c00801f780010242c00b9
:10b9c000801f780002007800f81f020000000000cd
:10b9d000e887570010002000401f98000200370041
:10b9e0000000eb00401f98004e1890000080fa0005
:10b9f000000006004c00fa00889fbe008a9fbe002f
:10ba00000000eb005007980030002000600798000d
:10ba100060d82000ce1b020000000000e30f5000a1
:10ba200026003600700147008042eb000042eb0028
:10ba300063022000ee00900060d82000f81c070090
:10ba40006007980070004700ce1b02000000000055
:10ba50004007980070004700104078008000fb000d
:10ba600000fd2f0000804000e90f500013003e0051
:10ba70004e0090000000e00010003400700047000d
:10ba80004c1f0200000000005007980070014700a2
:10ba90008042eb000042eb0063022000ee009000c9
:10baa00060d82000de1c0700600798007000470087
:10bab000ce1b020000000000400798005e009000ce
:10bac0000000e0000700320020172000e83e0200de
:10bad00000000000800078005e009000808f500021
:10bae00059013a00b0232c004c1f02000000000056
:10baf0000004780020172000e83e0200000000004b
:10bb00008000780062d82000d0232c00801f7800ad
:10bb1000881f7800f0232c00801f7800811f780098
:10bb200080252c00801f780002007800f81f02009a
:10bb300000000000ea875700809f8000919f8000ee
:10bb4000610060000004e0000400320060d82000c2
:10bb500021272c00c21f020000000000809f8000ef
:10bb6000919f80004e09dd004200de000000710060
:10bb7000c208de00610060000004e0002c0032001a
:10bb800020122000e83e020000000000cf80de000e
:10bb90006e0c0200000000003e0f020000000000da
:10bba000247e270035dd2200b6432900b70124009a
:10bbb0003410020000000000a20e0200000000008d
:10bbc000200798003107980080122000163f0200dd
:10bbd000000000003e0f0200000000000004be0054
:10bbe0000205be002e009000be0090003e0f020035
:10bbf0000000000070024700889fbe008a9fbe00c0
:10bc0000809fbe00829fbe0020282c00801f7800ed
:10bc100004007800f81f020000000000f2875700bf
:10bc200060d82000f0004700c21f020000000000a2
:10bc3000809f8000919f800002202000030120004f
:10bc4000000278008102780002007800830078000a
:10bc500000016200018062006102b80024279800a0
:10bc6000352798002e209000be209000c000dd00f7
:10bc70000000200020279800312798002e209000f7
:10bc8000be2090006112b800242798003527980044
:10bc90002e219000be219000020070008380700071
:10bca000e00f5000e08f58003200320000162000f4
:10bcb000e83e020000000000cf80de006e0c0200b3
:10bcc000000000003e0f020000000000e496260085
:10bcd00055432200e61e2000d70224003410020043
:10bce00000000000247e270035dd2200b643290035
:10bcf000b70124003410020000000000a20e020070
:10bd0000000000002007980031079800401620002e
:10bd1000163f0200000000003e0f0200000000007d
:10bd20000004be000205be002e009000be00900080
:10bd30003e0f02000000000070024700889fbe0016
:10bd40008a9fbe00809fbe00829fbe0050292c00ab
:10bd5000801f780004007800f81f02000000000037
:10bd6000f287570060d82000f0004700c21f020091
:10bd700000000000809f8000919f80000240200012
:10bd80008300200000027800810278000200780021
:10bd90008300780000016200018062006102b80047
:10bda00044279800552798004e209000de209000f0
:10bdb000c000dd00000020004027980051279800b7
:10bdc0004e209000de2090006112b80044279800b9
:10bdd000552798004e219000de219000020070004f
:10bde00083807000e00f5000e08f58006100320047
:10bdf0000040eb00004f780000192000fe3e0200da
:10be0000000000004308de00010020006100600027
:10be10000004e0001f0032001e04e0001d003a0094
:10be200080192000e83e0200000000001007980082
:10be30001e0090004800dd0010079800a0192000a7
:10be4000e83e020000000000800078001e00900024
:10be50000100400010079800f00047009e0190008c
:10be6000831f7800702a2c00801f78000100780062
:10be7000f81f020000000000e487570060d820008f
:10be8000f0004700c21f02000000000010c0b30015
:10be9000004f7800001a2000fe3e02000000000063
:10bea0004308de0001002000610060000004e000a3
:10beb0001f0032001e04e0001d003a00801920001f
:10bec000e83e020000000000100798001e009000ed
:10bed0004800dd0010079800a0192000e83e02008d
:10bee00000000000800078001e009000010040006b
:10bef00010079800f00047001e029000841f780091
:10bf0000702a2c00801f780001007800f81f0200c2
:10bf100000000000e487570060d82000f0004700d0
:10bf2000c21f02000000000010c0b300004f7800e4
:10bf3000809f8000919f8000c60add004a00de00dd
:10bf400000807200ca08de00610060000004e000aa
:10bf5000080032001e04e00006003a0060d820000d
:10bf6000912b2c00c21f02000000000010c0b30083
:10bf7000004f7800809f8000919f80004808de007d
:10bf800001002000610060000004e00006003200b3
:10bf900060d82000b12c2c00c21f0200000000005d
:10bfa00010c0b300004f7800809f8000919f8000f8
:10bfb0004b09dd004500de0000007100c508de0011
:10bfc000610060000004e0000400320060d820003e
:10bfd000c12e2c00c21f020000000000809f8000c4
:10bfe000919f8000c109dd004f00de0000807100dc
:10bff000cf08de00610060000004e00004003200b1
:10c0000060d82000d12f2c00c21f020000000000c9
:10c01000809f8000919f80004208de000100200088
:10c02000610060000004e0000400320060d82000dd
:10c03000e1302c00c21f02000000000014002000ac
:10c0400014279800020037008002eb0015279800a3
:10c050001e2090004f05be004f04be000080fa0075
:10c06000000006000a00fa0040479800019f800087
:10c070000004200000807000009f8800119f800055
:10c08000f07f2f0000806000109f880020df2000dc
:10c09000104078000080fb00e0ab8800e0ab80003f
:10c0a0000000e00020013200e1ab8000f00720003a
:10c0b000808f500015003c004e4090000004e000ce
:10c0c0000400320029010700e0ab8000f0ab8800db
:10c0d000f200370021df200010c0b3008c410200c5
:10c0e000000000000004e000040032001f0107000f
:10c0f000e0ab8000f0ab8800e8003700613e210033
:10c1000010c0b30080487800e40037001000200021
:10c110001007980040df2000104078000080fb00ee
:10c12000c800dd0050df2000104078000080fb00d8
:10c13000008f4000e0ab80006101b900a0f72f0044
:10c14000f1ff2f0002014000838148003207980070
:10c1500043079800a0062000010020003e01900047
:10c16000ce019000800f5100818f5900b7003e0032
:10c170003e009000ce009000006001006a00370091
:10c180006f00370071003700b000370075003700ce
:10c190007b00370080003700ac003700810037009b
:10c1a000aa003700a900370081003700830037005c
:10c1b0008500370087003700890037008b00370083
:10c1c0008d003700a100370091003700960037003e
:10c1d0009e0037009d0037009c0037009b00370011
:10c1e0009a00370099003700980037009700370011
:10c1f0009600370095003700940037009300370011
:10c200009200370091003700900037008f00370010
:10c210008e0037008d0037008c0037008b00370010
:10c220008a00370089003700880037008700370010
:10c230008600370085003700840037008300370010
:10c240008200370081003700800037007f00370010
:10c250007e0037007d0037007c0037007b00370010
:10c260007a00370079003700780037007700370010
:10c270007600370075003700740037007300370010
:10c280007200370071003700700037006f00370010
:10c290006e0037006d0037006c0037006b00370010
:10c2a0006a00370069003700680037006700370010
:10c2b0006600370065003700640037006300370010
:10c2c0006200370061003700600037005f00370010
:10c2d0005e0037005d0037005c0037005b00370010
:10c2e0005a00370059003700580037005700370010
:10c2f0005600370055003700540037005300370010
:10c300005200370051003700500037004f0037000f
:10c310004e0037004d0037004c0037004b0037000f
:10c320004a0037004600370030df20001040780018
:10c330000080fb000080e8001007980043003700f1
:10c3400080002000100798004000370030df2000f8
:10c35000104078000080fb000000400010079800ab
:10c360003a00370030df2000104078000080fb00ea
:10c370006600b9000080e80010079800330037001d
:10c3800030df2000104078000080fb000080e800d3
:10c39000100798002d00370090002000100798002b
:10c3a0002a003700c000200010079800270037003f
:10c3b00030002000100798002400370050002000b3
:10c3c0001007980021003700300020001007980067
:10c3d0001e00370050002000100798001b00370097
:10c3e000500020001007980018003700300020008f
:10c3f000100798001500370030df2000104078004b
:10c400000080fb000080e800100798000f00370054
:10c4100030df2000104078000080fb000080e80042
:10c42000100798000900370030df20001040780026
:10c430000080fb000080e800100798000300370030
:10c440009e00780064804000100798004e409000e5
:10c450000004e0000400320087000700e0ab800029
:10c46000f0ab88000d0037001e00900021df200097
:10c470008c410200000000000004e00004003200d3
:10c480007d000700e0ab8000f0ab880003003700c0
:10c49000613e210010c0b30080487800603e21005a
:10c4a000104078000004e0000e003200c1eb2000d4
:10c4b00000c0eb0080487800603e2100904078008a
:10c4c000d0eb200001487800c1eb200020002000c4
:10c4d000be4102000000000080407800e0eb200038
:10c4e000014878000000eb00e0ab88000000eb00a2
:10c4f00010079800070037001e01900021df200080
:10c500000040eb0000f178001e0090000000e80001
:10c51000100798009e009000700c2000808f500043
:10c52000f5ff34000500370050ea80000000e0000d
:10c53000020034001c7a020001000000019f80000c
:10c54000e0ff2f0000806000009f8800019f8000b6
:10c55000f0fb2f0000806000009f88004e1a020050
:10c56000010000000080fa00000006000400fa004c
:10c5700021df20000040eb00804878006000b80018
:10c58000d0228900e1228900e1ab8000e002200096
:10c59000808f50000c003a000000eb00000f780084
:10c5a000050037001e01780061f820000040eb0014
:10c5b00000f178001e0fe800700c20009e0f1000a4
:10c5c000f8ff34000b0037000000eb00000f78008c
:10c5d000050037001e017800c1eb20000040eb0091
:10c5e00000f178001e0fe800700c20009e0f100074
:10c5f000f8ff3400603e21008040eb0001487800e5
:10c60000e0ab80008040eb00314798000000e00084
:10c610000200350012c0b30032479800e1ab800041
:10c620000040eb0020479800e0032000808f50007e
:10c6300002003c0011c0b300214798003e41900029
:10c64000ae409000014061000004e00007003200ad
:10c65000e0ab800080004000e0312c000080400012
:10c66000100078000000010001003700c40007003e
:10c670000080fa00000006000600fa0021df20001a
:10c680000040eb00804878006000b800d0228900ac
:10c69000e12289000000eb00000f78000500370060
:10c6a0001e017800c1eb20000040eb0000f1780093
:10c6b0001e0fe800700c20009e0f1000f8ff3400e1
:10c6c0000000eb00000f7800050037001e01780025
:10c6d00061f820000040eb0000f178001e0fe80038
:10c6e000700c20009e0f1000f8ff3400613e210006
:10c6f0000040eb0080487800e0ab80006101b900a9
:10c70000a0f72f00f1ff2f000201400083814800b5
:10c710001207980023079800a006200001002000bf
:10c720001e019000ae019000800f5100818f5900d2
:10c7300090003e001e009000ae00900000600100de
:10c740006a0037006b0037006c0037008900370043
:10c750006c0037006d0037006e0037008500370031
:10c760006e00370083003700820037006d0037000d
:10c770006e0037006f00370070003700710037001f
:10c7800072003700730037007a00370073003700fb
:10c7900074003700770037007600370075003700e7
:10c7a00074003700730037007200370071003700e3
:10c7b000700037006f0037006e0037006d003700e3
:10c7c0006c0037006b0037006a00370069003700e3
:10c7d00068003700670037006600370065003700e3
:10c7e00064003700630037006200370061003700e3
:10c7f000600037005f0037005e0037005d003700e3
:10c800005c0037005b0037005a00370059003700e2
:10c8100058003700570037005600370055003700e2
:10c8200054003700530037005200370051003700e2
:10c83000500037004f0037004e0037004d003700e2
:10c840004c0037004b0037004a00370049003700e2
:10c8500048003700470037004600370045003700e2
:10c8600044003700430037004200370041003700e2
:10c87000400037003f0037003e0037003d003700e2
:10c880003c0037003b0037003a00370039003700e2
:10c8900038003700370037003600370035003700e2
:10c8a00034003700330037003200370031003700e2
:10c8b000300037002f0037002e0037002d003700e2
:10c8c0002c0037002b0037002a00370029003700e2
:10c8d00028003700270037002600370025003700e2
:10c8e000240037002300370020003700e20907004a
:10c8f00021003700fd0907001f003700410a07002b
:10c900001d003700830a07001b003700b50a070027
:10c9100019003700d60a070017003700ee0a070093
:10c9200015003700210b070013003700650b0700c7
:10c9300011003700b80b07000f003700780c070014
:10c940000d003700ac0d07000b0037007a10070010
:10c9500009003700d610070007003700b61107009e
:10c96000050037005512070003003700601207006a
:10c9700001003700020007000080fa0000000600f6
:10c980000000fa00613e210020c0b300804878001a
:10c990000080fa00000006000000fa00881f7800fe
:10c9a000f0232c004c1f02000000000080407800a3
:10c9b000d0eb200001487800b0232c004c1f02006f
:10c9c0000000000080407800e0eb20000148780083
:10c9d00040012000e83e0200000000008040780096
:10c9e00000c0eb0080c06000f0eb20000148780040
:10c9f00008ec200040002000fe3e02000000000085
:10ca00005d19070008017800da50020000000000fc
:10ca100080c0b300a8440200000000004f0478006a
:10ca20000080fa00000006001000fa0068004700cd
:10ca300001022000543f020000000000680047008f
:10ca400007000900305f78008e00b1008000b1005f
:10ca50009e407800d0eb2000014878009e40900076
:10ca6000e0eb200001487800ae409000f0eb2000a1
:10ca700001487800be40900000ec2000014878009a
:10ca8000ce40900010ec200001487800de4090007d
:10ca900020ec200001487800ee40900030ec2000af
:10caa00001487800fe40900040ec200001487800ea
:10cab00090c0b300a844020000000000109f800056
:10cac0004d00de00610060000004e0000100320063
:10cad000871507000080fa00000006000000fa0039
:10cae00010c0b300a84402000000000086b302009a
:10caf000000000000080fa00000006000000fa00bc
:10cb00007c4402000000000010c0b300a8440200f2
:10cb1000000000000080fa00000006000000fa009b
:10cb2000881f7800d8eb2000c0002000fe3e0200e5
:10cb30000000000008017800da5002000000000048
:10cb400050c0b300a844020000000000109f800005
:10cb50004d00de00610060000004e00001003200d2
:10cb6000271507004f0478000080fa000000060037
:10cb70001000fa00809f8000919f8000022020001a
:10cb80000301200000027800810278000200780092
:10cb90008300780000016200018062006102b80039
:10cba00064079800750798006e009000fe009000e2
:10cbb000c000dd00000020006007980071079800a9
:10cbc0006e009000fe0090006112b80064079800ab
:10cbd000750798006e019000fe0190000200700041
:10cbe00083807000e00f5000e08f58002500320075
:10cbf00040162000fe3e020000000000008fbe0034
:10cc00000080eb008080eb00be0f1000ae8f18009c
:10cc100004003a006000b8004007980051079800ef
:10cc20000f00370040162000163f020000000000f1
:10cc30003e0f020000000000247e270035dd2200a8
:10cc4000b6432900b70124003410020000000000a0
:10cc5000a20e020000000000400798005107980053
:10cc600020162000e83e020000000000cf80de0019
:10cc70006e0c0200000000002007980031079800a9
:10cc80002400370080122000fe3e02000000000059
:10cc9000008fbe000080eb008080eb00be0f100014
:10cca000ae8f180004003a006000b80040079800fa
:10ccb000510798000f00370080122000163f020035
:10ccc000000000003e0f020000000000247e27004c
:10ccd00035dd2200b6432900b701240034100200dc
:10cce00000000000a20e02000000000040079800b3
:10ccf0005107980020122000e83e020000000000ca
:10cd0000cf80de006e0c02000000000020079800bb
:10cd100031079800d2eb20004e009000de0090001a
:10cd2000da50020000000000809f8000919f800088
:10cd3000c709dd004900de0000807100c908de007f
:10cd4000610060000004e0000e0032002e00900040
:10cd5000be0090003e0f020000000000e496260096
:10cd600055432200e61e2000d70224001e110200b7
:10cd700000000000a20e0200000000002007980042
:10cd800031079800921d2a00c30d24002e00900048
:10cd9000be009000800d02000000000020079800f7
:10cda0003107980012ec20002e009000be00900089
:10cdb000da5002000000000090c0b300a844020056
:10cdc000000000000080fa00000006000400fa00e5
:10cdd00080132000163f020000000000008fbe00fc
:10cde000d1eb2000d0c1b3008048780002002000c1
:10cdf000030a24001e00be003010020000000000e4
:10ce00000000e0000100350003003700d1eb2000f6
:10ce100040cbb30080487800020020004323240068
:10ce20001e00be00f80e0200000000000000e0003e
:10ce300001003c0003003700d1eb2000a0c0b3008c
:10ce400080487800c0142000163f02000000000057
:10ce5000008fbe00e1eb2000d0c1b3008048780015
:10ce600002002000030a24001e00be003010020051
:10ce7000000000000000e000010035000300370062
:10ce8000e1eb200040cbb300804878000200200096
:10ce9000432324001e00be00f80e02000000000024
:10cea0000000e00001003c0003003700e1eb20003f
:10ceb000a0c0b30080487800f1eb20000040eb00f8
:10cec0008048780040c0b300a84402000000000081
:10ced0000080fa00000006000800fa000e0078004a
:10cee000c8ff0200010000002e4090008040780042
:10cef000d0eb2000014878001e4090008040780070
:10cf0000e0eb2000014878001e4078008040780067
:10cf1000f0eb2000014878003e409000804078000f
:10cf200000ec2000014878004e40900080407800de
:10cf300010ec2000014878005e40900080407800ae
:10cf400020ec2000014878006e409000804078007e
:10cf500030ec20000148780080c0b300a8440200f3
:10cf600000000000109f80004d00de0061006000a6
:10cf70000004e000010032001c1107000080fa00ec
:10cf8000000006001800fa00881f7800200020002a
:10cf900050079800613e21000040eb008048780077
:10cfa000809f8000919f80001200200003202000bd
:10cfb0000002780081027800020078008300780087
:10cfc00000016200018062006102b80064079800fd
:10cfd000750798006e009000fe009000c000dd0014
:10cfe0000000200060079800710798006e00900014
:10cff000fe0090006112b800640798007507980061
:10d000006e019000fe0190000200700083807000ad
:10d01000e00f5000e08f5800440032005e009000a6
:10d0200080007800c0eb20008080400010002000cd
:10d03000f6500200000000005e0090000080e80052
:10d0400050079800809f8000919f80004908de0073
:10d0500001002000610060000004e00015003200c3
:10d060005e00900080007800c0eb200080804000cf
:10d0700080382100f6500200000000005e009000a1
:10d080000080e800500798005e0090008000780063
:10d09000c0eb20008080400080c12f00f6500200cd
:10d0a000000000005e0090000080e800500798003b
:10d0b000140037005e00900080007800c0eb200074
:10d0c00080804000c0da2000f6500200000000001e
:10d0d0005e0090000080e800500798005e0090001d
:10d0e00080007800c0eb200080804000c0e02f006e
:10d0f000f6500200000000005e0090000080e80092
:10d10000500798005e00900080007800c0eb20007f
:10d1100080804000a0002000f650020000000000c7
:10d120005e0090000080e80050079800809f80001b
:10d13000919f8000ce09dd004200de00008071007a
:10d14000c208de00610060000004e000460032001a
:10d150005e00900080007800c0eb200080804000de
:10d1600020002000f6500200000000005e00900049
:10d170000080e8005007980020122000e83e0200de
:10d1800000000000cf80de006e0c020000000000f6
:10d1900020079800310798002e009000be009000f4
:10d1a0003e0f020000000000247e270035dd220033
:10d1b000b6432900b701240034100200000000002b
:10d1c0006022b80006002000070024007c0f020047
:10d1d0000000000018120200000000001007980074
:10d1e0005e00900080007800c0eb2000808040004e
:10d1f0001e009000f6500200000000005e0090004b
:10d200000080e8005007980080122000163f0200be
:10d21000000000002e019000be019000e80d020009
:10d220000000000002002500337c2400800d020075
:10d2300000000000fc0e0200000000004007980003
:10d240005e00900080007800c0eb200080804000ed
:10d250004e009000f6500200000000005e009000ba
:10d260000080e80050079800809f8000919f800018
:10d2700002202000030120000002780081027800d3
:10d2800002007800830078000001620001806200e3
:10d290006102b800040f9800150f98000e08900066
:10d2a0009e089000c000dd0000002000000f9800e4
:10d2b000110f98000e0890009e0890006112b800af
:10d2c000040f9800150f98000e0990009e09900019
:10d2d0000200700083807000e00f5000e08f580063
:10d2e000500032005e00900080007800c0eb20000b
:10d2f0008080400030002000f65002000000000056
:10d300005e0090000080e8005007980000162000a2
:10d31000e83e020000000000cf80de006e0c02003c
:10d32000000000003e0f020000000000e49626000e
:10d3300055432200e61e2000d702240034100200cc
:10d3400000000000a20e020000000000200798006c
:10d35000310798002e009000be0090003e0f0200a2
:10d3600000000000247e270035dd2200b64329009e
:10d37000b701240034100200000000006022b80051
:10d3800006002000070024007c0f020000000000bf
:10d390001812020000000000100798005e009000c4
:10d3a00080007800c0eb2000808040001e009000cc
:10d3b000f6500200000000005e0090000080e800cf
:10d3c0005007980040162000163f020000000000a1
:10d3d0002e019000be019000e80d02000000000048
:10d3e00002002500337c2400800d020000000000b4
:10d3f000fc0e020000000000400798005e00900054
:10d4000080007800c0eb2000808040004e0090003b
:10d41000f6500200000000005e0090000080e8006e
:10d4200050079800809f8000919f80004a08de008e
:10d4300001002000610060000004e00050003200a4
:10d440005e00900080007800c0eb200080804000eb
:10d4500030002000f6500200000000005e00900046
:10d460000080e80050079800002d2000e83e0200f0
:10d4700000000000cf80de006e0c02000000000003
:10d480003e0f020000000000e496260055432200f3
:10d49000e61e2000d7022400341002000000000025
:10d4a000a20e02000000000020079800310798003b
:10d4b0002e009000be0090003e0f02000000000011
:10d4c000247e270035dd2200b6432900b701240061
:10d4d00034100200000000006022b80006002000a6
:10d4e000070024007c0f0200000000001812020058
:10d4f00000000000100798005e0090008000780097
:10d50000c0eb2000808040001e009000f65002001a
:10d51000000000005e0090000080e80050079800c6
:10d52000802c2000163f0200000000002e01900019
:10d53000be019000e80d020000000000020025007e
:10d54000337c2400800d020000000000fc0e02006d
:10d5500000000000400798005e0090008000780006
:10d56000c0eb2000808040004e009000f65002008a
:10d57000000000005e0090000080e8005007980066
:10d58000809f8000919f8000024020008300200047
:10d5900000027800810278000200780083007800a1
:10d5a00000016200018062006102b800240f98004f
:10d5b000350f98002e089000be089000c000dd00d6
:10d5c00000002000200f9800310f98002e089000d6
:10d5d000be0890006112b800240f9800350f980023
:10d5e0002e099000be099000020070008380700038
:10d5f000e00f5000e08f5800bb0032000040eb000d
:10d60000004f780000192000fe3e020000000000dc
:10d610004308de0001002000610060000004e0001b
:10d620003a0032001e04e00038003a005e0090002c
:10d6300080007800c0eb2000808040004000200087
:10d64000f6500200000000005e0090000080e8003c
:10d65000500798005e00900080007800c0eb20002a
:10d660008080400000642000f650020000000000ae
:10d670005e0090000080e800500798005e00900077
:10d6800080007800c0eb20008080400080572000a0
:10d69000f6500200000000005e0090000080e800ec
:10d6a0005007980080192000e83e020000000000aa
:10d6b000400798004e0090004800dd0040079800a9
:10d6c000a0192000e83e0200000000008000780061
:10d6d0004e00900001004000400798005e0090005e
:10d6e00080007800c0eb2000808040004e00900059
:10d6f000f6500200000000005e0090000080e8008c
:10d700005007980010c0b300004f7800001a2000a6
:10d71000fe3e0200000000004308de000100200081
:10d72000610060000004e0003a0032001e04e000e6
:10d7300038003a005e00900080007800c0eb2000c6
:10d740008080400040002000f650020000000000f1
:10d750005e0090000080e800500798005e00900096
:10d7600080007800c0eb2000808040000064200032
:10d77000f6500200000000005e0090000080e8000b
:10d78000500798005e00900080007800c0eb2000f9
:10d790008080400080572000f6500200000000000a
:10d7a0005e0090000080e80050079800801a20007a
:10d7b000e83e020000000000400798004e00900084
:10d7c0004800dd0040079800a01a2000e83e020053
:10d7d00000000000800078004e0090000100400032
:10d7e000400798005e00900080007800c0eb2000a9
:10d7f000808040004e009000f650020000000000c3
:10d800005e0090000080e8005007980010c0b30050
:10d81000004f7800809f8000919f8000c609dd0046
:10d820004a00de0000807100ca08de00610060006e
:10d830000004e0002c0032001e04e0002a003a0040
:10d840005e00900080007800c0eb200080804000e7
:10d8500040002000f6500200000000005e00900032
:10d860000080e800500798005e009000800078007b
:10d87000c0eb20008080400000642000f6500200d1
:10d88000000000005e0090000080e8005007980053
:10d890005e00900080007800c0eb20008080400097
:10d8a00080572000f6500200000000005e0090004b
:10d8b0000080e800500798005e009000800078002b
:10d8c000c0eb200080804000e0012000f650020004
:10d8d000000000005e0090000080e8005007980003
:10d8e00010c0b300004f7800809f8000919f80009f
:10d8f0004808de0001002000610060000004e00034
:10d90000480032005e00900080007800c0eb2000ec
:10d910008080400000012000f6500200000000005e
:10d920005e0090000080e800500798005e009000c4
:10d9300080007800c0eb2000808040000064200060
:10d94000f6500200000000005e0090000080e80039
:10d95000500798005e00900080007800c0eb200027
:10d960008080400080572000f65002000000000038
:10d970005e0090000080e800500798005e00900074
:10d9800080007800c0eb200080804000e001200093
:10d99000f6500200000000005e0090000080e800e9
:10d9a000500798005e00900080007800c0eb2000d7
:10d9b0008080400000fa2000f650020000000000c5
:10d9c0005e0090000080e800500798005e00900024
:10d9d00080007800c0eb200080804000c0e02f0075
:10d9e000f6500200000000005e0090000080e80099
:10d9f000500798005e00900080007800c0eb200087
:10da000080804000a0002000f650020000000000ce
:10da10005e0090000080e8005007980010c0b3003e
:10da2000004f7800809f8000919f80004b0add00ae
:10da30004500de0000007200c508de0061006000e5
:10da40000004e000280032005e00900080007800b2
:10da5000c0eb20008080400050002000f650020003
:10da6000000000005e0090000080e8005007980071
:10da70005e00900080007800c0eb200080804000b5
:10da800040382000f6500200000000005e009000c8
:10da90000080e800500798005e0090008000780049
:10daa000c0eb20008080400040382000f65002008b
:10dab000000000005e0090000080e8005007980021
:10dac0005e00900080007800c0eb20008080400065
:10dad000a0002000f6500200000000005e00900050
:10dae0000080e80050079800809f8000919f800090
:10daf000c10add004f00de0000807200cf08de00aa
:10db0000610060000004e000280032005e00900028
:10db100080007800c0eb2000808040006000200082
:10db2000f6500200000000005e0090000080e80057
:10db3000500798005e00900080007800c0eb200045
:10db40008080400040062000f650020000000000e7
:10db50005e0090000080e800500798005e00900092
:10db600080007800c0eb200080804000400620004c
:10db7000f6500200000000005e0090000080e80007
:10db8000500798005e00900080007800c0eb2000f5
:10db90008080400020032000f650020000000000ba
:10dba0005e0090000080e80050079800809f800091
:10dbb000919f80004909dd004700de0000007100f0
:10dbc000c708de00610060000004e0000a003200c7
:10dbd0005e00900080007800c0eb20008080400054
:10dbe00070002000f6500200000000005e0090006f
:10dbf0000080e80050079800809f8000919f80007f
:10dc0000ca09dd004600de0000807100c608de00a3
:10dc1000610060000004e000140032005e0090002b
:10dc200080007800c0eb2000808040008000200051
:10dc3000f6500200000000005e0090000080e80046
:10dc4000500798005e00900080007800c0eb200034
:10dc50008080400010002000f6500200000000000c
:10dc60005e0090000080e80050079800809f8000d0
:10dc7000919f8000440add004c00de00000072002d
:10dc8000cc08de00610060000004e00017003200f4
:10dc90005e00900080007800c0eb20008080400093
:10dca00090002000f6500200000000005e0090008e
:10dcb0000080e800500798005e0090008000780027
:10dcc000c0eb20000084400000152000d23e02007e
:10dcd0000000000088007800f650020000000000fc
:10dce0005e0090000080e80050079800809f800050
:10dcf000919f8000c30add004d00de0000807200ad
:10dd0000cd08de00610060000004e0001400320075
:10dd10005e00900080007800c0eb20008080400012
:10dd2000a0002000f6500200000000005e009000fd
:10dd30000080e800500798005e00900080007800a6
:10dd4000c0eb20008080400010002000f650020050
:10dd5000000000005e0090000080e800500798007e
:10dd6000809f8000919f80004208de00010020001b
:10dd7000610060000004e000460032005e00900098
:10dd800080007800c0eb200080804000b0002000c0
:10dd9000f6500200000000005e0090000080e800e5
:10dda000500798005e00900080007800c0eb2000d3
:10ddb0008080400040382000f65002000000000043
:10ddc0005e0090000080e800500798005e00900020
:10ddd00080007800c0eb20008080400040382000a8
:10dde000f6500200000000005e0090000080e80095
:10ddf000500798005e00900080007800c0eb200083
:10de00008080400040062000f65002000000000024
:10de10005e0090000080e800500798005e009000cf
:10de200080007800c0eb200080804000406a200025
:10de3000f6500200000000005e0090000080e80044
:10de4000500798005e00900080007800c0eb200032
:10de500080804000406a2000f65002000000000070
:10de60005e0090000080e800500798005e0090007f
:10de700080007800c0eb200080804000400120003e
:10de8000f6500200000000005e0090000080e800f4
:10de900050079800809f8000919f80004809dd0016
:10dea0004800de0000007100c808de00610060006c
:10deb0000004e000210032005e0090008000780045
:10dec000c0eb200080804000c0002000f65002001f
:10ded000000000005e0090000080e80050079800fd
:10dee000709f80004c00de00610060000004e000d4
:10def000080032005e00900080007800c0eb200037
:10df00008080400020002000f65002000000000049
:10df1000070037005e00900080007800c0eb200012
:10df20008080400010002000f65002000000000039
:10df30005e0090000080e80050079800809f8000fd
:10df4000919f80004508de00010020006100600014
:10df50000004e0000a0032005e00900080007800bb
:10df6000c0eb200080804000d0002000f65002006e
:10df7000000000005e0090000080e800500798005c
:10df8000809f8000919f80004708de0001002000f4
:10df9000610060000004e0000a0032005e009000b2
:10dfa00080007800c0eb200080804000e00020006e
:10dfb000f6500200000000005e0090000080e800c3
:10dfc00050079800809f8000919f80004608de00e7
:10dfd00001002000610060000004e0000a0032003f
:10dfe0005e00900080007800c0eb20008080400040
:10dff000f0002000f6500200000000005e009000db
:10e000000080e800500798005e00900080007800d3
:10e01000c0eb2000808040000000eb00f6500200c2
:10e02000000000005e0090000080e80050079800ab
:10e030005e0090000080e90022002000110009002d
:10e040000200d80080407800d0eb20000148780022
:10e050005e009000a8440200000000004f04780019
:10e060000080fa00000006000600fa005ef80200d8
:10e0700001000000100798002107980020002000f0
:10e08000000f78001e0178001e009000ae00900086
:10e09000c2130700000f7800200020009e0f100020
:10e0a00005003a00e1eb20000000eb00f650020012
:10e0b000000000001e8fe8001e80e9002200200002
:10e0c000110009000200d80080407800d0eb200049
:10e0d000014878001e007800a844020000000000fb
:10e0e000109f80004d00de00610060000004e00031
:10e0f00001003200730d0700613e21000040eb007b
:10e10000804878000080fa00000006000600fa004f
:10e110005ef8020001000000100798002107980037
:10e1200020002000000f78001e0178001e009000e3
:10e13000ae009000b1140700000f7800200020000e
:10e140009e0f100005003a00e1eb20000000eb00fc
:10e15000f6500200000000001e8fe8001e80e9005b
:10e1600022002000110009000200d8008040780041
:10e17000d0eb2000014878001e007800a84402007f
:10e1800000000000109f80004d00de006100600074
:10e190000004e000010032004a0d0700613e21004a
:10e1a0000040eb00804878000080fa000000060084
:10e1b0000800fa00881f78000000eb0010079800a4
:10e1c000070037001e01900061f820000040eb00be
:10e1d00000f178001e0090000000e8001007980091
:10e1e0009e009000700c2000808f5000f5ff3400de
:10e1f000009f8000f1f72f0001006000009f880061
:10e20000409f8000300798003e009000e30f5000d0
:10e21000a30032003e009000e30f500007003c00d6
:10e220003e009000e10f5000320032003e009000ae
:10e23000e20f500080003200720137003e00900073
:10e24000e70f5000b00032003e009000e80f500091
:10e25000040032003e009000e40f5000c400320081
:10e2600068013700209f80004400de0061006000ec
:10e270000004e0000c003200709b80000000e80009
:10e28000709b8800709b8000e30f500002003400f8
:10e290000000eb00709b8800209f8000f1fe2f00a3
:10e2a00001006000209f8800f0022000e0ab8800a1
:10e2b000d1eb200080c0b30080487800e2eb200062
:10e2c00000e8800011e88000da5002000000000041
:10e2d00022ec2000e0e78000f1e78000da50020045
:10e2e00000000000a0c0b300a8440200000000002d
:10e2f00047013700209f80004400de00610060007d
:10e300000004e0000c003200709b80000000e80078
:10e31000709b8800709b8000e30f50000200340067
:10e320000000eb00709b8800209f8000f1fe2f0012
:10e3300001006000209f8800f0022000e0ab880010
:10e34000d1eb200040c0b30080487800204020007e
:10e35000e83e020000000000000f780001ec200001
:10e360001e007800f650020000000000004020006f
:10e37000d23e020000000000000f780021ec2000d7
:10e380001e007800f6500200000000000000eb00c4
:10e39000100798001e0090000000400080007800e8
:10e3a0004040200000804000e83e020000000000e5
:10e3b000000f78001e00e0000b0034001e009000eb
:10e3c000000040008000780040ec20008080400089
:10e3d0001e007800f6500200000000001e009000b1
:10e3e0000000e800100798001e009000ed0f50009c
:10e3f00002003c001e00e000e6ff3c001e00900012
:10e400000080e80010079800e1eb20001e0090005b
:10e41000f6500200000000001e0090000080e8009e
:10e42000100798001e00900000004000a844020061
:10e4300000000000f6003700209f80004400de004e
:10e44000610060000004e0000c003200709b80005e
:10e450000000e800709b8800709b8000e30f500074
:10e46000020034000000eb00709b8800209f8000b9
:10e47000f1fe2f0001006000209f8800f0022000c4
:10e48000e0ab8800d1eb200020c0b30080487800ca
:10e4900020c0b300a844020000000000dc003700e8
:10e4a000209f80004400de00610060000004e00066
:10e4b0000c003200709b80000000e800709b880018
:10e4c000709b8000e30f5000020034000000eb005e
:10e4d000709b8800209f8000f1fe2f0001006000eb
:10e4e000209f8800f0022000e0ab8800d1eb2000e4
:10e4f00030c0b3008048780020c0b300a8440200b8
:10e5000000000000c2003700209f80004400de00b1
:10e51000610060000004e0000c003200709b80008d
:10e520000000e800709b8800709b8000e30f5000a3
:10e53000020034000000eb00709b8800209f8000e8
:10e54000f1fe2f0001006000209f8800f0022000f3
:10e55000e0ab8800d1eb200070c0b30080487800a9
:10e5600020c0b300a844020000000000a80037004b
:10e57000209f80004400de00610060000004e00095
:10e580000c003200709b80000000e800709b880047
:10e59000709b8000e30f5000020034000000eb008d
:10e5a000709b8800209f8000f1fe2f00010060001a
:10e5b000209f8800709b8000a13721000000400050
:10e5c00001004000100078008040780080f82000b2
:10e5d000014878000000eb00100798004000200080
:10e5e0002007980011003700ae019000719b800059
:10e5f0001e019000800c20000088b90082004000bd
:10e60000e0042100614078008040780060f820003c
:10e61000817178002e0090000000e800200798002b
:10e620001e0090000000e800100798009e00900077
:10e63000700c2000808f50000c003c001e049000e5
:10e64000709b800080007800800c20000088b9005a
:10e6500080007800e004210000804000ce1b020012
:10e6600000000000800f5400dfff39002e009000f2
:10e67000644050008040780090f820000148780005
:10e680002e01900061f820000040eb0000f17800be
:10e690002e009000610060000004e00003003200e2
:10e6a0002e0090000000e800200798002e00900047
:10e6b00022002000110009000200d80080407800ec
:10e6c00070f82000014878002e009000d24402002b
:10e6d000000000002e0090000001e80061f820001a
:10e6e0000040eb0000f17800119f80000000210045
:10e6f00000807000109f8800c0122000409c88009d
:10e70000709b800080007800800c20000088b90099
:10e7100080007800e004210000804000c1392c0016
:10e72000941f0200000000000000e0000200320020
:10e73000c0122000409c8800709b80008000780000
:10e74000800c20000088b90080007800e0042100df
:10e7500000804000f1392c00941f020000000000ee
:10e760000000e00002003200c0122000409c88003f
:10e77000709b800080007800800c20000088b90029
:10e7800080007800e004210000804000213a2c0045
:10e79000941f0200000000000000e00002003200b0
:10e7a000c0122000409c8800709b80008000780090
:10e7b000800c20000088b90080007800e00421006f
:10e7c00000804000513a2c00941f0200000000001d
:10e7d0000000e00002003200e0012000409c8800c0
:10e7e000419c8000209e800000804000409c88006a
:10e7f000019f80000000240000807000009f8800be
:10e8000003003700613e210030c0b300804878002b
:10e810004f0478000080fa00000006000600fa00ad
:10e820005ef8020001000000100798002107980020
:10e8300020002000000f78001e0178001e009000cc
:10e84000ae00900030140700000f78002000200078
:10e850009e0f100005003a00e1eb20000000eb00e5
:10e86000f6500200000000001e8fe8001e80e90044
:10e8700022002000110009000200d800804078002a
:10e88000d0eb2000014878001e007800a844020068
:10e8900000000000109f80004d00de00610060005d
:10e8a0000004e00001003200860b0700613e2100f9
:10e8b0000040eb00804878000080fa00000006006d
:10e8c0000600fa005ef80200010000001007980040
:10e8d0002107980020002000000f78001e0178001a
:10e8e0001e009000ae00900059150700000f780040
:10e8f000200020009e0f100005003a00e1eb2000f0
:10e900000000eb00f6500200000000001e8fe8003f
:10e910001e80e90022002000110009000200d8003a
:10e9200080407800d0eb2000014878001e0078007d
:10e93000a844020000000000109f80004d00de008f
:10e94000610060000004e000010032005d0b070080
:10e95000613e21000040eb00804878000080fa0012
:10e96000000006000600fa005ef802000100000048
:10e97000100798002107980020002000000f780061
:10e980001e0178001e009000ae0090007116070076
:10e99000000f7800200020009e0f10000f003a00aa
:10e9a00020002000000f78001e0178001e0090005b
:10e9b000ae0090004b190700000f780020002000e7
:10e9c0009e0f100005003a00e1eb20000000eb0074
:10e9d000f6500200000000001e8fe8001e80e900d3
:10e9e00022002000110009000200d80080407800b9
:10e9f000d0eb2000014878001e007800a8440200f7
:10ea000000000000109f80004d00de0061006000eb
:10ea10000004e000010032002a0b0700613e2100e3
:10ea20000040eb00804878000080fa0000000600fb
:10ea30000600fa005ef802000100000010079800ce
:10ea40002107980020002000000f78001e017800a8
:10ea50001e009000ae0090001f170700000f780006
:10ea6000200020009e0f100005003a00e1eb20007e
:10ea70000000eb00f6500200000000001e8fe800ce
:10ea80001e80e90022002000110009000200d800c9
:10ea900080407800d0eb2000014878001e0078000c
:10eaa000a844020000000000109f80004d00de001e
:10eab000610060000004e00001003200010b07006b
:10eac000613e21000040eb00804878000080fa00a1
:10ead000000006000000fa00009f80000030a00047
:10eae000009f880010c0b300a8440200000000008e
:10eaf0000080fa00000006000600fa005ef802003e
:10eb00000100000010079800210798002000200055
:10eb1000000f78001e0178001e009000ae009000eb
:10eb2000f6160700000f7800200020009e0f10004e
:10eb300005003a00e1eb20000000eb00f650020077
:10eb4000000000001e8fe8001e80e9002200200067
:10eb5000110009000200d80080407800d0eb2000ae
:10eb6000014878001e007800a84402000000000060
:10eb7000109f80004d00de00610060000004e00096
:10eb800001003200cf0a0700613e21000040eb0087
:10eb9000804878000080fa00000006000000fa00bb
:10eba000401f2000109d880010c0b300a844020040
:10ebb000000000000080fa00000006000000fa00db
:10ebc000881f7800f0232c004c1f0200000000007a
:10ebd00080407800d0eb200001487800b0232c0062
:10ebe0004c1f02000000000080407800e0eb200095
:10ebf00001487800c0c4b30080407800f0eb2000ea
:10ec00000148780040012000e83e020000000000ba
:10ec10008040780000c0eb0080c0600000ec200065
:10ec20000148780040012000e83e0200000000009a
:10ec30004880de008040780000c0eb0080c06000ab
:10ec400010ec20000148780028ec20004000200053
:10ec5000fe3e020000000000c71007000801780017
:10ec6000da50020000000000a0c0b300a844020077
:10ec700000000000109f80004d00de006100600079
:10ec80000004e00001003200630d07004f0478002b
:10ec90000080fa00000006000600fa005ef802009c
:10eca00001000000100798002107980020002000b4
:10ecb000000f78001e0178001e009000ae0090004a
:10ecc00088180700000f7800200020009e0f100019
:10ecd00005003a00e1eb20000000eb00f6500200d6
:10ece000000000001e8fe8001e80e90022002000c6
:10ecf000110009000200d80080407800d0eb20000d
:10ed0000014878001e007800a844020000000000be
:10ed1000109f80004d00de00610060000004e000f4
:10ed200001003200670a0700613e21000040eb004d
:10ed3000804878000080fa00000006000600fa0013
:10ed40005ef80200010000001007980021079800fb
:10ed500020002000000f78001e0178001e009000a7
:10ed6000ae00900035190700000f78002000200049
:10ed70009e0f100005003a00e1eb20000000eb00c0
:10ed8000f6500200000000001e8fe8001e80e9001f
:10ed900022002000110009000200d8008040780005
:10eda000d0eb2000014878001e007800a844020043
:10edb00000000000109f80004d00de006100600038
:10edc0000004e000010032003e0a0700613e21001d
:10edd0000040eb00804878000080fa000000060048
:10ede0004e00fa006000b800200798003107980034
:10edf000d0f92f0010079800709f80004d00de00b2
:10ee0000610060000004e000340032000080eb008c
:10ee1000100798006801470040922300d1a020000d
:10ee20000089be000040eb004041980068004700a8
:10ee3000d2022000411f2000a012020001000000a9
:10ee4000e80f50002500340068004700a2032000ae
:10ee50000e0141003301200011002000246d02004a
:10ee600001000000000f780068004700a2032000a6
:10ee70000e014100330120009e007800246d020045
:10ee800001000000000f7800a00320000e004000e9
:10ee90009e1e020000000000a20e02000000000002
:10eea000200798003107980068004700a20320005f
:10eeb0000e014100330120009e007800246d020005
:10eec00001000000000f7800a00320000e004000a9
:10eed0004c1f02000000000010079800d1eb20003a
:10eee00040002000f650020000000000f1eb20007e
:10eef0001e009000f65002000000000012ec2000fe
:10ef00002e009000be009000da50020000000000c9
:10ef100090c0b300a844020000000000613e210040
:10ef20000040eb00804878000080fa0000000600f6
:10ef30000600fa005ef802000100000010079800c9
:10ef40002107980020002000000f78001e017800a3
:10ef50001e009000ae009000e8130700000f78003c
:10ef6000200020009e0f100005003a00e1eb200079
:10ef70000000eb00f6500200000000001e8fe800c9
:10ef80001e80e90022002000110009000200d800c4
:10ef900080407800d0eb2000014878001e00780007
:10efa000a844020000000000109f80004d00de0019
:10efb000610060000004e00001003200c1090700a8
:10efc000613e21000040eb00804878000080fa009c
:10efd000000006000600fa005ef8020001000000d2
:10efe000100798002107980020002000000f7800eb
:10eff0001e0178001e009000ae0090007710070000
:10f00000000f7800200020009e0f100005003a003d
:10f01000e1eb20000000eb00f650020000000000d1
:10f020001e8fe8001e80e900220020001100090068
:10f030000200d80080407800d0eb20000148780022
:10f040001e007800a844020000000000109f80000d
:10f050004d00de00610060000004e00001003200ad
:10f0600098090700613e21000040eb0080487800cd
:10f070000080fa00000006000400fa0030df2000e3
:10f08000104078000080fb00000f78000000eb00cb
:10f09000100798000a0037001e0190001e00900023
:10f0a0008080e80020df2000e140780020df2000a1
:10f0b000017178001e0090000000e8001007980021
:10f0c0001e0090009e0f5000f3ff35001e019000bf
:10f0d00021df20000040eb0000f178001e04020058
:10f0e000010000000080fa00000006000800fa009d
:10f0f00030df2000104078002047980040df2000db
:10f10000104078001047980050df20001040780031
:10f11000004f780060df20001040780030479800f2
:10f1200070df2000104078004047980080df20000a
:10f13000104078005047980090df20001040780081
:10f14000604798000e007800c8030200020000002b
:10f1500080d62100c8ff0200010000000e007800e8
:10f16000c8ff0200010000002e409000804078009f
:10f17000d0eb2000014878001e40900080407800cd
:10f18000e0eb2000014878001e40780080407800c5
:10f19000f0eb2000014878003e409000804078006d
:10f1a00000ec2000014878004e409000804078003c
:10f1b00010ec2000014878005e409000804078000c
:10f1c00020ec2000014878006e40900080407800dc
:10f1d00030ec20000148780080c0b300a844020051
:10f1e00000000000109f80004d00de006100600004
:10f1f0000004e000010032007c0807000080fa00f3
:10f2000000000600ca00fa002e4c020000000000b8
:10f210000004e00037003200829b800040df2000c5
:10f22000104078008081fb00a137210002004100de
:10f2300001004000030878000000eb00000f780098
:10f240000a0037001e0178001e007800e40040002c
:10f2500020df200061407800804078000e80e800c8
:10f2600000004100014878001e0fe80050df200038
:10f27000104078000080fb009e0f5000f1ff3c0022
:10f280009e0078000e80e800808040000040eb0087
:10f2900080487800809b800080007800800c2000ef
:10f2a0000088b90080007800e00421000080400060
:10f2b0008e80e8002620020000000000809b800075
:10f2c0002137210000004000810040001000200094
:10f2d00080087800809b80000000e800809b880008
:10f2e000809b8000e30f5000020034000000eb0020
:10f2f000809b8800613e21000040eb008048780040
:10f3000010c0b300a8440200000000000080fa0012
:10f31000000006000a00fa00d0d521001040780055
:10f320000004e000240032000000eb0040079800d9
:10f330001b0037004e0090006600b9000080e80016
:10f34000300798003e0090008000780020df200009
:10f3500000804000ea50020000000000000f78002a
:10f360003e0090008000780040df200000804000d8
:10f37000c650020000000000100798002107980006
:10f380001e019000ae0190001e007800fe81020078
:10f39000010000004e0090000000e80040079800c7
:10f3a00030df2000104078008080fb004e0090008d
:10f3b000808f5000dfff3c00209f80000010a000e5
:10f3c000209f8800613e21000040eb0080487800cb
:10f3d00010c0b300a8440200000000000080fa0042
:10f3e000000006000400fa0030df20001040780022
:10f3f0000080fb00000f78000000eb001007980071
:10f400000a0037001e0190001e0090008080e80076
:10f4100020df2000e140780020df2000017178002b
:10f420001e0090000000e800100798001e009000e9
:10f430009e0f5000f3ff35001e01900021df2000d9
:10f440000040eb0000f17800d23d02000100000016
:10f45000109f80004d00de00610060000004e000ad
:10f46000010032002b0807000080fa0000000600af
:10f470000000fa0030df200090407800a0d021008a
:10f480000148780040df200090407800b0d0210093
:10f490000148780050df2000ea5002000000000020
:10f4a00080e8880070df2000c650020000000000e5
:10f4b00090e88800a1e88800209f80000030a0002c
:10f4c000209f880010c0b300a84402000000000084
:10f4d0000080fa00000006000000fa0030df200083
:10f4e00090407800a0d021000148780040df200043
:10f4f00090407800b0d021000148780050df200013
:10f5000090407800c0d021000148780060df2000e2
:10f5100090407800d0d021000148780070df2000b2
:10f5200090407800e0d021000148780080df200082
:10f530009040780040d021000148780090df200002
:10f540009040780050d0210001487800a0df2000d2
:10f550009040780060d0210001487800b0df2000a2
:10f560009040780070d0210001487800c0df200072
:10f570009040780080d0210001487800d0df200042
:10f580009040780090d0210001487800209f8000b2
:10f590000030a000209f880010c0b300a8440200e3
:10f5a000000000000080fa00000006000400fa00dd
:10f5b0000000eb00209d8800809f8000919f8000cc
:10f5c0004809dd004800de0000007100c808de00c8
:10f5d000610060000004e0002900320030df2000fc
:10f5e000ea5002000000000010079800709f8000a1
:10f5f0004c00de00610060000004e00010003200fa
:10f600001e009000f40b0700000f7800d1eb2000e3
:10f610001e007800f650020000000000f1eb200010
:10f62000409d8000f65002000000000021ec200008
:10f63000509d8000f6500200000000001c003700c2
:10f640001e009000cb0c0700000f7800d1eb2000cb
:10f650001e007800f650020000000000f1eb2000d0
:10f66000209d8000f65002000000000011ec2000f8
:10f670000000eb00f6500200000000000c00370014
:10f68000d1eb20000000eb00f6500200000000006b
:10f69000f1eb20000000eb00f6500200000000003b
:10f6a00011ec20000000eb00f6500200000000000a
:10f6b00070c0b300a8440200000000000080fa00ff
:10f6c000000006000800fa0030df2000104078003b
:10f6d0000080fb0001002000008fbe001e00be0065
:10f6e000c808dd000080fd00804078000040eb008d
:10f6f000008fbe0040df2000104078000080fb003b
:10f70000010020001e0f40005e9748001e00be0052
:10f71000c808dd000080fd00804078000040eb005c
:10f72000008fbe0050df2000104078000080fb00fa
:10f73000010020001e0f40005e9748001e00be0022
:10f74000c808dd000080fd00804078000040eb002c
:10f75000008fbe0060df2000104078000080fb00ba
:10f76000010020001e0f40005e974800809f80002f
:10f77000919f800000017800810178001e007800d0
:10f780009e00900000016100018061006102b800ec
:10f7900024079800350798002e009000be009000c6
:10f7a000c000dd000000200020079800310798000d
:10f7b0002e009000be0090006112b800240798004f
:10f7c000350798002e019000be01900002007000e5
:10f7d00083807000008fbe00609e8000719e80005c
:10f7e0003e027000ae8270000400be00609e880081
:10f7f000719e8800d2eb20001e00be00da5002008d
:10f800000000000050c0b300a84402000000000047
:10f810000080fa00000006000c00fa005ef802000a
:10f8200001000000300798004107980040002000c8
:10f8300050079800d1eb200010c0b300804878003a
:10f84000e1eb20000000eb00f65002000000000099
:10f85000809f8000919f80004708de00010020000b
:10f86000610060000004e000a500320030df2000ed
:10f87000ea50020000000000000f78000080eb005a
:10f8800090a48800e09e8000f19e80004708de0082
:10f8900001002000610060000004e0001e00320052
:10f8a00082a6800093a680003e009000ce009000cb
:10f8b000020050008380580010079800210798002c
:10f8c0001e009000ae009000e00f5000e08f580046
:10f8d00008003d001e009000ae00900002a823002a
:10f8e000930020000000410081804900100798002b
:10f8f000210798001e019000ae019000f0522700f1
:10f9000001002000800f5100818f590002003c004f
:10f910001e00900090a48800a002200050079800cc
:10f92000d1eb200080c1b30080487800e1eb2000db
:10f9300080002000f65002000000000001ec2000d2
:10f9400090a48000f65002000000000021ec20008e
:10f9500070a38000f65002000000000041ec20007f
:10f9600080a38000f65002000000000062ec20003e
:10f97000a0a38000b1a38000da50020000000000c4
:10f98000a1ec2000c0a38000f6500200000000009f
:10f99000c1ec2000d0a38000f6500200000000005f
:10f9a000e1ec2000e0a38000f6500200000000001f
:10f9b00001ed2000f0a38000f650020000000000de
:10f9c00021ed200000a48000f6500200000000009d
:10f9d00041ed200010a48000f6500200000000005d
:10f9e00061ed200020a48000f6500200000000001d
:10f9f00081ed200030a48000f650020000000000dd
:10fa0000a1ed200040a48000f6500200000000009c
:10fa1000c1ed200050a48000f6500200000000005c
:10fa2000c048210090407800e0ed200001487800b7
:10fa3000d048210090407800f0ed20000148780087
:10fa4000e04821009040780000ee20000148780056
:10fa5000f04821009040780010ee20000148780026
:10fa6000b00481008040780020ee2000014878003a
:10fa700020472100104078008040780030ee2000c0
:10fa80000148780041ee200080a48000f65002007a
:10fa9000000000001e00e00019003400800c20006f
:10faa0009e0f100016003c0060172000e83e020088
:10fab000000000009e0f500007003200b0048100db
:10fac0000000e00004003c009e0078006017200069
:10fad000c43d020000000000629e8000739e800012
:10fae00000002000010820000000710081807100ea
:10faf000609e8800719e8800309e8000d0a888009b
:10fb00005e009000a844020000000000613e210059
:10fb10000040eb00804878000080fa0000000600fa
:10fb20001a00fa0030df2000104078000080fb004f
:10fb30000100200030079800410798003e00900027
:10fb4000ce009000c808dd000080fd0080407800f5
:10fb50000040eb00300798004107980040df20008c
:10fb6000104078000081fb00030020003e00900060
:10fb7000ce009000000041008180490030079800cd
:10fb8000410798003e009000ce009000c808dd00bc
:10fb90000080fd00804078000040eb0030079800b6
:10fba0004107980050df2000104078000081fb00e2
:10fbb000030020003e009000ce00900000004100b5
:10fbc0008180490030079800410798003e0090006e
:10fbd000ce009000c808dd000080fd008040780065
:10fbe0000040eb00300798004107980060df2000dc
:10fbf000104078000081fb00030020003e009000d0
:10fc0000ce0090000000410081804900300798003c
:10fc1000410798005ef802000100000010079800fc
:10fc20002107980020002000000f78003e0090007f
:10fc3000610060000004e000050032001e01780051
:10fc40001e009000ae009000d40c0700000f78005a
:10fc50003e009000ce0090004908de000100200028
:10fc6000610060000004e000050032001e01780021
:10fc70001e009000ae009000580d0700000f7800a5
:10fc80003e009000ce0090004220200003012000a2
:10fc9000000278008102780002007800830078007a
:10fca00000016200018062006102b8005407980000
:10fcb000650798005e009000ee009000c000dd0037
:10fcc0000000200050079800610798005e00900037
:10fcd000ee0090006112b800540798006507980084
:10fce0005e019000ee0190000200700083807000c1
:10fcf000e00f5000e08f5800050032001e01780030
:10fd00001e009000ae009000bc0d0700000f7800b0
:10fd10003e009000ce009000020228004300200028
:10fd200000027800810278000200780083007800e9
:10fd300000016200018062006102b800740798004f
:10fd4000050f98007e0090008e089000c000dd0036
:10fd50000000200070079800010f98007e009000be
:10fd60008e0890006112b80074079800050f980083
:10fd70007e0190008e099000020070008380700068
:10fd8000e00f5000e08f5800050032001e0178009f
:10fd90001e009000ae009000db0e0700000f780000
:10fda0003e009000ce009000024020008300200022
:10fdb0000002780081027800020078008300780059
:10fdc00000016200018062006102b800140f980017
:10fdd000250f98001e089000ae089000c000dd00be
:10fde00000002000100f9800210f98001e089000be
:10fdf000ae0890006112b800140f9800250f98000b
:10fe00001e099000ae09900002007000838070000f
:10fe1000e00f5000e08f5800050032001e0178000e
:10fe20001e009000ae00900009100700000f78003f
:10fe30003e009000ce009000c409dd004c00de00c2
:10fe400000807100cc08de00610060000004e0006a
:10fe5000050032001e0178001e009000ae009000e8
:10fe60003c110700000f78003e009000ce0090008b
:10fe7000490add004700de0000007200c708de000e
:10fe8000610060000004e000050032001e017800ff
:10fe90001e009000ae0090000f120700000f7800c7
:10fea0003e009000ce009000422020000341200040
:10feb0000002780081027800020078008300780058
:10fec00000016200018062006102b800340f9800f6
:10fed000450f98003e089000ce089000c000dd005d
:10fee00000002000300f9800410f98003e0890005d
:10fef000ce0890006112b800340f9800450f9800aa
:10ff00003e099000ce0990000200700083807000ce
:10ff1000e00f5000e08f5800050032001e0178000d
:10ff20001e009000ae009000f4110700000f780052
:10ff30003e009000ce0090004508de000100200049
:10ff4000610060000004e000050032001e0178003e
:10ff50001e009000ae009000e2130700000f780032
:10ff60003e009000ce0090004508de000100200019
:10ff7000610060000004e000050032001e0178000e
:10ff80001e009000ae009000ac140700000f780037
:10ff9000230020009e8f110005003a00e1eb2000b5
:10ffa0000000eb00f6500200000000001e8fe80089
:10ffb0001e80e90022002000110009000200d80084
:10ffc00080407800d0eb2000014878001e007800c7
:10ffd000a844020000000000613e21000040eb0048
:10ffe000804878001e007800a8440200000000004d
:10fff0000080fa00000006003800fa0030df200020
:020000040001f9
:10000000104078000080fb0001002000008fbe003f
:100010001e00be00c808dd000080fd0080407800a2
:100020000040eb00008fbe0040df20001040780051
:100030000080fb00010020001e0f40005e9748007a
:100040001e00be00c808dd000080fd008040780072
:100050000040eb00008fbe0050df20001040780011
:100060000080fb00010020001e0f40005e9748004a
:100070001e00be00c808dd000080fd008040780042
:100080000040eb00008fbe0060df200010407800d1
:100090000080fb00010020001e0f40005e9748001a
:1000a000809f8000919f800000017800810178008e
:1000b0001e0078009e009000000161000180610038
:1000c0006102b80024079800350798002e009000c0
:1000d000be009000c000dd00000020002007980056
:1000e000310798002e009000be0090006112b80009
:1000f00024079800350798002e019000be0190005b
:100100000200700083807000008fbe001e00be00e1
:100110000081ea008181ea00609e8000719e80007b
:100120000000710081807100609e8800719e8800cf
:100130001e00be00cb09dd004500de00008071001e
:10014000c508de00610060000004e00032003200fb
:10015000609e8000719e8000f2fd2f00f3ff2f0053
:1001600000027800810278000200780083007800a5
:1001700000016200018062006102b800440798003b
:10018000550798004e009000de009000c000dd0092
:100190000000200040079800510798004e00900092
:1001a000de0090006112b8004407980055079800df
:1001b0004e019000de01900002007000838070000c
:1001c000609e8800719e8800a29e8000b39e800081
:1001d00000022000010020000000710081807100f9
:1001e000a09e8800b19e8800c29e8000d39e8000a1
:1001f00000042000010020000000710081807100d7
:10020000c09e8800d19e88000000eb0080a7880077
:100210000000eb00e0a888001e00be00c109dd0060
:100220004f00de0000807100cf08de00610060003a
:100230000004e00032003200609e8000719e800069
:10024000f2ff2700f3ff2f00000278008102780000
:1002500002007800830078000001620001806200e3
:100260006102b80064079800750798006e0090005e
:10027000fe009000c000dd00000020006007980034
:10028000710798006e009000fe0090006112b800a7
:1002900064079800750798006e019000fe019000b9
:1002a0000200700083807000609e8800719e88004c
:1002b000a29e8000b39e8000000028000100200064
:1002c0000000710081807100a09e8800b19e8800ae
:1002d000c29e8000d39e8000000024000100200008
:1002e0000000710081807100c09e8800d19e88004e
:1002f0000000eb0080a788000000eb00e0a8880069
:1003000040202000010120009e0178001e02900084
:1003100000017800010078000281610000006200a5
:100320006102b800040f9800150f98000e089000a5
:100330009e089000c000dd0000002000000f980023
:10034000110f98000e0890009e0890006112b800ee
:10035000040f9800150f98000e0990009e09900058
:100360000200700083807000e00f5000e08f5800a2
:100370002c003200609e8000719e8000b2df2f0052
:10038000f3fe2f000002780081027800020078005e
:100390008300780000016200018062006102b80001
:1003a000240f9800350f98002e089000be0890008a
:1003b000c000dd0000002000200f9800310f9800e1
:1003c0002e089000be0890006112b800240f98001b
:1003d000350f98002e099000be09900002007000b1
:1003e00083807000609e8800719e8800a09e8000bf
:1003f000b19e80000020a000a09e8800b19e8800d1
:10040000c09e8000d19e80000040a000c09e880059
:10041000d19e88000000eb0090a788000000eb0050
:10042000f0a888001e007800610060000004e00071
:1004300032003200609e8000719e8000e2ff2f003b
:10044000f3ff2f000002780081027800020078009c
:100450008300780000016200018062006102b80040
:10046000440f9800550f98004e089000de08900049
:10047000c000dd0000002000400f9800510f9800e0
:100480004e089000de0890006112b800440f9800fa
:10049000550f98004e099000de0990000200700090
:1004a00083807000609e8800719e8800a29e8000fc
:1004b000b39e800010002000012020000000710089
:1004c00081807100a09e8800b19e8800c29e80003d
:1004d000d39e800000022000010020000000710077
:1004e00081807100c09e8800d19e88000000eb00d2
:1004f000a0a788000000eb0000a988001e00be0035
:100500004908de0001002000610060000004e000f6
:1005100032003200609e8000719e8000f2ff2f004a
:10052000f3df2f00000278008102780002007800db
:100530008300780000016200018062006102b8005f
:10054000640f9800750f98006e089000fe089000e8
:10055000c000dd0000002000600f9800710f9800bf
:100560006e089000fe0890006112b800640f9800b9
:10057000750f98006e099000fe099000020070004f
:1005800083807000609e8800719e8800a29e80001b
:10059000b39e8000100020000120200000007100a8
:1005a00081807100a09e8800b19e8800c29e80005c
:1005b000d39e800000002000110020000000710088
:1005c00081807100c09e8800d19e88000000eb00f1
:1005d000a0a788000000eb0000a988001e00be0054
:1005e0004a08de0001002000610060000004e00015
:1005f00032003200609e8000719e8000f2ff2f006a
:10060000f3bf2f000002780081027800020078001a
:100610008300780000016200018062006102b8007e
:1006200004179800151798000e1090009e10900067
:10063000c000dd000000200000179800111798008e
:100640000e1090009e1090006112b80004179800e0
:10065000151798000e1190009e1190000200700076
:1006600083807000609e8800719e8800a29e80003a
:10067000b39e8000000020000140200000007100b7
:1006800081807100a09e8800b19e8800c29e80007b
:10069000d39e8000000021000100200000007100b6
:1006a00081807100c09e8800d19e88000000eb0010
:1006b000b0a788000000eb0010a988001e00be0053
:1006c000c609dd004a00de0000807100ca08de00b5
:1006d000610060000004e00032003200609e800093
:1006e000719e8000f2bf2f00f3ff2f000002780000
:1006f0008102780002007800830078000001620027
:10070000018062006102b800241798003517980034
:100710002e109000be109000c000dd0000002000f0
:1007200020179800311798002e109000be109000ee
:100730006112b80024179800351798002e11900008
:10074000be1190000200700083807000609e8800df
:10075000719e8800a29e8000b39e80000040200011
:10076000010020000000710081807100a09e8800bf
:10077000b19e8800c29e8000d39e800000102000a1
:10078000010020000000710081807100c09e88007f
:10079000d19e88000000eb00c0a788000000eb009d
:1007a00020a988001e00be004208de0001002000d3
:1007b000610060000004e00032003200609e8000b2
:1007c000719e8000f2ff2f00b3ff2f00000278001f
:1007d0008102780002007800830078000001620046
:1007e000018062006102b800441798005517980014
:1007f0004e109000de109000c000dd0000002000d0
:1008000040179800511798004e109000de1090008d
:100810006112b80044179800551798004e119000c7
:10082000de1190000200700083807000609e8800de
:10083000719e8800a29e8000b39e80000000200070
:10084000410020000000710081807100a09e88009e
:10085000b19e8800c29e8000d39e800000002800c8
:10086000010020000000710081807100c09e88009e
:10087000d19e88000000eb00e0a788000000eb009c
:1008800040a988001e00be004308de0001002000d1
:10089000610060000004e00032003200609e8000d1
:1008a000719e8000f2ff2f0073ff2f00000278007e
:1008b0008102780002007800830078000001620065
:1008c000018062006102b8006417980075179800f3
:1008d0006e109000fe109000c000dd0000002000af
:1008e00060179800711798006e109000fe1090002d
:1008f0006112b80064179800751798006e11900087
:10090000fe1190000200700083807000609e8800dd
:10091000719e8800a29e8000b39e8000000020008f
:10092000810020000000710081807100a09e88007d
:10093000b19e8800c29e8000d39e800000002000ef
:10094000110020000000710081807100c09e8800ad
:10095000d19e88000000eb00f0a788000000eb00ab
:1009600050a988001e00be004508de0001002000de
:10097000610060000004e00030003200609e8000f2
:10098000719e8000f2ff2f00f3fd2f00000278001f
:100990008102780002007800830078000001620084
:1009a000018062006102b800041f9800151f9800c2
:1009b0000e1890009e189000c000dd00000020007e
:1009c000001f9800111f98000e1890009e189000ac
:1009d0006112b800041f9800151f98000e199000ae
:1009e0009e1990000200700083807000609e880055
:1009f000719e8800a29e8000b39e800000002000af
:100a0000010220000000710081807100a09e88001a
:100a1000b19e8800c29e8000d39e8000000020000e
:100a2000210020000000710081807100c09e8800bc
:100a3000d19e88000000eb0070a988001e00be0057
:100a40004708de0001002000610060000004e000b3
:100a500030003200609e8000719e8000f2ff2f0007
:100a6000f3f72f000002780081027800020078007e
:100a70008300780000016200018062006102b8001a
:100a8000241f9800351f98002e189000be18900063
:100a9000c000dd0000002000201f9800311f9800da
:100aa0002e189000be1890006112b800241f980004
:100ab000351f98002e199000be199000020070009a
:100ac00083807000609e8800719e8800a29e8000d6
:100ad000b39e80000000200001082000000071008b
:100ae00081807100a09e8800b19e8800c29e800017
:100af000d39e800000002000410020000000710013
:100b000081807100c09e8800d19e88000000eb00ab
:100b100080a98800d2eb20001e00be00da5002003f
:100b20000000000050c0b300a84402000000000014
:100b30000080fa00000006000a00fa0030df200002
:100b4000104078000080fb00b0e88800b0e880002a
:100b50004800dd00b0e88800b1e8800040df2000f8
:100b6000104078000080fb0000804000b0e8880062
:100b70000080eb00400798005ef8020001000000d2
:100b80002007980031079800a2a68000b3a6800035
:100b90002e009000be009000021f500003975800e6
:100ba0001e00be00e00f5000e08f580004003d0022
:100bb00000a82300910020001e0f40005e9748000f
:100bc00070bb200001002000be0f1000ae8f180087
:100bd00003003c001e0078006a00b900400798003e
:100be000d1eb20004e009000f65002000000000003
:100bf000e0e8800080407800f0eb200001487800b9
:100c0000d0e880008040780000ec200001487800a7
:100c100012ec2000f0e8800001e98000da500200c8
:100c20000000000051ec200010e98000f6500200a6
:100c30000000000072ec200020e9800031e9800013
:100c4000da50020000000000b2ec200040e9800011
:100c500051e98000da50020000000000f1ec2000b1
:100c600060e98000f65002000000000012ed200054
:100c700070e9800081e98000da5002000000000085
:100c800052ed200090e98000a1e98000da500200d6
:100c900000000000d0c1b300a84402000000000022
:100ca00030002000c0e888000080fa000000060044
:100cb0000800fa0030df2000104078000080fb00c0
:100cc0000000e9002007980040df20001040780075
:100cd0000080fb00300798000000eb001007980030
:100ce000130037001e009000e300400020df2000ca
:100cf000614f7800f0c1b3009e4f10000500360030
:100d00009e00900020df20001e4178008270780055
:100d1000040037001e01900021df20000040eb009e
:100d200000f178001e0090000000e8001007980015
:100d30009e0090002e009000808f5000e9ff35004b
:100d40001e01900021df20000040eb0000f1780040
:100d5000109f80004c00de00610060000004e00095
:100d60000300320021df20003e0090000500070054
:100d700010c0b300a8440200000000000080fa0088
:100d8000000006000800fa00881f7800200798007d
:100d900031079800119f8000f0ff2e000080600056
:100da000109f8800019f8000f0ff2b0000806000f2
:100db000009f88000000eb00000f78000000eb00af
:100dc000100798001e009000800078003e00900000
:100dd0000080400090407800a0c3b30080cf500056
:100de000080032001e009000800078003e00900055
:100df0000080400090407800c0c2b30080cf500017
:100e000014003a001e0090000000e800100798004f
:100e10001e009000800078003e009000008040009e
:100e2000104078000000fb003e0c020000000000b3
:100e30000000e000070032001e00900080007800f3
:100e40003e00900000804000104078000000fb0051
:100e5000000f78001e0090000000e80010079800c6
:100e60001e0490003e009000ce1b02000000000017
:100e7000800f5400020031001e00e000d1ff32005c
:100e8000600420009e0f10000d003a00309c80008e
:100e90000000e800309c8800019f800000002800ce
:100ea00000807000009f8800209e80007e0040002f
:100eb000709c8800309c8000e20f50005b00340082
:100ec0002e009000e20f500039003a00e0042000ac
:100ed0009e0f10001b003a00719b800022372100fa
:100ee0000180400002004000100078008001e9000d
:100ef00022372100018040000200400003087800f2
:100f0000709b80002137210000004000010040005c
:100f1000100078000000e00008003c00709b80009a
:100f20000000e800709b8800709b8000e30f500079
:100f3000020034000000eb00709b88000000eb0012
:100f4000309c8800100420009e0f10000a003a0018
:100f5000709b80000000e800709b8800709b800000
:100f6000e30f5000020034000000eb00709b88008b
:100f70000000eb00309c8800f00420009e0f100061
:100f80002a003a00709b80000000e800709b8800f7
:100f9000709b8000e30f5000020034000000eb0063
:100fa000709b88000000eb00309c88001f00370019
:100fb0002e009000e30f500012003a003e00900017
:100fc000801f7800a01a2c00801f7800da1f020012
:100fd00000000000e4875700709b80000000e800dc
:100fe000709b8800709b8000e30f5000020034006b
:100ff0000000eb00709b88000000eb00309c880034
:101000000a003700709b80000000e800709b880099
:10101000709b8000e30f5000020034000000eb00e2
:10102000709b88000000eb00309c88004f04780023
:101030000080fa00000006000600fa00c0df200071
:10104000904078000039210001487800d0df20006e
:10105000904078001039210001487800e0df20003e
:101060009040780020392100014878000040eb00d2
:10107000504798000040eb0040479800201820009f
:10108000e83e020000000000100798001e009000db
:101090000000e0000b00340010c0b300404798008f
:1010a00040df2000104078000080fb00000f780037
:1010b0001e0090009e0f50000200310010c0b300cf
:1010c0005047980040182000e83e02000000000051
:1010d000100798001e0090000000e0000b00340094
:1010e00010c0b3004047980050df20001040780047
:1010f0000080fb00000f78001e0090009e0f500043
:101100000200360010c0b300504798004e409000d7
:101110000004e00008003a0060df20001040780082
:101120000080fb00000f78001e00e000020032008b
:1011300010c0b3005047980070df200010407800c6
:101140000004e000020032000040eb00504798002d
:101150005e4090000004e00005003200100007002f
:10116000e1eb200010c0b300804878000400370095
:101170004b000700e1eb20000040eb0080487800c6
:10118000d1eb200010c0b3008048780030c0b3001d
:10119000a8440200000000000080fa0000000600e1
:1011a0000800fa00009f80004d00de000000a20051
:1011b000610060000004e0001f00320002860200af
:1011c000010000000004e0001b003200f2ff2f00cd
:1011d000f3ff2700100020000100200050bb020098
:1011e000010000000e007800c8ff020001000000ae
:1011f0000e007800eaf502000100000060ea8800b5
:1012000071ea880060ea800071ea8000e47a0200f6
:101210000100000010c0b300ec85020001000000d6
:10122000f2ff2f00f3ff2700100020000100200034
:10123000dcbb020001000000019f800000002200d2
:1012400000807000009f88000000eb00e0a888008c
:101250000000eb00f0a888000000eb0000a9880067
:101260000000eb0010a988000000eb0020a9880016
:101270000000eb0030a988000000eb0040a98800c6
:101280000000eb0050a988000000eb0070a9880066
:101290000000eb0080a988000080fa000000060032
:1012a0000000fa00009f8000f1ff2d0001006000a7
:1012b000009f88000080fa00000006000000fa008d
:1012c00031df200030df2000104078000080fb007c
:1012d000c683020001000000219f80000000210061
:1012e00000807000209f88000080fa000000060047
:1012f0003800fa0040df2000104078000080fb003a
:10130000c800dd0050df2000104078000080fb00a6
:10131000008040001007980010002000000f7800a7
:101320000000eb00200798000b0037002e01900012
:101330009e00780020df2000e14078006600470032
:1013400000004100014878001e0fe8002e009000c8
:101350000000e800200798001e009000e300400015
:101360002e009000808f5000f0ff3e001e00900085
:10137000e30040006600470068d80200010000005a
:101380002007980010002000000f78000000eb00fc
:10139000100798000b0037001e0178009e00900097
:1013a000660047000080400090407800c0eb2000bd
:1013b000017178001e0fe8001e0090000000e80098
:1013c000100798009e0090002e009000808f500023
:1013d000f1ff39002e0090000040e800a844020010
:1013e000000000000080fa00000006002a00fa0059
:1013f000881f78002e4c0200000000000004e0006e
:1014000041003200809b8000a13721000000400095
:10141000810040002000200080087800eb030700d6
:10142000000f7800f0eb2000104078008080fb0077
:10143000e0eb2000104078000081fb00d0eb2000a2
:10144000104078008081fb0000ec20001040780004
:101450000082fb0030ec2000104078008082fb000e
:1014600020ec2000104078000083fb0010ec2000ee
:10147000104078008083fb00c0eb20001040780013
:101480000080fb000e84e800811f7800821f780036
:10149000831f7800841f7800851f7800861f7800de
:1014a000871f7800801f7800803a2c00801f78000a
:1014b00008007800f81f020000000000f2875700c3
:1014c0008e80e8001e00780019040700000f7800e5
:1014d000809b8000213721000000400081004000f7
:1014e0001000200080087800809b80000000e80049
:1014f000809b8800809b8000e30f50000200340036
:101500000000eb00809b88004f0478000080fa0008
:10151000000006001a00fa002e4c02000000000035
:101520000004e00065003200809b8000a1372100ac
:10153000000040008100400020002000800878006a
:10154000a203070020079800c0eb2000104078009d
:101550000080fb00e6004700801f7800103d2c0053
:10156000801f780001007800f81f020000000000d2
:10157000e4875700e60047002e009000ec030700c8
:1015800020079800e0eb2000ea5002000000000075
:1015900010079800610c20002e0090008080500001
:1015a0001e009000808f500018003d00660047002c
:1015b000613d2c000e00090031587800f000b100a8
:1015c000e60047002e009000d9030700200798008e
:1015d000809b8000213721000000400081004000f6
:1015e0001000200080087800809b80000000e80048
:1015f000809b8800809b8000e30f50002f00340008
:101600000000eb00809b88002c0037000000eb00fe
:10161000000f780010003700829b8000ae01900020
:101620001e007800e4004000c0eb2000614078001c
:1016300000427800800c20000090b9008300400038
:10164000e0042100847078002e0090000000e80083
:10165000200798001e0fe8001e0090009e0f10004b
:10166000edff3500819b80002e019000800c200052
:101670000088b90002014000e10421000040eb00b5
:1016800000f17800809b800021372100000040009d
:10169000810040001000200080087800809b8000be
:1016a0000000e800809b8800809b8000e30f5000d2
:1016b000020034000000eb00809b88000080fa00ec
:1016c000000006006e00fa00889fbe008a9fbe00e0
:1016d0002e4c0200000000000004e0004402320032
:1016e0003a030700300f9800e0eb2000104078002c
:1016f0000080fb00000f78001e0078004800dd002d
:10170000000f7800f0eb2000104078000080fb0014
:101710001e0f400000ec2000ea5002000000000014
:10172000200f98002e0890000000e0000c003d0003
:10173000c0eb2000104078000080fb00f80047005c
:10174000801f7800503e2c00801f78000100780038
:10175000f81f020000000000e48757001d0037005a
:101760002e089000cf80de006e0c0200000000000a
:101770000200200003122400e80d02000000000017
:1017800060079800710798006e009000fe009000be
:101790003e0f0200000000000002be000203be0077
:1017a000c0eb2000104078000080fb00f8004700ec
:1017b000849fbe00869fbe00801f7800603f2c0083
:1017c000801f780001007800f81f02000000000070
:1017d000ec875700f80047003e08900054030700cc
:1017e000300f98007800470091402c000d00090050
:1017f00031587800e000b1001e0078006101b800a7
:101800000080eb008080eb000201400083814800f3
:101810001237980023379800b00020000100200004
:101820001e319000ae319000800f5100818f590021
:10183000dd013e001e309000ae30900000600100df
:101840000b003700260037003800370054003700ff
:10185000d501370084003700d3013700d2013700ab
:10186000dd0037003801370093013700bc01370035
:1018700020ec2000ea50020000000000200f980039
:101880002e089000cf80de006e0c020000000000e9
:1018900002002000832c2400e80d0200000000005c
:1018a00060079800710798006e009000fe0090009d
:1018b0003e0f02000000000078024700809fbe003b
:1018c000829fbe0070412c00801f780004007800c9
:1018d000f81f020000000000ea875700b20137003d
:1018e00020ec2000c65002000000000060079800b5
:1018f000710798006e009000fe0090003e0f0200fd
:101900000000000078024700809fbe00829fbe005a
:1019100020422c00801f780004007800f81f02008d
:1019200000000000ea8757009f01370020ec2000ec
:10193000c650020000000000000f9800110f980030
:101940000e0890009e0890006e0c0200000000003f
:1019500002002000a3472400e80d02000000000060
:1019600060079800710798006e009000fe009000dc
:101970003e0f02000000000078024700809fbe007a
:10198000829fbe00b0422c00801f780004007800c7
:10199000f81f020000000000ea87570082013700ac
:1019a00020ec2000ea50020000000000200f980008
:1019b0002e089000cf80de006e0c020000000000b8
:1019c00002002000a3472400e80d020000000000f0
:1019d000600798007107980040ec2000ea50020070
:1019e00000000000200f98002e089000cf80de003d
:1019f0006e0c02000000000002002000a34724003b
:101a0000e80d020000000000400798005107980010
:101a10002e009000be0090003e0f0200000000006b
:101a20000004be000205be004e009000de009000e3
:101a30003e0f02000000000078024700889fbe00b1
:101a40008a9fbe00809fbe00829fbe0040432c0044
:101a5000801f780004007800f81f020000000000da
:101a6000f28757005001370040ec2000ea50020096
:101a700000000000100798002e089000cf80de00c4
:101a80006e0c02000000000002002000832c2400e5
:101a9000e80d020000000000600798007107980040
:101aa00020ec2000ea50020000000000100798001f
:101ab00060ec2000ea50020000000000200f9800b7
:101ac0002e089000cf80de006e0c020000000000a7
:101ad00002002000832c2400e80d0200000000001a
:101ae000400798005107980080ec2000ea5002005f
:101af00000000000200f98002e089000cf80de002c
:101b00006e0c02000000000002002000832c240064
:101b1000e80d02000000000020079800310798003f
:101b20002e009000be0090003e0f0200000000005a
:101b3000502f9800612f9800722f9800033798005b
:101b40004e009000de0090003e0f020000000000fa
:101b50000004be000205be004e009000de009000b2
:101b60003e0f020000000000303798004137980017
:101b70005237980063379800780247009e00900023
:101b8000811f78005e289000ee2890007e2990004a
:101b90008e319000809fbe00829fbe00889fbe0055
:101ba0008a9fbe003e309000ce3090005e319000a3
:101bb000ee319000809fbe00829fbe0030452c0019
:101bc000801f780004007800f81f02000000000069
:101bd000fc875700f400370040ec2000ea50020078
:101be00000000000100798002e089000cf80de0053
:101bf0006e0c02000000000002002000832c240074
:101c0000e80d0200000000006007980071079800ce
:101c100020ec2000ea5002000000000010079800ad
:101c200060ec2000ea50020000000000200f980045
:101c30002e089000cf80de006e0c02000000000035
:101c400002002000832c2400e80d020000000000a8
:101c5000400798005107980080ec2000ea500200ed
:101c600000000000200f98002e089000cf80de00ba
:101c70006e0c02000000000002002000832c2400f3
:101c8000e80d0200000000002007980031079800ce
:101c90002e009000be0090003e0f020000000000e9
:101ca000102f9800212f9800322f9800432f980072
:101cb0004e009000de0090003e0f02000000000089
:101cc0000004be000205be004e009000de00900041
:101cd0003e0f0200000000003037980041379800a6
:101ce0005237980063379800780247009e009000b2
:101cf000811f78001e289000ae2890003e29900099
:101d0000ce299000809fbe00829fbe00889fbe00ab
:101d10008a9fbe003e309000ce3090005e31900031
:101d2000ee319000809fbe00829fbe0030452c00a7
:101d3000801f780004007800f81f020000000000f7
:101d4000fc8757009800370020ec2000ea50020082
:101d5000000000001007980040ec2000ea5002004c
:101d600000000000200f98002e089000cf80de00b9
:101d70006e0c02000000000002002000a3472400b7
:101d8000e80d02000000000060079800710798004d
:101d900060ec2000ea50020000000000200f9800d4
:101da0002e089000cf80de006e0c020000000000c4
:101db00002002000a3472400e80d020000000000fc
:101dc000400798005107980080ec2000ea5002007c
:101dd00000000000200f98002e089000cf80de0049
:101de0006e0c02000000000002002000a347240047
:101df000e80d02000000000020079800310798005d
:101e00002e009000be0090003e0f02000000000077
:101e1000502798006127980072279800032f980098
:101e20004e009000de0090003e0f02000000000017
:101e30000004be000205be004e009000de009000cf
:101e40003e0f020000000000303798004137980034
:101e50005237980063379800780247009e00900040
:101e6000811f78005e209000ee2090007e2190007f
:101e70008e299000809fbe00829fbe00889fbe007a
:101e80008a9fbe003e309000ce3090005e319000c0
:101e9000ee319000809fbe00829fbe00b0482c00b3
:101ea000801f780004007800f81f02000000000086
:101eb000fc8757003c00370020ec2000c650020091
:101ec00000000000000f9800110f98000e0890000d
:101ed0009e0890006e0c020000000000020020002e
:101ee000a3472400e80d02000000000060079800ee
:101ef0007107980060ec2000c6500200000000004e
:101f000040079800510798004e009000de009000b6
:101f10003e0f0200000000000004be000205be00eb
:101f20006e009000fe0090003e0f020000000000d6
:101f300078024700889fbe008a9fbe00809fbe0037
:101f4000829fbe00e04b2c00801f780004007800c8
:101f5000f81f020000000000f2875700120037004f
:101f600020ec2000c650020000000000600798002e
:101f7000710798006e009000fe0090003e0f020076
:101f80000000000078024700809fbe00829fbe00d4
:101f9000204d2c00801f780004007800f81f0200fc
:101fa00000000000ea875700f80047003e08900054
:101fb0005f010700300f9800809b800021372100cf
:101fc00000004000810040001000200080087800e0
:101fd000809b80000000e800809b8800809b800040
:101fe000e30f5000020034000000eb00809b8800eb
